:100000004BC0000042C2000040C200003EC20000DF
:100010003CC200000C94BA6738C2000036C200002F
:1000200034C2000032C200000C94B0670C94A66782
:100030002CC200002AC2000028C2000026C2000014
:1000400024C2000022C2000020C200001EC2000024
:100050001CC200000C94666818C2000016C20000A2
:1000600014C2000012C2000010C200000EC2000044
:100070000CC200000AC2000008C2000006C2000054
:1000800004C2000002C2000000C20000FEC1000065
:10009000FCC10000FAC1000011241FBECFEFD0E266
:1000A000DEBFCDBF0E9400F0D7C10000076342361B
:1000B000B79BD8A71A39685618AEBAAB558C1D3CF9
:1000C000B7CC5763BD6DEDFD753EF6177231BF00BD
:1000D0000000803F05A84CCDB2D44EB93836A902F5
:1000E0000C50B9918688083CA6AAAA2ABE00000036
:1000F000803F08000000BE922449123EABAAAA2A03
:10010000BECDCCCC4C3E00000080BEABAAAAAA3E1D
:1001100000000000BF000000803F00000000000859
:100120004178D3BB4387D1133D190E3CC3BD4282F6
:10013000AD2B3E68EC8276BED98FE1A93E4C80EFB4
:10014000FFBE01C4FF7F3F0000000000FF004C8A9B
:1001500097509545406BA6D8E4B2282EAE90BF26A6
:10016000B14EE86FD0FBE0709A51862C379845323B
:10017000539D06840D971A8CE61E2E0DB41D401655
:100180009AC591F9F786A142660620AFAE19EE270F
:10019000C2BB0EBAB90AAA95CA45040444C1796A19
:1001A00091EE7D3E2E4C960BA96E5A6A9FF56D0519
:1001B000BB8F808DB4F54FC14AE99E674536394FF4
:1001C00075ADF44CB227A939D78036F7C49C7E6A46
:1001D000605F677992B4DD0E4786CD1A6DC6258AB9
:1001E000F464D953D154DB67F78B22BD5CFEA44D78
:1001F000F9A7590EC57E3BF9BA7D430AD39F6C3BE4
:100200000BDEB2875E3710ECC8A6856546290CF177
:10021000D6BCA38C755E4934200DFAE9D7C7B6A7C2
:10022000988A7C6E6155493D32271D1209FFF6EE12
:10023000E5DDD5CEC6BFB9B2ACA6A09A958F8A85AA
:10024000817C78736F6B6864605D5A56FF59E97DF5
:1002500015B150F39942EE9D4F04BC7632F1B2765F
:100260003B03CC98653405D8AC8259320CE7C4A264
:100270008161432509EDD3B9A089725C46321E0B1A
:10028000F8E6D5C4B4A596887A6D6053473C30260D
:100290001B1108FEF5EDE4DCD4CDC6BFB8B1ABA5AB
:1002A0009F99948F8A85807C77736F6B6763605D9D
:1002B000595653504D4A484543403E3C3A383634EF
:1002C00032302E2D2B2A282725242321201F1E1DC6
:1002D0001C1B1A19181716161514131312111110C6
:1002E0000F0F0E0E0D0D0C0C0B0B0B0A0A09090952
:1002F0000808080807070706060606060505050597
:1003000005040404040404030303030303030302B6
:1003100002020202020202020202010101010101C3
:1003200001010101010101010101010101000000C0
:1003300000000000000000000000000000000000BD
:10034000000000000000000000000000FF0C0B0B8C
:100350000B0A0A090909080808080707070606061C
:100360000606050505050504040404040403030347
:100370000303030303020202020202020202020258
:10038000010101010101010101010101010101015D
:10039000010101000000000000000000000000005A
:1003A000000000000000000000000000000000004D
:1003B000000000000000000000000000000000003D
:1003C000000000000000000000000000000000002D
:1003D000000000000000000000000000000000001D
:1003E000000000000000000000000000000000000D
:1003F00000000000000000000000000000000000FD
:1004000000000000000000000000000000000000EC
:1004100000000000000000000000000000000000DC
:1004200000000000000000000000000000000000CC
:1004300000000000000000000000000000000000BC
:1004400000000000000000000000000011241FBE9A
:10045000CFEFD0E2DEBFCDBF1AE1A4EAB9E001C020
:100460001D92AC38B107E1F719E0A0E0B1E0ECED86
:10047000FBEE00E00BBF02C007900D92A43AB1075B
:10048000D9F70E949F680C94EC75BACD2F923F92D9
:100490004F925F926F927F928F929F92AF92BF9294
:1004A000CF92DF92EF92FF920F931F93CF93DF9340
:1004B00000D01F92CDB7DEB78AE090E10E94FA200B
:1004C00080903B1090903C102091D41020FF15C0DC
:1004D00025FD02C00C94EF0D640124FD0FC0809136
:1004E00020109091211095958795880E991E21FDD9
:1004F00007C0412C512C32010BC0640121FFF9CF00
:100500004090201050902110662457FC6094762C67
:100510000091F5101091F61020E030E010582109FC
:1005200031098091D010882311F40C94EB0D809147
:10053000071190910811A0E0B0E09058A109B1090D
:10054000B7FF02C00C942E10B595A7959795879587
:100550009B838A833FB73983F8948091160E9091DC
:10056000170EA091180EB091190E8B2F9927AA275C
:10057000BB27892B8A2B8B2B21F082E19EE00E94E6
:10058000102080913B0E823011F40C943B0C10F043
:100590000C94340C813011F40C94FA0C80E090E04F
:1005A0006091340E7091350E0E9484192090320EA5
:1005B0003090330E280E391E3092370E2092360EB0
:1005C0008091120E9091130EA091140EB091150E01
:1005D0004091160E5091170E6091180E7091190EE1
:1005E000840F951FA61FB71F8093160E9093170EAA
:1005F000A093180EB093190EEE24D7FCE094FE2CB5
:10060000AA2497FCA094BA2C80914C1090914D1084
:10061000B501A401480F591F611D711D41155105F8
:1006200081E06807710524F04FEF5FEF60E070E054
:10063000DB01CA0177FF02C00C94950D0E94332B99
:1006400046EC41BB469A31E035B925E428B950EF74
:100650005BB992EA9EB987E881BB00C000C041BB8C
:10066000469A35B928B960ED6BB99EB981BB00C017
:1006700000C041BB469A35B928B95BB99EB981BB68
:100680004A815B81B101AA27469FB12D5703900192
:10069000749FB00D211D3A1F56033A0BB00D211D5A
:1006A0003A1F1124A901662757FD6095762F4C0D3E
:1006B0005D1D6E1D7F1D8091401090914110480F6F
:1006C000591F611D711D4115510581E068077105B4
:1006D00024F04FEF5FEF60E070E0DB01CA0177FFCD
:1006E00002C00C94900D0E94332B46EC41BB469AFD
:1006F00031E035B921E428B950EF5BB990EA9EB9F1
:1007000087E881BB00C000C041BB469A35B928B913
:1007100060ED6BB99EB981BB00C000C041BB469A79
:1007200035B928B95BB99EB981BB9101AA27029F4F
:10073000B12D1303C001309FB00D811D9A1F12030C
:100740009A0BB00D811D9A1F1124AA2797FDA09521
:10075000BA2F840D951DA61DB71D209158103091FC
:100760005910820F931FA11DB11D20918810309147
:100770008910A90160E070E0481759076A077B07F4
:100780000CF0E4C7CA010E94332B46EC41BB469AE9
:1007900031E035B921E428B950EF5BB992EA9EB94E
:1007A00087E881BB00C000C041BB469A35B928B973
:1007B00060EE6BB99EB981BB00C000C041BB469AD8
:1007C00035B928B95BB99EB981BB8091120F909160
:1007D000130FA091140FB091150F8B2F9927AA27F3
:1007E000BB27892B8A2B8B2B11F00C94B30C809197
:1007F000370F823011F40C94220C10F00C941B0C67
:10080000813011F40C94640D80E090E06091300F21
:100810007091310F0E94841920912E0F30912F0F6B
:10082000280F391F3093330F2093320F80910E0F12
:1008300090910F0FA091100FB091110F4091120FD6
:100840005091130F6091140F7091150F840F951F25
:10085000A61FB71F8093120F9093130FA093140F2E
:10086000B093150F2115310511F00C94CC0C80E0DC
:1008700090E00E94332B46EC41BB469A31E035B9FB
:1008800025E428B950EF5BB990EA9EB987E881BBAF
:1008900000C000C041BB469A35B928B960EB6BB9BE
:1008A0009EB981BB00C000C041BB469A35B928B98A
:1008B0005BB99EB981BB39813FBF3FB73983F8949B
:1008C0008091400E9091410EA091420EB091430E46
:1008D0008B2F9927AA27BB27892B8A2B8B2B11F0CB
:1008E0000C94C60C8091650E823009F493C708F011
:1008F0008BC7813011F40C944E0D80E090E0609134
:100900005E0E70915F0E0E94841920905C0E3090F4
:100910005D0E280E391E3092610E2092600E80917D
:100920003C0E90913D0EA0913E0EB0913F0E409135
:10093000400E5091410E6091420E7091430E840F13
:10094000951FA61FB71F8093400E9093410EA09352
:10095000420EB093430E80914E1090914F10B5010E
:10096000A401480F591F611D711D4115510581E0FA
:100970006807710524F04FEF5FEF60E070E0DB0186
:10098000CA0177FF02C00C947F0D0E94332B46EC06
:1009900041BB469A31E035B927E428B950EF5BB93D
:1009A00092EA9EB987E881BB00C000C041BB469A6D
:1009B00035B928B960ED6BB99EB981BB00C000C0E4
:1009C00041BB469A35B928B95BB99EB981BB4A810A
:1009D0005B81B101AA27469FB12D57039001749FF7
:1009E000B00D211D3A1F56033A0BB00D211D3A1FC1
:1009F0001124A901662757FD6095762F4C0D5D1DCA
:100A00006E1D7F1D8091421090914310480F591F19
:100A1000611D711D4115510581E06807710524F0C4
:100A20004FEF5FEF60E070E0DB01CA0177FF02C0CB
:100A30000C949E0D0E94332B46EC41BB469A31E04C
:100A400035B923E428B950EF5BB990EA9EB987E83D
:100A500081BB00C000C041BB469A35B928B960EDE2
:100A60006BB99EB981BB00C000C041BB469A35B985
:100A700028B95BB99EB981BB9101AA27029FB12D0C
:100A80001303C001309FB00D811D9A1F12039A0BF2
:100A9000B00D811D9A1F1124AA2797FDA095BA2F8A
:100AA000840D951DA61DB71D20915A1030915B1025
:100AB000820F931FA11DB11D20918A1030918B10C0
:100AC000A90160E070E0481759076A077B070CF03E
:100AD00042C6CA010E94332B46EC41BB469A31E024
:100AE00035B923E428B950EF5BB992EA9EB987E89B
:100AF00081BB00C000C041BB469A35B928B960EE41
:100B00006BB99EB981BB00C000C041BB469A35B9E4
:100B100028B95BB99EB981BB80913C0F90913D0F84
:100B2000A0913E0FB0913F0F8B2F9927AA27BB278B
:100B3000892B8A2B8B2B09F0EFC68091610F8230B5
:100B400009F4B1C608F0A9C6813009F47FC780E076
:100B500090E060915A0F70915B0F0E948419209170
:100B6000580F3091590F280F391F30935D0F209384
:100B70005C0F8091380F9091390FA0913A0FB0918E
:100B80003B0F40913C0F50913D0F60913E0F709193
:100B90003F0F840F951FA61FB71F80933C0F9093A4
:100BA0003D0FA0933E0FB0933F0F2115310509F083
:100BB000ABC680E090E00E94332B46EC41BB469AE6
:100BC00031E035B927E428B950EF5BB990EA9EB916
:100BD00087E881BB00C000C041BB469A35B928B93F
:100BE00060EB6BB99EB981BB00C000C041BB469AA7
:100BF00035B928B95BB99EB981BB39813FBF2FB7E1
:100C00002983F89480916A0E90916B0EA0916C0EDE
:100C1000B0916D0E8B2F9927AA27BB27892B8A2B82
:100C20008B2B09F06CC680918F0E823009F454C66C
:100C300008F04CC6813009F4EDC680E090E0609188
:100C4000880E7091890E0E9484192090860E309033
:100C5000870E280E391E30928B0E20928A0E8091BC
:100C6000660E9091670EA091680EB091690E40914A
:100C70006A0E50916B0E60916C0E70916D0E840F28
:100C8000951FA61FB71F80936A0E90936B0EA093BB
:100C90006C0EB0936D0E8091501090915110B50173
:100CA000A401480F591F611D711D4115510531E007
:100CB0006307710524F04FEF5FEF60E070E0DB0148
:100CC000CA0177FD37C70E94332B46EC41BB469AD9
:100CD00031E035B921E428B950EF5BB990EA9EB90B
:100CE00087E881BB00C000C041BB469A35B928B92E
:100CF00060EE6BB99EB981BB00C000C041BB469A93
:100D000035B928B95BB99EB981BB4A815B81B10114
:100D1000AA27469FB12D57039001749FB00D211D46
:100D20003A1F56033A0BB00D211D3A1F1124A90199
:100D3000662757FD6095762F4C0D5D1D6E1D7F1D3E
:100D40008091441090914510480F591F611D711DED
:100D50004115510581E06807710524F04FEF5FEF01
:100D600060E070E0DB01CA0177FDEDC60E94332B25
:100D700046EC41BB469A31E035B925E428B950EF3D
:100D80005BB990EA9EB987E881BB00C000C041BB57
:100D9000469A35B928B960ED6BB99EB981BB00C0E0
:100DA00000C041BB469A35B928B95BB99EB981BB31
:100DB0009101AA27029FB12D1303C001309FB00DEE
:100DC000811D9A1F12039A0BB00D811D9A1F1124C9
:100DD000AA2797FDA095BA2F840D951DA61DB71DB6
:100DE00020915C1030915D10820F931FA11DB11DE9
:100DF00020918C1030918D10A90160E070E04817AF
:100E000059076A077B070CF0ABC4CA010E94332B59
:100E100046EC41BB469A31E035B925E428B950EF9C
:100E20005BB992EA9EB987E881BB00C000C041BBB4
:100E3000469A35B928B960EE6BB99EB981BB00C03E
:100E400000C041BB469A35B928B95BB99EB981BB90
:100E500082E69FE00E9436498091860F9091870F2D
:100E6000009709F063C50E94332B46EC41BB469ABC
:100E700031E035B921E428B950EF5BB992EA9EB967
:100E800087E881BB00C000C041BB469A35B928B98C
:100E900060EB6BB99EB981BB00C000C041BB469AF4
:100EA00035B928B95BB99EB981BB29812FBF3FB73E
:100EB0003983F8948091940E9091950EA091960E9E
:100EC000B091970E8B2F9927AA27BB27892B8A2BA6
:100ED0008B2B09F026C58091B90E823009F483C4AA
:100EE00008F07BC4813009F474C580E090E0609123
:100EF000B20E7091B30E0E9484192090B00E309003
:100F0000B10E280E391E3092B50E2092B40E80918B
:100F1000900E9091910EA091920EB091930E4091EF
:100F2000940E5091950E6091960E7091970E840FCD
:100F3000951FA61FB71F8093940E9093950EA093B4
:100F4000960EB093970E8091521090915310B50168
:100F5000A401480F591F611D711D4115510581E004
:100F60006807710524F04FEF5FEF60E070E0DB0190
:100F7000CA0177FDCDC50E94332B46EC41BB469A92
:100F800031E035B923E428B950EF5BB990EA9EB956
:100F900087E881BB00C000C041BB469A35B928B97B
:100FA00060EE6BB99EB981BB00C000C041BB469AE0
:100FB00035B928B95BB99EB981BB4A815B81B10162
:100FC000AA27469FB12D57039001749FB00D211D94
:100FD0003A1F56033A0BB00D211D3A1F1124A901E7
:100FE000662757FD6095762F4C0D5D1D6E1D7F1D8C
:100FF0008091461090914710480F591F611D711D37
:101000004115510581E06807710524F04FEF5FEF4E
:1010100060E070E0DB01CA0177FD7EC50E94332BE2
:1010200046EC41BB469A31E035B927E428B950EF88
:101030005BB990EA9EB987E881BB00C000C041BBA4
:10104000469A35B928B960ED6BB99EB981BB00C02D
:1010500000C041BB469A35B928B95BB99EB981BB7E
:101060009101AA27029FB12D1303C001309FB00D3B
:10107000811D9A1F12039A0BB00D811D9A1F112416
:10108000AA2797FDA095BA2F840D951DA61DB71D03
:1010900020915E1030915F10820F931FA11DB11D32
:1010A00020918E1030918F10A90160E070E04817F8
:1010B00059076A077B070CF058C3CA010E94332BFB
:1010C00046EC41BB469A31E035B927E428B950EFE8
:1010D0005BB992EA9EB987E881BB00C000C041BB02
:1010E000469A35B928B960EE6BB99EB981BB00C08C
:1010F00000C041BB469A35B928B95BB99EB981BBDE
:101100008091900F9091910FA091920FB091930FB9
:101110008B2F9927AA27BB27892B8A2B8B2B09F08A
:101120001DC48091B50F823009F446C308F03EC358
:10113000813009F49FC480E090E06091AE0F70911F
:10114000AF0F0E9484192091AC0F3091AD0F280F82
:10115000391F3093B10F2093B00F80918C0F909175
:101160008D0FA0918E0FB0918F0F4091900F5091E5
:10117000910F6091920F7091930F840F951FA61F8E
:10118000B71F8093900F9093910FA093920FB093FD
:10119000930F2115310509F0F1C380E090E00E9422
:1011A000332B46EC41BB469A31E035B923E428B9EC
:1011B00050EF5BB992EA9EB987E881BB00C000C0DE
:1011C00041BB469A35B928B960EB6BB99EB981BB72
:1011D00000C000C041BB469A35B928B95BB99EB979
:1011E00081BB39813FBF3FB73983F8948091BE0EF0
:1011F0009091BF0EA091C00EB091C10E8B2F992778
:10120000AA27BB27892B8A2B8B2B09F0B2C380918D
:10121000E30E823009F4B9C208F0B1C2813009F49A
:10122000C9C380E090E06091DC0E7091DD0E0E94F9
:1012300084192090DA0E3090DB0E280E391E309281
:10124000DF0E2092DE0E8091BA0E9091BB0EA0911F
:10125000BC0EB091BD0E4091BE0E5091BF0E60917C
:10126000C00E7091C10E840F951FA61FB71F8093EB
:10127000BE0E9093BF0EA093C00EB093C10E80918E
:10128000541090915510B501A401480F591F611DCC
:10129000711D4115510581E06807710524F04FEF7C
:1012A0005FEF60E070E0DB01CA0177FD2DC40E94B2
:1012B000332B46EC41BB469A31E035B925E428B9D9
:1012C00050EF5BB990EA9EB987E881BB00C000C0CF
:1012D00041BB469A35B928B960EE6BB99EB981BB5E
:1012E00000C000C041BB469A35B928B95BB99EB968
:1012F00081BB4A815B81B101AA27469FB12D57036B
:101300009001749FB00D211D3A1F56033A0BB00D8A
:10131000211D3A1F1124A901662757FD6095762FDC
:101320004C0D5D1D6E1D7F1D8091481090914910E0
:10133000480F591F611D711D4115510581E0680756
:10134000710524F04FEF5FEF60E070E0DB01CA0150
:1013500077FDFDC30E94332B46EC41BB469A31E03A
:1013600035B921E428B950EF5BB992EA9EB987E814
:1013700081BB00C000C041BB469A35B928B960EDB9
:101380006BB99EB981BB00C000C041BB469A35B95C
:1013900028B95BB99EB981BB9101AA27029FB12DE3
:1013A0001303C001309FB00D811D9A1F12039A0BC9
:1013B000B00D811D9A1F1124AA2797FDA095BA2F61
:1013C000840D951DA61DB71D2091601030916110F0
:1013D000820F931FA11DB11D20919010309191108B
:1013E000A90160E070E0481759076A077B070CF015
:1013F000C1C1CA010E94332B46EC41BB469A31E081
:1014000035B921E428B950EF5BB990EA9EB987E875
:1014100081BB00C000C041BB469A35B928B960EB1A
:101420006BB99EB981BB00C000C041BB469A35B9BB
:1014300028B95BB99EB981BB86EB9FE00E94364913
:101440008091DA0F9091DB0F009709F077C20E942C
:10145000332B46EC41BB469A31E035B925E428B937
:1014600050EF5BB992EA9EB987E881BB00C000C02B
:1014700041BB469A35B928B960EB6BB99EB981BBBF
:1014800000C000C041BB469A35B928B95BB99EB9C6
:1014900081BB39813FBF4FB74983F89484EE9EE00A
:1014A0000E9436492090080F3090090F8091561005
:1014B00090915710880E991EA11CB11C81149104A3
:1014C00051E0A506B1042CF088248A94982CA12C14
:1014D000B12CD501C401B7FC42C30E94332B46ECAA
:1014E00041BB469A31E035B927E428B950EF5BB9E2
:1014F00090EA9EB987E881BB00C000C041BB469A14
:1015000035B928B960EE6BB99EB981BB00C000C087
:1015100041BB469A35B928B95BB99EB981BB6A818E
:101520007B819101AA27629FB12D7303A001369F91
:10153000B00D411D5A1F72035A0BB00D411D5A1FA9
:101540001124662757FD6095762F4C0D5D1D6E1D8D
:101550007F1D80914A1090914B10480F591F611DBB
:10156000711D4115510531E06307710524F04FEFFE
:101570005FEF60E070E0DB01CA0177FDECC20E9422
:10158000332B46EC41BB469A31E035B923E428B908
:1015900050EF5BB992EA9EB987E881BB00C000C0FA
:1015A00041BB469A35B928B960ED6BB99EB981BB8C
:1015B00000C000C041BB469A35B928B95BB99EB995
:1015C00081BBB101AA27069FB12D1703A001709F0F
:1015D000B00D411D5A1F16035A0BB00D411D5A1F65
:1015E0001124662757FD6095762F440D551D661D05
:1015F000771D8091621090916310480F591F611DF3
:10160000711D8091921090919310A0E0B0E084172A
:101610009507A607B70724F077FDA5C2DB01CA012D
:101620000E94332B46EC41BB469A31E035B923E4A6
:1016300028B950EF5BB990EA9EB987E881BB00C03A
:1016400000C041BB469A35B928B960EB6BB99EB969
:1016500081BB00C000C041BB469A35B928B95BB90F
:101660009EB981BB80EE9FE00E94364980910410B4
:1016700090910510009709F069C10E94332B46EC48
:1016800041BB469A31E035B927E428B950EF5BB940
:1016900092EA9EB987E881BB00C000C041BB469A70
:1016A00035B928B960EB6BB99EB981BB00C000C0E9
:1016B00041BB469A35B928B95BB99EB981BB29812E
:1016C0002FBF2091A809922F9C7111E009F010E022
:1016D000922F9370923009F48CC2933009F4B3C402
:1016E000913009F492C21111C4C480E00E94D55017
:1016F0008091A4099091A509A091A609B091A7098C
:101700000196A11DB11D8093A4099093A509A093F2
:10171000A609B093A7092091A8092F5F2093A809D3
:101720000F900F900F90DF91CF911F910F91FF902D
:10173000EF90DF90CF90BF90AF909F908F907F9071
:101740006F905F904F903F902F900895B7FD18C213
:10175000AC01BD0117C8B7FD09C2AC01BD01B9C9D3
:10176000B7FD08C2AC01BD0150CBB7FD0DC2AC0145
:10177000BD01A3CCB7FD01C2AC01BD013ACE83309F
:1017800009F473C1843009F04CCD6091BE0E7091A4
:10179000BF0E8091C00E9091C10E2091E00E40EAE4
:1017A00051E00E94CD20809590953DCD833009F485
:1017B0009BC1843009F0BFCC6091900F7091910F64
:1017C0008091920F9091930F2091B20F40EA51E0D7
:1017D0000E94CD2080959095B0CC833009F4E5C06F
:1017E000843009F082CB6091940E7091950E8091B7
:1017F000960E9091970E2091B60E40EA51E00E940D
:10180000CD208095909573CB833009F457C18430F7
:1018100009F073C86091400E7091410E8091420EA4
:101820009091430E2091620E40EA51E00E94CD203B
:101830008095909564C8833009F45BC1843011F0C1
:101840000C9404046091120F7091130F8091140F87
:101850009091150F2091340F40EA51E00E94CD2065
:10186000809590950C940604833009F4E9C0843087
:1018700011F00C94CE026091160E7091170E8091AB
:10188000180E9091190E2091380E40EA51E00E94F6
:10189000CD20809590950C94D002833009F4F9C046
:1018A000843009F054C960913C0F70913D0F8091D4
:1018B0003E0F90913F0F20915E0F211182C1BB27F7
:1018C000A92F982F872F8095909543C9833009F4CD
:1018D000B2C0843009F0B1C960916A0E70916B0E8C
:1018E00080916C0E90916D0E20918C0E21115FC134
:1018F000BB27A92F982F872F80959095A0C986E6A2
:101900009EE00E9410208FC921154DEF340708F486
:1019100040C18FEF9FEF4FC988E39FE00E941020E6
:101920000CC980E99EE00E941020D5CA81153DEFC8
:10193000930708F42CC18FEF9FEF95CA81153DEFF7
:10194000930708F430C18FEF9FEF81CD81157DEFB4
:10195000970708F42AC18FEF9FEF8FCE8CE89FE0A6
:101960000E941020DECB8EE09FE00E9410200C949D
:10197000F7038AEB9EE00E94102049CC21154DEF21
:10198000340708F409C18FEF9FEF09CC8CE39EE088
:101990000E9410200C94720421154DEF340708F4B6
:1019A000FEC08FEF9FEF0C9439048091A40E9091AC
:1019B000A50E9DCA6091BE0E7091BF0E8091C00EA3
:1019C0009091C10E2091E00E40EA53E00E94CD209C
:1019D0002ACC6091940E7091950E8091960E909104
:1019E000970E2091B60E2111F1C0BB27A92F982F79
:1019F000872F7DCA6091160E7091170E8091180E78
:101A00009091190E2091380E40EA53E00E94CD20AB
:101A10000C94D00260916A0E70916B0E80916C0EE6
:101A200090916D0E20918C0E2111C6C0BB27A92F5D
:101A3000982F872F04C980917A0E90917B0EFFC852
:101A40008091260E9091270E0C94D00260913C0F4D
:101A500070913D0F80913E0F90913F0F20915E0F4E
:101A600040EA53E00E94CD2074C88091CE0E909140
:101A7000CF0ED9CB6091900F7091910F8091920F02
:101A80009091930F2091B20F40EA53E00E94CD2035
:101A900054CB80914C0F90914D0F5BC86091400EDC
:101AA0007091410E8091420E9091430E2091620EF2
:101AB00040EA53E00E94CD200C947F048091500EA8
:101AC0009091510E0C947F046091120F7091130F3E
:101AD0008091140F9091150F2091340F40EA53E03C
:101AE0000E94CD200C9406048091A00F9091A10F2C
:101AF00024CB8091220F9091230F0C94060480E058
:101B000090E0DC010C94C50480E090E0DC01CFCBD8
:101B100080E090E0DC012FCA80E090E0DC017ECA2A
:101B200080E090E0DC010C94730380E090E0DC0145
:101B30000C941E0380E090E0DC01C5C880E090E0DA
:101B4000DC010C941A0580E090E0DC010FC980E014
:101B500090E0DC01FFCB80E090E0DC0110CD80E084
:101B600090E0DC01BACC80E090E05ACD80E090E0DB
:101B70000C946A0580E090E049C980E090E03ACC9E
:101B800080E090E00C94C30380E090E097CA9D5FF2
:101B90006AC9C9019D5F0FC8C9019D5F00CBC9011A
:101BA0009D5F0C9439049D5F52CC9D5F66CD40EAE9
:101BB00051E00E949519A0CE40EA53E00E94951989
:101BC0003EC840EA51E00E9495197DCE40EA53E0BC
:101BD0000E9495198CC91B821A820C94AA02C0908B
:101BE0002010D0902110D594C794C80CD91C0C9407
:101BF0006D0285E290E10E94FA208091D4108870F5
:101C00000E9409292091A80988CD0E94C056809180
:101C10005D12882309F427C28091C710882379F0C8
:101C200081508093C7108091030D811125C280914E
:101C3000040D811121C28091020D81113BC380915D
:101C4000C010882309F407C28091BE109091BF1084
:101C500040916410509165102091401030914110D6
:101C60002417350708F4F6C24217530770F4B90178
:101C7000641B750BAB018617970708F4AC01241B96
:101C8000350B3093411020934010409170105091CB
:101C9000711020914C1030914D102417350708F425
:101CA000CDC24217530770F4F901E41BF50BAF01E5
:101CB0008E179F0708F4AC01241B350B30934D1091
:101CC00020934C1040917C1050917D102091581021
:101CD000309159102417350708F4A4C2421753074E
:101CE00070F4B901641B750BAB018617970708F4F4
:101CF000AC01241B350B30935910209358104091A0
:101D000066105091671020914210309143102417B3
:101D1000350708F47BC24217530770F4F901E41B3E
:101D2000F50BAF018E179F0708F4AC01241B350B90
:101D300030934310209342104091721050917310D1
:101D400020914E1030914F102417350708F451C2DE
:101D50004217530770F4B901641B750BAB0186176A
:101D6000970708F4AC01241B350B30934F102093D8
:101D70004E1040917E1050917F1020915A1030915A
:101D80005B102417350708F427C24217530770F475
:101D9000F901E41BF50BAF018E179F0708F4AC01A6
:101DA000241B350B30935B1020935A104091681020
:101DB0005091691020914410309145102417350737
:101DC00008F4FDC14217530770F4B901641B750B89
:101DD000AB018617970708F4AC01241B350B309331
:101DE000451020934410409174105091751020912B
:101DF0005010309151102417350708F4D3C1421701
:101E0000530770F4F901E41BF50BAF018E179F0720
:101E100008F4AC01241B350B309351102093501063
:101E2000409180105091811020915C1030915D1094
:101E30002417350708F4A9C14217530770F4B901F4
:101E4000641B750BAB018617970708F4AC01241BC4
:101E5000350B30935D1020935C1040916A105091C7
:101E60006B1020914610309147102417350708F465
:101E70007FC14217530770F4F901E41BF50BAF0162
:101E80008E179F0708F4AC01241B350B30934710C5
:101E90002093461040917610509177102091521067
:101EA000309153102417350708F455C142175307D2
:101EB00070F4B901641B750BAB018617970708F422
:101EC000AC01241B350B30935310209352104091DA
:101ED00082105091831020915E1030915F10241772
:101EE000350708F42BC14217530770F4F901E41BBE
:101EF000F50BAF018E179F0708F4AC01241B350BBF
:101F000030935F1020935E1040916C1050916D10D3
:101F100020914810309149102417350708F401C169
:101F20004217530770F4B901641B750BAB01861798
:101F3000970708F4AC01241B350B3093491020930C
:101F400048104091781050917910209154103091A0
:101F500055102417350708F4D7C04217530770F4FB
:101F6000F901E41BF50BAF018E179F0708F4AC01D4
:101F7000241B350B3093551020935410409184103E
:101F80005091851020916010309161102417350711
:101F900008F4ADC04217530770F4B901641B750B08
:101FA000AB018617970708F4AC01241B350B30935F
:101FB00061102093601040916E1050916F1020912D
:101FC0004A1030914B102417350708F07DC0421B92
:101FD000530B8417950708F46BC1420F531F50939E
:101FE0004B1040934A1040917A1050917B102091F1
:101FF0005610309157102417350708F052C0421B75
:10200000530B8417950708F451C1420F531F509387
:102010005710409356104091861050918710209190
:102020006210309163102417350748F5421B530B9B
:102030008417950708F438C1420F531F509363105B
:102040004093621008C022FD68CB812F0E94403768
:10205000812F0E94B02D2091A8095FCB0196A11D70
:10206000B11D0C94A4028091C710882309F4DBCD24
:10207000D7CD0E94792639CB0E94CB57DCCD4217B1
:10208000530748F7F901E41BF50BAF018E179F07C3
:1020900008F4AC01241B350B3093631020936210BD
:1020A000DACF4217530708F0B6CFB901641B750B9E
:1020B000AB018617970708F4AC01241B350B30934E
:1020C000571020935610A7CF4217530708F08BCF15
:1020D000F901E41BF50BAF018E179F0708F4AC0163
:1020E000241B350B30934B1020934A107CCF421B9E
:1020F000530B8417950708F4D5C0420F531F509314
:1021000061104093601057CF421B530B8417950703
:1021100008F4C6C0420F531F5093551040935410FB
:102120002DCF421B530B8417950708F4B7C0420FFD
:10213000531F509349104093481003CF421B530B39
:102140008417950708F4A8C0420F531F50935F10DF
:1021500040935E10D9CE421B530B8417950708F4A9
:1021600099C0420F531F5093531040935210AFCE5B
:10217000421B530B8417950708F48AC0420F531F64
:10218000509347104093461085CE421B530B841743
:10219000950708F47BC0420F531F50935D10409386
:1021A0005C105BCE421B530B8417950708F46CC080
:1021B000420F531F509351104093501031CE421B89
:1021C000530B8417950708F45DC0420F531F5093BB
:1021D00045104093441007CE421B530B84179507BC
:1021E00008F44EC0420F531F50935B1040935A1097
:1021F000DDCD421B530B8417950708F43FC0420FF7
:10220000531F50934F1040934E10B3CD421B530BAE
:102210008417950788F1420F531F50934310409342
:1022200042108ACD421B530B8417950718F1420FB9
:10223000531F509359104093581061CD421B530BBC
:1022400084179507A8F0420F531F50934D104093E9
:102250004C1038CD421B530B8417950738F0420FB2
:10226000531F50934110409340100FCDAC01F7CF56
:10227000AC01E9CFAC01DBCFAC01CDCFAC01BFCF1E
:10228000AC01B0CFAC01A1CFAC0192CFAC0183CFF8
:10229000AC0174CFAC0165CFAC0156CFAC0147CFD8
:1022A000AC0138CFAC0129CFAC01C6CEAC01ADCE6C
:1022B000AC0193CE0E94E255C2CCE82FF0E0EE0FC5
:1022C000FF1FEB5CFE4E808191810895803891055F
:1022D00038F4FC01E45EFE4F208130E0C90108952E
:1022E0002FEF3FEFFBCFCF93DF93CCE9D7E1E8812E
:1022F000F98185EA96E1A1E6B0E081939193A193FB
:10230000B193F983E883DF91CF910895ACE9B7E108
:10231000ED91FC9111978191ED93FC930895ACE9B7
:10232000B7E1ED91FC9111978191ED93FC930895A4
:10233000ACE9B7E1ED91FC911197808191813296E2
:10234000ED93FC930895ACE9B7E1ED91FC91119701
:1023500060817181828193813496ED93FC9308951D
:10236000E82FE695E695E695F0E0E659F54F908181
:10237000992351F08770E82FF0E0E75CF84F208157
:10238000292381E009F0089580E00895FC01A18DE2
:10239000BB27A1950CF4B095AA0FBB1F1196208501
:1023A0003185428553850E94897564877587868744
:1023B00097870895CF92DF92EF92FF92CF93603E7E
:1023C000710581059105F8F4DC01CB019F5FAF4FEA
:1023D000BF4FCC24D82EE92EFA2EA0E0B0E020E0AA
:1023E00030E0EBBEF601C791A40FB51FCC932F5F71
:1023F0003F4FD9018FEFC81AD80AE80AF80A211509
:1024000081E0380771F7CF91FF90EF90DF90CF9088
:102410000895CF93DF93BC0180E090E04CE955E153
:10242000C9DFCCE9D5E1D0939D17C0939C171092DA
:102430009E1789DF653A76418146910551F080E02B
:1024400092E0FE019C01119221503040E1F780E0C2
:1024500004C065DF80939E1781E0DF91CF910895DE
:10246000AF92BF92CF92DF92EF92FF920F931F93A2
:10247000CF93DF935C01C12CD12C7601C0E0D0E07A
:10248000062F10E00EC0A60144565A4EBE016A0D3A
:102490007B1D80E090E08EDF21962FEFD21AE20ABA
:1024A000F20AC017D10778F3CCE9D5E1D0939D1794
:1024B000C0939C1710929E1746DF653A764181467D
:1024C000910551F080E092E0FE019C0111922150B3
:1024D0003040E1F780E004C022DF80939E1781E066
:1024E000DF91CF911F910F91FF90EF90DF90CF90F0
:1024F000BF90AF900895EF92FF920F931F93CF93E9
:10250000DF93EC01162FF42EE22E8091C419843053
:1025100071F1C230D10509F453C0C330D10571F156
:10252000C130D105F9F1C430D105C8F5E091BB192E
:10253000F091BC19309739F00E2D2F2D412FBE018F
:102540008FE999E10995E091BD19F091BE19309795
:1025500039F00E2D2F2D412FBE018FE999E10995FC
:10256000DF91CF911F910F91FF90EF900895E0912F
:10257000B919F091BA193097F9F6D8CF862F807F24
:10258000803A09F48DC008F041C0803809F456C083
:10259000803961F6E091A319F091A41942C0C0E01E
:1025A000D0E0C4CF683F50F1E091B519F091B61971
:1025B000309709F4BBCF612F8FE999E10995C3CF1B
:1025C000862F807F803D09F455C0803F09F440C0CC
:1025D000803C09F0ABCFE091AD19F091AE19309786
:1025E00009F4A4CF133F09F43FC0113FE9F1612F73
:1025F0006F704F2D8FE999E10995A5CF663F09F0DE
:1026000095CFE091B719F091B819D2CF803ED9F0AB
:10261000803FA9F1803B09F089CFE091A119F091A9
:10262000A219309709F482CF123F99F1612F6F7090
:102630002E2D4F2D8FE999E1099585CFE091A519B0
:10264000F091A619EECFE091A919F091AA19E9CF5E
:10265000633F59F1613F09F069CFE091B319F091FF
:10266000B419309709F462CF4F2D612F8FE999E1AA
:10267000099569CFE091AF19F091B019B0CF623FE1
:1026800009F054CFE091AB19F091AC19309709F4EF
:102690004DCF2E2D4F2D62EF8FE999E1099553CF44
:1026A000E091A719F091A819BCCFE091B119F09170
:1026B000B2193097C9F63ACF86EC81BB469A15B865
:1026C00080E488B980E58BB980E68EB987E881BB64
:1026D00085E08A95F1F70000089586EC81BB469A63
:1026E00015B880E488B980ED8BB980E68EB987E8AB
:1026F00081BB85E08A95F1F70000089586EC81BBE7
:10270000469A15B885E488B980E58BB980E68EB91C
:1027100087E881BB85E08A95F1F700000895EF9284
:10272000FF920F931F93CF93DF93F82EE62EABEA21
:102730008A9FA12D1124A695A695A6951A2F1F5FF5
:1027400050E0A83008F06AC08A2F90E0880F991FE7
:10275000FC01EE0FFF1FEE0FFF1FEE0FFF1FE80F34
:10276000F91FE40FF51FEE0FFF1FEB5CFE4EC0815B
:10277000D181183008F476C0FA01EE0FFF1FEF5C2C
:10278000FD4E0190F081E02DDA01AA0FBB1FA35F7F
:10279000BD4E8D919C919F01281B390BA12FB0E05C
:1027A00017970E94C1706E0F7F1F811D911D6115CB
:1027B000710521E08207910508F06AC08B010C1BAE
:1027C0001D0B3E2D20E09BEAF99E912D112496953C
:1027D00096959695892F880F890F880F880F6F2DF2
:1027E000681B862F90E0A0E0B0E077276627620F95
:1027F000731F811D911D2CE030E040E050E00E94ED
:10280000CA75D8010E947F75C80FD91FCE01DF910C
:10281000CF911F910F91FF90EF900895FA01EE0F65
:10282000FF1FEF5CFD4E0190F081E02DEA01CC0F1F
:10283000DD1FC35FDD4E888199819F01281B390B05
:10284000B0E017970E94C1706E0F7F1F811D911D10
:102850006115710521E082079105F8F4EB0118304C
:1028600008F08ACF812F90E0880F991FFC01EE0FAE
:10287000FF1FEE0FFF1FEE0FFF1FE80FF91FE40F02
:10288000F51FEE0FFF1FEB5CFE4E6081718196CF4E
:102890006FEF7FEF80E090E091CF6FEF7FEF80E010
:1028A00090E0EB01DCCFFF920F931F93CF93DF9368
:1028B000F82EABEA8A9FA12D1124A695A695A69580
:1028C0001A2F1F5F462F50E0A83008F063C08A2FF0
:1028D00090E0880F991FFC01EE0FFF1FEE0FFF1F06
:1028E000EE0FFF1FE80FF91FE40FF51FEE0FFF1F9C
:1028F000EB5CFE4EC081D181183008F46FC0FA0144
:10290000EE0FFF1FEF5CFD4E0190F081E02DDA012C
:10291000AA0FBB1FA35FBD4E8D919C919F01281BE9
:10292000390BA12FB0E017970E94C1706E0F7F1F67
:10293000811D911D6115710521E08207910508F047
:1029400063C08B010C1B1D0B9BEAF99E912D11247A
:10295000969596959695892F880F890F880F880FE1
:102960006F2D681B862F90E0A0E0B0E077276627E8
:102970002CE030E040E050E00E94CA75D8010E948F
:102980007F75C80FD91FCE01DF91CF911F910F9195
:10299000FF900895FA01EE0FFF1FEF5CFD4E0190CE
:1029A000F081E02DEA01CC0FDD1FC35FDD4E888191
:1029B00099819F01281B390BB0E017970E94C170C5
:1029C0006E0F7F1F811D911D6115710521E082072A
:1029D0009105F8F4EB01183008F091CF812F90E0C9
:1029E000880F991FFC01EE0FFF1FEE0FFF1FEE0F68
:1029F000FF1FE80FF91FE40FF51FEE0FFF1FEB5C41
:102A0000FE4E608171819DCF6FEF7FEF80E090E09F
:102A100098CF6FEF7FEF80E090E0EB01DCCFEF929B
:102A2000FF920F931F93CF93DF93E8E9F0E11192A8
:102A3000119280E1EC3BF807D1F71092BD10109293
:102A4000BC108091DD10823009F4F4C0833009F4A9
:102A5000D7C0813039F0DF91CF911F910F91FF9056
:102A6000EF900895C0919610D09197101091DC10BE
:102A7000110F60E0812F17DF7C0180E01EDC9701E1
:102A8000281B390BDE010E94C1709093991080932E
:102A9000981061E0812F07DF7C0181E00EDC970157
:102AA000281B390BDE010E94C17090939B1080930C
:102AB0009A1062E0812FF7DE7C0182E0FEDB970155
:102AC000281B390BDE010E94C17090939D108093EA
:102AD0009C1063E0812FE7DE7C0183E0EEDB970151
:102AE000281B390BDE010E94C17090939F108093C8
:102AF0009E1064E0812FD7DE7C0184E0DEDB97014D
:102B0000281B390BDE010E94C1709093A1108093A5
:102B1000A01065E0812FC7DE7C0185E0CEDB970148
:102B2000281B390BDE010E94C1709093A310809383
:102B3000A21066E0812FB7DE7C0186E0BEDB970144
:102B4000281B390BDE010E94C1709093A510809361
:102B5000A41067E0812FA7DE7C0187E0AEDB970140
:102B6000281B390BDE010E94C1709093A71080933F
:102B7000A61068E0812F97DE7C0188E09EDB97013C
:102B8000281B390BDE010E94C1709093A91080931D
:102B9000A81069E0812F87DE7C0189E08EDB970138
:102BA000281B390BDE010E94C1709093AB108093FB
:102BB000AA106AE0812F77DE7C018AE07EDB970134
:102BC000281B390BDE010E94C1709093AD108093D9
:102BD000AC106BE0812F67DE8C018BE06EDB98011F
:102BE000281B390BDE010E94C1709093AF108093B7
:102BF000AE10DF91CF911F910F91FF90EF9008954C
:102C00002091DC10A0919610B091971030E00E94B6
:102C1000C1709B01AC01A5E5B5E10E947F75909361
:102C2000BD108093BC10DF91CF911F910F91FF9049
:102C3000EF9008952091DC10A0919610B09197101C
:102C400030E00E94C1709B01AC01A5E5B5E10E9496
:102C50007F75BB2797FDB095AB2F9093B1108093F4
:102C6000B0109093B3108093B2109093B5108093EE
:102C7000B4109093B7108093B6109093B9108093CE
:102C8000B8109093BB108093BA10DF91CF911F9131
:102C90000F91FF90EF9008950F931F93E82FF0E0AE
:102CA000DF01AA0FBB1FAF5CBD4E0D911C91EE0F53
:102CB000FF1FE35FFD4E80819181A801481B590BE6
:102CC00020E030E060E070E0DB01CA01880F991F6E
:102CD000AA1FBB1F840F951FA61FB71F800F911F30
:102CE000A21FB31F0097E1E0AE07B10520F08FEF00
:102CF0009FEFA0E0B0E0440F551F661F771F440F01
:102D0000551F661F771F400F511F621F731F41150C
:102D1000510521E06207710520F04FEF5FEF60E0A1
:102D200070E0481B590B8A0120E030E0369527956A
:102D300017950795080F191FC8011F910F91089546
:102D400021E030E002C0220F331F8A95E2F7D9015B
:102D5000A095B0958091290A90912A0A8A239B23F5
:102D600090932A0A8093290AE0912B0AF0912C0A69
:102D7000EA23FB23F0932C0AE0932B0A662371F0DD
:102D8000822B932B90932A0A8093290A442331F0B3
:102D90002E2B3F2B30932C0A20932B0A089521E0F1
:102DA00030E002C0220F331F8A95E2F7F901E09567
:102DB000F0958091290A90912A0A8E239F2390935F
:102DC0002A0A8093290A40912B0A50912C0A4E23FB
:102DD0005F2350932C0A40932B0A662331F0282B53
:102DE000392B30932A0A2093290A0895CF93DF9331
:102DF0001F92CDB7DEB790E0698368DA80932D0A21
:102E00006981862F90E062DA80932E0A0F90DF911D
:102E1000CF91089524E630E040E050E00E94A37591
:102E20002AE030E040E050E00E94A375605D822F10
:102E3000805DDCCF21E02093330A009721F48FEFEF
:102E40008093320A08951092320ABC0189E39AE015
:102E50000E94F27469EC78E088E39AE00C94E774DD
:102E60001092820B1092840B8FEF8093810B8093D2
:102E7000800B10927A0B10927B0B10927C0B1092AD
:102E80007D0B10928D0B10928F0B80938C0B809387
:102E90008B0B1092850B1092860B1092870B109261
:102EA000880B1092980B10929A0B8093970B80933B
:102EB000960B1092900B1092910B1092920B109215
:102EC000930B1092A30B1092A50B8093A20B8093EF
:102ED000A10B10929B0B10929C0B10929D0B1092C9
:102EE0009E0B1092AE0B1092B00B8093AD0B8093A3
:102EF000AC0B1092A60B1092A70B1092A80B10927D
:102F0000A90B1092B90B1092BB0B8093B80B809356
:102F1000B70B1092B10B1092B20B1092B30B109230
:102F2000B40B08951F93CF93DF93D82FC92F162F7B
:102F30008091C40B68130AC046E050E06CEB7BE064
:102F40008D2F0E94B974009711F424C089DF10936B
:102F5000C40B46E050E06FEF70E08CEB9BE00E940A
:102F6000E074ED2FFC2FACEBBBE080E091919F3F34
:102F700019F4882341F004C09D938F5F8630B1F728
:102F80001092BC0B07C086E0ECEBFBE0DF011D926A
:102F90008A95E9F7DF91CF911F910895CF93DF9341
:102FA00000D000D000D0CDB7DEB786E0E2EDF6E08D
:102FB000DE01119601900D928A95E1F760E0CE0155
:102FC0000196B0DF26960FB6F894DEBF0FBECDBFD8
:102FD000DF91CF910895EF92FF920F931F93CF93BC
:102FE000DF9300D000D000D0CDB7DEB746E050E090
:102FF0006FEF70E08E010F5F1F4FC8010E94E074F9
:10300000F12CE12C8F2DACD98823A9F0F801EE0D1D
:10301000F11DE7FCFA95F082EE2021F089819F2DC9
:10302000981B9083E39485E08E152CF461E0CE012B
:10303000019678DF05C0F39490E8F912E3CFF6CF5C
:1030400026960FB6F894DEBF0FBECDBFDF91CF91AD
:103050001F910F91FF90EF90089586E0ECEBFBE05D
:10306000AFE1B1E101900D928A95E1F7089555E045
:103070005A95F1F7000036EC31BB469A80EE87B9DD
:1030800097E09AB98DB915B880E488B91BB880E289
:103090008EB987E481BB82E08A95F1F700C026B142
:1030A00099B18CB131BB479A37EE37B937EF3AB99E
:1030B00032EE3DB9422F4695437050E8259F90016E
:1030C0001124422B292F2071422B292F269526953A
:1030D0002870422B96959076492B90E0880F991F87
:1030E00084709927842B08951092CD0B1092CE0BEB
:1030F0001092CF0B1092D00B8FEF8093320C8093F5
:1031000028118FEF9FEFDC018093291190932A11F2
:10311000A0932B11B0932C1108958F929F92AF9290
:10312000BF92CF92DF92EF92FF920F931F934A01CB
:103130005B0168017901BC0180E090E00E9422728D
:103140009058A50194010E945D710E94CA71A70167
:1031500096010E9482730E94F671CB011F910F911C
:10316000FF90EF90DF90CF90BF90AF909F908F90A7
:1031700008950F931F93809115119091161100E0FF
:1031800010E42CE135E440E050E86BE376E4809510
:103190009095C3DF9093C6108093C5101F910F9137
:1031A000089580916A0A90916B0A892B90916C0A1C
:1031B000892B90916D0A892B90916E0A892B9091A1
:1031C0006F0A892B9091700A892B9091710A892B33
:1031D0009091720A892B9091730A892B9091740AAD
:1031E000892B9091750A892B9091760A892B909161
:1031F000770A892B9091780A892B9091790A982BDC
:1032000021E009F420E08091980B90918D0B892B9F
:103210009091A30B892B9091AE0B892B9091820BEF
:10322000892B9091B90B892B59F48FEF9FEFDC011B
:103230008093C1109093C210A093C310B093C41098
:103240002223A1F080918814811110C08091A409DB
:103250009091A509A091A609B091A7098093C110EA
:103260009093C210A093C310B093C41020938814FD
:1032700008950F931F93CF93DF93EC018A899B8965
:1032800000E01FEF2FE737E440E050E26BE476E424
:103290008095909542DFAC0160E070E0088C04C03E
:1032A000440F551F661F771F0A94D2F74887598726
:1032B0006A877B87DF91CF911F910F910895CF93FC
:1032C000DF93EC01888D681739F0688FCE01D1DF6C
:1032D000CE01DF91CF915AC8DF91CF910895CF935E
:1032E000DF93EC01598B488B8A899B896817790792
:1032F00041F07B8B6A8BCE01BCDFCE01DF91CF9199
:1033000045C8DF91CF910895AC01AA27469FB12D02
:10331000579F9001749FB00D211D3A1F569FB00D0D
:10332000211D3A1F1124C9010895A72F8F3FF9F0DD
:10333000282F2F5F30E0220F331FE82FF0E0EE0F31
:10334000FF1FE40FF51F60817181FA01E20FF31F87
:1033500080819181861B970B892F9927A89F9001C7
:10336000A99F300D1124260F371FC90108952EEF94
:1033700031E0E3CF8FBF0895F89481E008958FBFC7
:103380000895ECE9F7E1A081B1818C93808191816E
:103390000196918380830895ECE9F7E1A081B181E2
:1033A0008C93808191810196918380830895CF933E
:1033B000DF93ECE9F5E180E092E0DF019C011D92F2
:1033C00021503040E1F7F0939D17E0939C17CEE930
:1033D000D7E184E088830E9473118881DF91CF91C7
:1033E000DBCFACE9B7E1ED91FC911197819391931B
:1033F000ED93FC930895F89481E00895CF93DF93C3
:10340000DFB7F9DF882309F448C08CE5E9ECF0E187
:10341000DF011D928A95E9F720E030E83093E8104B
:103420002093E7103093EE102093ED104FEF5FEFF5
:103430005093F2104093F1103093F6102093F51052
:1034400050930211409301115093E6104093E51000
:10345000309312112093111130931E1120931D11DE
:10346000309318112093171185E08093DC10C1E090
:10347000C093DD10C093D610C093D810C093DE1057
:1034800082E08093DF1046E050E06FEF70E08FE164
:1034900091E10E94E074C093C9108D2FDF91CF910C
:1034A0006ECFCF92DF92EF92FF920F931F93CF9345
:1034B000DF931F92CDB7DEB7F82E8B01EFB699835D
:1034C0009ADF99818823F1F08F2D0E940912ECE98F
:1034D000F6E16F018CE995E1C81AD90A8291882337
:1034E000C1F3F0929F1720EA37E1ECE9F5E1A6017C
:1034F000BF01C9010E94C6749FEFC91AD90AF80119
:10350000D182C0828E2D0F90DF91CF911F910F91AC
:10351000FF90EF90DF90CF9032CF0F931F93CF9318
:10352000DF93182FEB010FB766DF811104C0802FE6
:1035300026DF81E016C0812F992787FD909588535B
:103540009F4F0E940912811108C0802F18DF80E070
:1035500008C00E948F11899301C011E8115039F3FE
:10356000F8CFDF91CF911F910F9108951F93CF93C3
:10357000DF93EC011FB73FDF811104C0812FFFDE15
:10358000C1E05EC0CE010E940912882309F455C033
:103590001092DB1010921F119FEF909320119093C7
:1035A00021119093221190932311909324118091D3
:1035B0009E17811102C0C1E041C0C0E00E94981175
:1035C000EC2FF0E0EE0FFF1FED51FF4E9183808353
:1035D000CF5FC93199F7D0E00E948F11ED2FF0E055
:1035E000E753FF4E8083DF5FD731B1F78091D91069
:1035F0008093E21080919E178230E8F20E94981129
:10360000EC2FF0E0EE0FFF1FED51FF4E9183808312
:10361000CF5FCE3199F70E948F118093E0100E9406
:103620008F118093E110CFE1D1E10E948F11899336
:1036300081E1C532D807C9F7A1CFC0E0812F9FDE55
:103640008C2FDF91CF911F9108951F93CF93DF931C
:10365000182FDFB7D0DE882309F448C08CE5E9ECE9
:10366000F0E1DF011D928A95E9F720E030E8309320
:10367000E8102093E7103093EE102093ED104FEFF9
:103680005FEF5093F2104093F1103093F6102093B7
:10369000F51050930211409301115093E61040939E
:1036A000E510309312112093111130931E112093C5
:1036B0001D11309318112093171185E08093DC10B1
:1036C000C1E0C093DD10C093D610C093D810C09352
:1036D000DE1082E08093DF1046E050E06FEF70E094
:1036E0008FE191E10E94E074111105C08D2FDF91EF
:1036F000CF911F9144CEC093C910F8CFFF920F9382
:103700001F93CF93DF93FFB676DE811104C08F2D18
:1037100036DEC1E06FC062E08CED90E00E943012B6
:10372000882309F464C08FE380935C1210925E12C8
:1037300010925F1280919E17882319F0C5E3D1E1A2
:1037400013C0C1E055C00E949811FE01E00FF11FA7
:10375000918380830E5F1F4F04321105A1F7A49659
:1037600082E1C535D80719F000E010E0ECCF0E94E7
:10377000981190935812809357120E949811909329
:103780005612809355120E948F11809359120E94F5
:10379000861180935A1280919E17823090F20E9477
:1037A0008F1180935C120E94861180935B1280912E
:1037B0009E17833030F20E948F1180935D128091AA
:1037C0009E17843008F4BDCF0E94861180935E124C
:1037D00080919E17853008F4B4CF0E9486118093A3
:1037E0005F1280919E17863008F091CFAACFC0E07B
:1037F0008F2DC5DD8C2FDF91CF911F910F91FF9001
:103800000895DF92EF92FF920F931F93CF93DF9370
:10381000982FB091C30BFF24F394FB22B0FFCAC0D2
:103820002091800BE22FE695E695E695F0E0E659CB
:10383000F54F80818111B5C040917A0B50917B0B7F
:1038400060917C0B70917D0B4F3F2FEF5207620709
:10385000720709F0A1C18FEF12E0E12EEB22B1FF58
:103860001AC030918B0BC32FC695C695C695D0E074
:10387000C659D54F2881211137C10091850B109170
:10388000860B2091870B3091880B041715072607AC
:10389000370708F483C1AB2FA470B2FF1AC0309170
:1038A000960BC32FC695C695C695D0E0C659D54F81
:1038B000288121110FC10091900B1091910B209143
:1038C000920B3091930B041715072607370708F45E
:1038D00069C1CB2FC870B3FF1BC0D091A10B2D2F96
:1038E00026952695269530E02659354FF901108109
:1038F0001111E5C000919B0B10919C0B20919D0B29
:1039000030919E0B041715072607370708F44EC1A0
:10391000D0E1DD2EDB22B4FF1BC01091AC0B212FB8
:1039200026952695269530E02659354FF901D08108
:10393000D111BAC00091A60B1091A70B2091A80B32
:103940003091A90B041715072607370708F420C183
:10395000DB2FD072B5FF1BC00091B70B202F26952F
:103960002695269530E02659354FF9011081111121
:1039700025C00091B10B1091B20B2091B30B309187
:10398000B40B041715072607370708F484C08F3FC8
:1039900001F1DF91CF911F910F91FF90EF90DF9098
:1039A00008952770E22FF0E0E75CF84F208128238C
:1039B00009F442CF4FEF5FEFBA014DCF0770202FD0
:1039C00030E0275C384FF9012081212391F28F3FAD
:1039D00001F7B091C20BFF2009F493C0B13009F494
:1039E0003EC108F08BC040917A0B50917B0B6091E7
:1039F0007C0B70917D0B4F3FFFEF5F076F077F07D9
:103A000009F080E0EE2009F48BC08A019B0140910F
:103A1000850B5091860B6091870B7091880B401736
:103A200051076207730708F45CC1B901A801A1112D
:103A30007FC0CC2309F490C0B13009F42CC108F048
:103A4000C1C000919B0B10919C0B20919D0B30915C
:103A50009E0B041715072607370708F4BEC08A0116
:103A60009B01B901A801D1107EC0DD2309F491CFDB
:103A7000B13009F421C108F0A8C00091B10B109138
:103A8000B20B2091B30B3091B40B04171507260726
:103A9000370708F07ECF85E0DF91CF911F910F911E
:103AA000FF90EF90DF9008951770212F30E0275C92
:103AB000384FF90120812D2309F04ACF3BCFD77031
:103AC0002D2F30E0275C384FF9012081212309F0A8
:103AD0001FCF10CF3770C32FD0E0C75CD84F3881CD
:103AE000322309F0F6CEE7CE3770C32FD0E0C75CA3
:103AF000D84F3881322309F0CECEBFCEB23009F490
:103B000072C0EE2051F0B13009F4B2C008F056C0D6
:103B10000FEF1FEF98017BCF922F4FEF5FEFBA01AE
:103B2000AA2309F486CFB13009F4ADC008F042C031
:103B30000091900B1091910B2091920B3091930B6F
:103B4000041715072607370708F449C08A019B01A7
:103B5000B901A801C11175CFDD2009F486CFB130BC
:103B600009F4A1C0B0F50091A60B1091A70B20910C
:103B7000A80B3091A90B041715072607370788F102
:103B80008A019B01DD2309F404CFB901A80175CF97
:103B9000B901A80184E0DCCE80E05ECEB901A801C5
:103BA00081E079CEB901A80182E093CEB901A801E4
:103BB00083E0AECEB23009F03CCF2CC0B23009F079
:103BC000ACCF1BC0B23041F62FC0B23009F0E1CE0D
:103BD0003FC0B23009F049CF31C083E042CF82E02C
:103BE000B7CF84E0CFCF2091810B291708F47BC099
:103BF000292FEE2009F490CF922F20918C0B2917BA
:103C000008F46BC0292FAA2309F477C0922F4FEF35
:103C10005FEFBA012091970B291708F460C0292F94
:103C2000CC2309F468C0922F2091A20B291708F425
:103C30005CC0292FDD2009F45CC0922F2091AD0BD0
:103C4000291708F454C0292FDD2309F4A2CE922F9E
:103C50002091B80B291708F09CCE85E01DCF20914C
:103C6000810B9217A0F1292FEE2009F455CF922F46
:103C700020918C0B921738F1292FAA23F1F1922F62
:103C80004FEF5FEFBA012091970B9217F0F0292FB9
:103C9000CC2389F1922F2091A20B9217D0F0292FDB
:103CA000DD2039F1922F2091AD0B9217A0F0292F32
:103CB000DD2309F46ECE922F2091B80B921708F0F5
:103CC00068CE85E0E9CE81E0D8CF82E0E1CF80E028
:103CD000CBCF83E0E5CF84E0EBCF81E094CF82E0EF
:103CE0009FCF81E0A4CE80E084CF83E0A3CF84E0A7
:103CF000ABCF922FBACE922F2FCF922F4FEF5FEFF5
:103D0000BA0197CE833061F0893151F08F3141F0A3
:103D100091E08F3019F0803109F090E0892F0895FB
:103D200091E0892F0895BF92CF92DF92EF92FF9298
:103D30000F931F93CF93DF9310928C14C0E0D0E0C9
:103D400004E2B02E0CC00193119313870287778B86
:103D5000668B8150C1F72196C830D10591F16C2F47
:103D6000772767FD7095872F972F0E9424726B012C
:103D70007C012DEB3EE140EC55E40E94827320E093
:103D800030E44CE955E40E94F6700E94F6718B0114
:103D900021E33CE043E455E4C701B6010E9482738D
:103DA00020E030E44CE156E40E94F6700E94F67187
:103DB000BC9EF001BD9EF00D1124EB5CFE4E86E032
:103DC000C2CFDF91CF911F910F91FF90EF90DF90C5
:103DD000CF90BF900895CF93CFB70DDB8823B1F07C
:103DE0002BE231E0E5E3F1E1DF01C9011D9201972A
:103DF000E9F720E030E830935612209355128FEF08
:103E000080935A128FE380935C128DDF8C2FCF91B9
:103E1000B6CA8FBF0895E9E8F4E180818F5F80839F
:103E20000895F89481E008958C3F59F08138C1F1EC
:103E30009091030D933039F19091040D9330B1F0CE
:103E400008958091030D8330E9F18091040D833052
:103E5000B9F7E091060EEE2399F3E150E093060ED8
:103E6000F0E0EB57F24F8FEF808308959091060EAC
:103E700097FDE6CFE92FF0E0EB57F24F80839F5F8D
:103E80009093060E08959091050E97FDD5CFE92FDA
:103E9000F0E0ED5FF24F82839F5F9093050ECCCFF1
:103EA0008091030D8330E1F08091040D833041F661
:103EB0001092060E40E850E06FEF70E085E89DE05C
:103EC0000C94E074E091050EEE2309F4BECFE150AE
:103ED000E093050EF0E0ED5FF24F8FEF8283B5CFF8
:103EE0001092050E40E850E06FEF70E085E09DE035
:103EF0000E94E074D9CFCF93DF93EC016A8F888161
:103F00009981AA81BB81892B8A2B8B2B51F46091DB
:103F1000A4097091A5098091A6099091A7090E9412
:103F200047750E944475688379838A839B83DF91F8
:103F3000CF9108950F931F93CF93DF93FC018BE1F3
:103F4000DF011D928A95E9F703E812E160E070E075
:103F500080E89FEBC0E0D0E01BC0BE01882777FD62
:103F60008095982F0E94247221E830E840E85BE3B6
:103F70000E94827320E030E040E85FE30E94F67028
:103F80002BED3FE049E450E40E9482730E945A7195
:103F900020E030E040E85FE30E94F67020E03FEF71
:103FA0004FEF56E40E9482730E94F671F80161930C
:103FB00071938F012196C115F1E0DF0771F6DF9152
:103FC000CF911F910F9108950F931F93082F10E029
:103FD000F801E45BFE4F8491F801E45BFD4F94919E
:103FE000F801E45BFC4F049110E020E030E0980120
:103FF00011270027192B082BB801C9011F910F9118
:10400000089510922D0A10922E0A10922A0A1092E8
:10401000290A10922C0A10922B0A1092330A089542
:10402000FC0114821582168217821082118212827C
:10403000138281A58F5F81A7833009F43BC085304F
:1040400009F434C0823009F008952689378935A3F0
:1040500024A344895589AA27429FB12D539FC001AB
:10406000349FB00D811D9A1F529FB00D811D9A1F64
:10407000112480A391A340955095AA27429FB12D6A
:10408000539FC001349FB00D811D9A1F529FB00DE8
:10409000811D9A1F112482A393A3448555856685AB
:1040A00077854083518362837383089511A615A297
:1040B00014A2089511A210A28689978993A382A3BE
:1040C0000895FF920F931F93CF93DF93EC01F62E89
:1040D0001C821D821E821F820E891F896CA17DA1F8
:1040E000CB01A0E0B0E077276627980140E050E0E0
:1040F0000E94CA753F8F2E8FF11023C084E089A7DC
:1041000019A218A2AA27209FB12D319FC001129F8A
:10411000B00D811D9A1F309FB00D811D9A1F112473
:104120008AA39BA388899989AA89BB898883998353
:10413000AA83BB83FFA2DF91CF911F910F91FF90C4
:10414000089581E089A7CE010E94294BFFA2DF914B
:10415000CF911F910F91FF900895FC0111A210A221
:10416000268D378D46895789AA27249FB12D359FE3
:10417000C001529FB00D811D9A1F349FB00D811D4B
:104180009A1F112482A393A340895189628973895C
:1041900040835183628373830895211107C0BB2735
:1041A000A92F982F872FBC01CB010895A72FE82FA7
:1041B0008F3FE9F08F5F90E0880F991FF0E0EE0FDE
:1041C000FF1FE40FF51F20813181FA01E80FF91F6D
:1041D00080819181821B930B892F9927A89FB00121
:1041E000A99F700D1124620F731FCB0108958EEFEC
:1041F00091E0E4CF8F929F92AF92BF92CF92DF92E5
:10420000EF92FF920F931F93CF93DF93EC010C81FA
:104210001D812E813F81832F9927AA27BB27892BB8
:104220008A2B8B2B09F054C04A8D6C857D858E8539
:104230009F85433009F473C008F02FC0413009F462
:10424000B7C0EC89FD89060F171F281F391F0C8383
:104250001D832E833F839F01305848895989AA279F
:10426000249FB12D3503C001529FB00D811D9A1FAF
:1042700034039A0BB00D811D9A1F11248E8B9F8BD6
:10428000DF91CF911F910F91FF90EF90DF90CF9032
:10429000BF90AF909F908F900895443009F463C011
:1042A000453009F0CECF68017901A9E0F694E79492
:1042B000D794C794AA95D1F7F601DD8ACC8A498DA7
:1042C000442309F4C0CFE095F095FD8BEC8BBBCF78
:1042D000E1E0898DE81BE98FE11172C0C12CD12C7E
:1042E0007601CC82DD82EE82FF82FF27E1950CF41D
:1042F000F095DF01AA0FBB1F1196288539854A85E5
:104300005B850E9489756C877D878E879F874A8D24
:1043100041115CC0FD8BEC8B9701860192CFF12E91
:10432000E22F2F3F09F465C0422F4F5F50E0440F4A
:10433000551FF0E0EE0FFF1FED57FD4EA081B1813C
:10434000FA01ED57FD4E408151814A1B5B0B452F11
:104350005527F49EF001F59EF00D1124EA0FFB1F86
:10436000FD8BEC8B70CF4B8942954F708880998084
:10437000AA80BB80FB2D880C991CAA1CBB1CEF2FAC
:10438000EE1FEE27EE1FEF2EE294E69457E0E522B3
:10439000EE25EF27F695EF27E1708E2A415050F772
:1043A00088829982AA82BB82F4019D8A8C8A4BCF33
:1043B000C12ED22EE32EFF24F601DD8ACC8A43CF14
:1043C000CC24CA94DC2CEC2CF12C8BCF423019F08D
:1043D000970186012ECF0E9444757D8B6C8B4A8D90
:1043E0006C857D858E859F850C811D812E813F8109
:1043F00020CF4EEF51E09DCFCF92DF92EF92FF9210
:104400000F931F93CF93DF938091D310C82FCC0FBE
:10441000C80FCF5F6091D2108AE090E16CDD6C2F05
:104420008AE090E10E945F198091C1109091C210C2
:10443000A091C310B091C4108F3F2FEF9207A20735
:10444000B20709F49CC02091151130911611211565
:10445000324008F05DC0CFEFDFEFE0909410F090B5
:1044600095100090DE1002C0F694E7940A94E2F7EB
:1044700040910D1150910E11411582E0580708F43A
:10448000ACC09A0132508091191190911A119695F1
:10449000879596958795811542E0940708F472C038
:1044A0008C0112508091E010882309F471C0AE0194
:1044B000AA27249FB12D359FC001529FB00D811DA9
:1044C0009A1F349FB00D811D9A1F112460910B110A
:1044D00070910C11AC018AE090E10E946F19C80143
:1044E000809590958E159F0508F07AC04FEF5FEF8D
:1044F000609117117091181185E290E1DF91CF91D1
:104500001F910F91FF90EF90DF90CF900C946F1957
:104510002091C5103091C61040E050E0820F931FEB
:10452000A41FB51FC090A409D090A509E090A609CA
:10453000F090A709C816D906EA06FB0600F1C0905C
:10454000A409D090A509E090A609F090A709C81A7F
:10455000D90AEA0AFB0AC216D306E406F50608F0F1
:104560007ACF9E2D8D2D7C2D66270E94CA75F9016C
:10457000EE0FFF1FE056FC4FC081D1816ECFC0E02F
:10458000D0E06BCF00E010E08091E01081118FCF80
:10459000C901809590958E159F0530F54FEF5FEF1F
:1045A00060910B1170910C118AE090E10E946F19DB
:1045B0009E01AA27029FB12D139FC001309FB00D0D
:1045C000811D9A1F129FB00D811D9A1F11246091A9
:1045D000171170911811AC018FCF20E030E053CF4C
:1045E000A8014E0D5F1D84CFA9014E0D5F1DD8CFD0
:1045F00080915A1287FD09C06F7070E0992787FD7E
:1046000090956817790709F0089580E8289F900130
:104610001124242B3052220F331F220F331F3093CB
:104620009710209396100E940F156FEF81E00C9465
:1046300036594F925F926F927F928F929F92AF9274
:10464000BF92CF92DF92EF92FF920F931F93CF937F
:10465000DF938091551290915612909301018093AF
:104660000001C0900401D09005017C01EC18FD0808
:10467000C80ED91EC0910201D091030197012C1BD5
:104680003D0B40E050E0812C912CA12CF0E8BF2E96
:10469000C501B4010E94CA7529013A01209306019F
:1046A0003093070140930801509309018E01009552
:1046B000109598012C193D0940E050E0C501B40166
:1046C0000E94CA7549015A0120930A0130930B01D7
:1046D00040930C0150930D018091110C9091120C9C
:1046E00008171907E0F48FEF9FE7909397108093D6
:1046F00096100E940F156FEF81E0DF91CF911F910F
:104700000F91FF90EF90DF90CF90BF90AF909F9070
:104710008F907F906F905F904F900C9436598C17CC
:104720009D07C0F0AC0160E070E08E159F0530F091
:10473000C816D90690F080E090E0D7CFCB01BA013F
:104740006C1B7D0B81099109A30192010E94C77026
:104750009058CBCF80E090E8C8CF9A01AB012C19DC
:104760003D0941095109C501B4010E94C770905823
:104770009058BBCFCF93DF93CDB7DEB728970FB656
:10478000F894DEBF0FBECDBF92E09D8394E09E8380
:1047900097E09F839CE0988795E0998393E09A83C4
:1047A00091E09B831C82823081F134F4882361F094
:1047B000813009F069C013C0843009F450C0D4F1CD
:1047C000853009F061C05AC0440F551F661F771F1E
:1047D0008091D2108170842B8093D21055C080912B
:1047E000D4108F7C413051056105710521F4806141
:1047F0008093D41049C0423051056105710509F01C
:1048000001C080628093D4103FC0DB01CA01817077
:104810009927AA27BB2721E082278093D8104270CE
:104820005527662777277595679557954795409340
:10483000E2102AC0DB01CA0181709927AA27BB2791
:1048400021E082278093D61042705527662777276C
:1048500075956795579547954093D71015C0FE01FC
:10486000E40FF51F85818093DC1028960FB6F8942D
:10487000DEBF0FBECDBFDF91CF91DBCEFE01E40FD7
:10488000F51F81818093DE1028960FB6F894DEBF65
:104890000FBECDBFDF91CF910895BF92CF92DF922F
:1048A000EF92FF920F931F93CF93DF93CDB7DEB7B5
:1048B00064970FB6F894DEBF0FBECDBF00913311E1
:1048C0008CE008028001112400561A4F0E947418CF
:1048D000D80112966D917C911397CE0101960E949A
:1048E000F27467EC78E0CE0101960E94E774F8015B
:1048F00080818130D9F020F0823009F05EC029C07B
:10490000E181EE0FFF0BED51FF4E8081918190937D
:104910002E1180932D11A0E0B0E080932911909387
:104920002A11A0932B11B0932C1147C0E181FF27CE
:10493000E7FDF095E753FF4E8081F801E80FF11D88
:10494000E80FF11D64817581CE0101960E94E77424
:1049500034C08AE1E9ECF0E1AFE9B7E101900D92F2
:104960008A95E1F7C12CD12C7601B701A601F80197
:10497000818100DF4AE150E069EC70E18FE997E165
:104980000E94B974009771F4F8018C2D92E08902AD
:10499000E00DF11D112464817581CE0101960E9404
:1049A000E7740BC0AFEFCA1ADA0AEA0AFA0AB4E0EF
:1049B000CB16D104E104F104C1F6CE0101960E94A8
:1049C0001A1764960FB6F894DEBF0FBECDBFDF9105
:1049D000CF911F910F91FF90EF90DF90CF90BF90FC
:1049E0000895CF92DF92EF92FF920F931F93CF9390
:1049F0008091030D833009F49CC08091040D8330B5
:104A000009F4B7C080912511882309F4B4C081301E
:104A100009F4DEC08091261187FDD5C060E2805D7B
:104A20000E94F6166091591284E00E94CF16809180
:104A3000251181115EC061E080915912882309F42B
:104A400058C086E00E94CF166091B809617087E077
:104A50000E94CF168091030D41E0823009F467C0B7
:104A600061E0811101C060E080E00E94A0168091A9
:104A7000040D41E0823009F458C061E0811101C0A9
:104A800060E081E00E94A01661E08091020D81301B
:104A900009F060E082E00E94CF168091020D41E0B3
:104AA000823009F040E061E0823008F460E083E0A9
:104AB0000E94A0168091020D81111DC08091030DEE
:104AC0008330C9F08091040D8330A9F080912511C5
:104AD00061E0823019F0843009F060E0462F85E013
:104AE000CF911F910F91FF90EF90DF90CF900C949A
:104AF000A01660E0A6CF8091010D882359F061E0F7
:104B000085E0CF911F910F91FF90EF90DF90CF90B4
:104B10000C94CF168091030D61E0833089F380916E
:104B2000040D833069F360E0EBCF40E0A6CF40E0B6
:104B300097CF2091040D81E090E0233011F080E0C8
:104B400090E08D5F924FFC01EE5FFE4FC0816C2FB5
:104B500070E080E090E00E940A1741E0C03809F060
:104B600040E061E0C43608F460E089E00E94A016ED
:104B700059CF23E0E0CF60E089E00E94CF1680911A
:104B8000291190912A11A0912B11B0912C11B7FDF0
:104B90001AC0E0912811E031E1F120912D113091FE
:104BA0002E11A4E6B0E00E94BE756C01FF24D7FC74
:104BB000F094EF2C8E2FA6D8811118C0C701B60132
:104BC0000E940A172FCF60E280E20E94F6162ACFD9
:104BD000609157127091581280E090E00E940A177D
:104BE0006091271189E00E94CF161CCF82E3C81A7A
:104BF000D108D7FC2AC0EE24D7FCE094FE2C6091AB
:104C00002E116095661F6627661F89E00E94CF16E9
:104C1000D5CF8091110C9091120CA0910001B09110
:104C20000101E0900401F090050160910201709192
:104C300003019B01209530952817390750F423E68E
:104C4000C22ED12CE12CF12CB5CFD194C194D10836
:104C5000D2CF8617970760F18C0120E030E06D011C
:104C6000CE18DF088C159D0538F5A9019801261B83
:104C7000370B41095109609106017091070180913C
:104C80000801909109010E94C7709C013058442787
:104C900037FD4095542F30584F4F5F4FA4E6B0E09A
:104CA0000E947F756C01FF24D7FCF094EF2C82CF1B
:104CB000C12CD12C76017ECFAE0DBF1DA817B90730
:104CC00030F092E3C92ED12CE12CF12C73CFA90145
:104CD00098012A1B3B0B4109510960910A0170910F
:104CE0000B0180910C0190910D010E94C7709058AA
:104CF000CCCF9091810B8091800B2091820B211160
:104D000031C02091370F2111EBC120918D0B211162
:104D10006CC02091610F211151C12091980B21117C
:104D200056C020918B0F2111B7C02091A30B2111E8
:104D300040C02091B50F21118AC12091AE0B2111E5
:104D40002AC02091DF0F2111F0C02091B90B211151
:104D500014C020910910211156C09093810B8093AB
:104D6000800B08952091370F2111CFCF1092820B25
:104D70001092840B8FEF9FEFC8CF20910910211163
:104D8000ECCF1092B90B1092BB0B2FEF2093B80B06
:104D90002093B70BE2CF2091DF0F2111D6CF1092D5
:104DA000AE0B1092B00B2FEF2093AD0B2093AC0BFA
:104DB000CCCF2091B50F2111C0CF1092A30B109230
:104DC000A50B2FEF2093A20B2093A10BB6CF209120
:104DD0008B0F2111AACF1092980B10929A0B2FEFE4
:104DE0002093970B2093960BA0CF2091610F211158
:104DF00094CF10928D0B10928F0B2FEF20938C0B72
:104E000020938B0B8ACF10920710109205101092EE
:104E100004101092E40F1092E50F1092E60F10921A
:104E2000E70F1092FF0F1092FE0F109209101092D0
:104E300001101092001010920310109202101092A4
:104E4000E00F1092E10F1092E20F1092E30F109218
:104E50000B0F1092090F1092080F1092E80E10928B
:104E6000E90E1092EA0E1092EB0E1092030F1092C0
:104E7000020F10920D0F1092050F1092040F109256
:104E8000070F1092060F1092E40E1092E50E10928A
:104E9000E60E1092E70E61CF1092890F1092870FE5
:104EA0001092860F1092660F1092670F1092680F83
:104EB0001092690F1092810F1092800F10928B0F39
:104EC0001092830F1092820F1092850F1092840F10
:104ED0001092620F1092630F1092640F1092650F80
:104EE00010928D0E10928B0E10928A0E10926A0EF6
:104EF00010926B0E10926C0E10926D0E1092850E29
:104F00001092840E10928F0E1092870E1092860EC1
:104F10001092890E1092880E1092660E1092670EF3
:104F20001092680E1092690E00CF1092DD0F109251
:104F3000DB0F1092DA0F1092BA0F1092BB0F109283
:104F4000BC0F1092BD0F1092D50F1092D40F10927B
:104F5000DF0F1092D70F1092D60F1092D90F109228
:104F6000D80F1092B60F1092B70F1092B80F109280
:104F7000B90F1092E10E1092DF0E1092DE0E109219
:104F8000BE0E1092BF0E1092C00E1092C10E109263
:104F9000D90E1092D80E1092E30E1092DB0E1092E2
:104FA000DA0E1092DD0E1092DC0E1092BA0E1092F4
:104FB000BB0E1092BC0E1092BD0EC7CE10925F0FAA
:104FC00010925D0F10925C0F10923C0F10923D0FEB
:104FD00010923E0F10923F0F1092570F1092560FE3
:104FE0001092610F1092590F1092580F10925B0F90
:104FF00010925A0F1092380F1092390F10923A0FE8
:1050000010923B0F1092630E1092610E1092600E80
:105010001092400E1092410E1092420E1092430ECA
:1050200010925B0E10925A0E1092650E10925D0E49
:1050300010925C0E10925F0E10925E0E10923C0E5B
:1050400010923D0E10923E0E10923F0E66CE1092C0
:10505000B30F1092B10F1092B00F1092900F1092E8
:10506000910F1092920F1092930F1092AB0F10921B
:10507000AA0F1092B50F1092AD0F1092AC0F1092B4
:10508000AF0F1092AE0F10928C0F10928D0F1092E6
:105090008E0F10928F0F1092B70E1092B50E1092C5
:1050A000B40E1092940E1092950E1092960E1092CD
:1050B000970E1092AF0E1092AE0E1092B90E109283
:1050C000B10E1092B00E1092B30E1092B20E10925A
:1050D000900E1092910E1092920E1092930E2DCE71
:1050E0001092350F1092330F1092320F1092120F50
:1050F0001092130F1092140F1092150F10922D0F83
:1051000010922C0F1092370F10922F0F10922E0F1B
:105110001092310F1092300F10920E0F10920F0F4D
:105120001092100F1092110F1092390E1092370E2C
:105130001092360E1092160E1092170E1092180E34
:105140001092190E1092310E1092300E10923B0EEA
:105150001092330E1092320E1092350E1092340EC1
:105160001092120E1092130E1092140E1092150E31
:10517000CCCD80915D12813009F00895683FE9F04F
:105180006A3FD9F78FEF9FEF9093080E8093070E39
:105190002FEF3FE730930F0E20930E0E90930A0EE1
:1051A0008093090E9093F90C8093F80C3093FE0CC9
:1051B0002093FD0C1092C71008958091C7108F5F47
:1051C0008093C71008959091030D933021F0909132
:1051D000040D9330E9F48130C1F028F0823079F089
:1051E0008330B1F406C08BEC98E00E941A1781E876
:1051F0000DC081ED98E00E941A178EEF07C086ED72
:1052000098E00E941A178DEF01C08CEF0C94141FC8
:105210000895CF92DF92EF92FF92CF939091CB10AF
:105220002091CE10992309F490C04091E71050913D
:10523000E81060E070E0222309F483C0C090ED1014
:10524000D090EE10E12CF12C8823A1F0992381F06D
:105250008091D41085FD0CC0809120109091211078
:10526000AA2797FDA095BA2F480F591F6A1F7B1FC9
:10527000211170C0CFB7F8944115510521E06207A4
:10528000710524F04FEF5FEF60E070E0DB01CA01D1
:1052900077FD75C0E8D146EC41BB469A31E035B99F
:1052A00021E428B950EF5BB992EA9EB987E881BB47
:1052B00000C000C041BB469A35B928B960E76BB958
:1052C0009EB981BB00C000C041BB469A35B928B920
:1052D0005BB99EB981BBD701C601C114D10421E0DD
:1052E000E206F10424F08FEF9FEFA0E0B0E0B7FDFD
:1052F00042C0B9D146EC41BB469A31E035B927E40A
:1053000028B950EF5BB992EA9EB987E881BB00C02B
:1053100000C041BB469A35B928B960E76BB99EB960
:1053200081BB00C000C041BB469A35B928B95BB902
:105330009EB981BBCFBFCF91FF90EF90DF90CF9010
:105340000895C12CD12C76017FCF4FEF5FEF60E045
:1053500070E071CF8091D41084FD8CCF80912010AB
:1053600090912110AA2797FDA095BA2FC80ED91E9B
:10537000EA1EFB1E7FCF80E090E0DC01BACF80E028
:1053800090E0DC0187CF6095EBE8F4E19081982B09
:105390006923608386EC81BB469A362F330F962FA4
:1053A0009695262F221F2227221F832F8670282BB7
:1053B00020646071832F880F8072862B307C832B52
:1053C0009270906C31E035B928B98BB99EB987E8F5
:1053D00081BB85E08A95F1F70000EAE8F4E180817D
:1053E0008F5F80830895809590918B14892380939B
:1053F0008B1496EC91BB469A482F440F282F269584
:10540000382F331F3327331F942F9670392B306476
:105410008071942F990F9072982B407C942B22705E
:10542000206C81E085B938B99BB92EB987E881BB7A
:1054300085E08A95F1F7000080918A148F5F809350
:105440008A14089580918B14806180938B1496EC5C
:1054500091BB469A382F330F982F9695282F221FED
:105460002227221F832F8670282B2064832F880FEA
:1054700080728061307C832B9270906C31E035B902
:1054800028B98BB99EB987E881BB85E08A95F1F789
:10549000000080918A148F5F80938A140895809110
:1054A0008B1481608F7E80938B1496EC91BB469A0F
:1054B000382F330F982F9695881F8827881F232F02
:1054C0002670822B8064232F220F2072307C232BA6
:1054D0009270906C31E035B988B92BB99EB987E8E4
:1054E00081BB85E08A95F1F7000080918A148F5F77
:1054F00080938A14089530918B14832F88608E7F57
:1055000080938B1496EC91BB469A282F220F982FEC
:105510009695881F8827881F422F4670842B8064A9
:10552000207C30713062232B9270906C31E035B961
:1055300088B92BB99EB987E881BB85E08A95F1F7D8
:10554000000080918A148F5F80938A14089540919F
:105550008B14242F226020938B1486EC81BB469AF7
:10556000322F330F922F9695221F2227221F832F2F
:105570008670282B2064832F880F80724071842BC3
:10558000307C832B9270906C31E035B928B98BB99F
:105590009EB987E881BB85E08A95F1F7000080918C
:1055A0008A148F5F80938A1408954FB7F89480917E
:1055B000770C96EC91BB469A382F330F982F96951F
:1055C000232F26702064582F551F5527551F252B34
:1055D000582F5071832F880F8072852B307C832B3E
:1055E0009270906631E035B928B98BB99EB987E8D9
:1055F00081BB4FBF08959091770C977F8111986080
:105600009093770CD2CF9091770C9E7F811191600F
:105610009093770CCACF9091770C9B7F8111946007
:105620009093770CC2CF9091770C9F7B81119064FF
:105630009093770CBACF9091770C9F7D81119062F7
:105640009093770CB2CF9091770C9F7E81119061EF
:105650009093770CAACF9091770C9D7F81119260E7
:105660009093770CA2CF9C01232F33272695269564
:10567000722F66EC61BB469A522F550F452F46702C
:105680004068207133272260352F330F3072322B60
:10569000507C352B272F26952270206215B848B9EB
:1056A0003BB92EB957E851BB969587959695879546
:1056B000282F61BB469A482F440F382F3695221F5A
:1056C0002227221F642F6670262B2068807199275D
:1056D0008260942F990F9072982B407C942B32709B
:1056E00015B828B99BB93EB951BB08951F93CF9304
:1056F000DF93D82FD86F86958695869528E030E081
:1057000001C0220F8A95EAF7C22FC095CD231FB79B
:10571000F894CB01A8DFE6ECE1BB469A3D2F330FAE
:10572000367031649D2F96959270906A71E075B9CC
:1057300038B9A0EFABB99EB967E861BB85E08A953F
:10574000F1F70000E1BB469AFC2FFF0F4C2F469566
:105750005C2F551F5527551F8F2F8670582B50646F
:10576000C0718F2F880F80728C2BF07C8F2B427032
:10577000406A75B958B98BB94EB961BB8AE08A9550
:10578000F1F700C0E1BB469A75B938B9ABB99EB91B
:1057900061BB8AE08A95F1F700C01FBFDF91CF910E
:1057A0001F910895E82FF0E0EE0FFF1FE95CF34F23
:1057B000718360830895E82FF0E0EE0FFF1FE95C2E
:1057C000F34F118210820895E82FF0E0EE0FFF1FD3
:1057D000E95CF34F86EC94E9918380830895E82F88
:1057E000F0E0EE0FFF1FE95CF34F83E094E6918356
:1057F00080830895E82FF0E0EE0FFF1FE95CF34F80
:1058000082EA9BEB918380830895E82FF0E0EE0F0E
:10581000FF1FE95CF34F83E99BE591838083089543
:10582000E82FF0E0EE0FFF1FE95CF34F8FEF9FEFE3
:1058300091838083089560FD05C090936C0C8093E4
:105840006B0C0895BC018AE151CF60FD05C09093B7
:105850006A0C8093690C0895BC0189E147CF60FD13
:1058600005C09093740C8093730C0895BC018EE175
:105870003DCF0E94012061E088E00E94CF168BE1BD
:105880009ADF80E0C0DE80E0E6DE80E0B4DE80E02B
:10589000DADE80E0D0DE80E0C6DE80E0BCDE60E004
:1058A00080E090E0DCDF8CE186DF8FE184DF88E15F
:1058B00082DF8DE180DF0E945C130E946D130C94E7
:1058C0007E13EF92FF920F931F93CF93DF937C0190
:1058D000EB01142F40FF09C02091831430918414F0
:1058E000282739272C7F232B71F511FF0AC08091BF
:1058F0008514909186148C279D2788279E7F892B5D
:1059000039F4DF91CF911F910F91FF90EF9008959F
:105910000D2F069540915B124F70406BE0919F19DF
:10592000F091A01921E063E070E08FE999E1099519
:10593000D0938614C0938514DF91CF911F910F915E
:10594000FF90EF90089590589C01359527953595D7
:105950002795092F06952F77332740915B124F70BB
:10596000406EE0919F19F091A01963E070E08FE91B
:1059700099E10995F0928414E0928314B6CF0F93C5
:105980001F93072F069510E00F771127282F2F77E9
:1059900040915B124F704069E0919F19F091A019FE
:1059A00063E070E08FE999E109951F910F910895E7
:1059B0000F93262F4F772F778F708068E0919F1974
:1059C000F091A019042F482F63E070E08FE999E16E
:1059D00009950F91089596EC91BB469A982F96954C
:1059E000969596958295880F807E95B990E498B9A2
:1059F0001BB88EB987E881BB85E08A95F1F7000076
:105A0000089536EC20EE97E0A0E8F7E4E7EE77EFB4
:105A100062EE5FB7F89431BB469A27B99AB92DB9AF
:105A200015B8A8B99BB91EB8F1BB42E04A95F1F789
:105A300000C046B1B9B1BCB131BB479AE7B97AB938
:105A40006DB95FBF55E05A95F1F7000042FFE1CF15
:105A50005FB7F89496EC91BB469A382F330F982F86
:105A60009695232F26702068482F441F4427441FF3
:105A7000242B80718360432F440F4072842B307C31
:105A8000832B9270906215B828B98BB99EB987E8BC
:105A900081BB85E08A95F1F700005FBF089526EC91
:105AA00090EE87E0F0E8E7E477EE67EF52EE4FB76D
:105AB000F89421BB469A97B98AB99DB915B8F8B937
:105AC0008BB91EB8E1BB32E03A95F1F700C036B1B0
:105AD000A9B1ACB121BB479A77B96AB95DB94FBFDB
:105AE00045E04A95F1F7000032FFE1CF9FB7F89407
:105AF00086EC81BB469A15B887E888B923ED2BB9A7
:105B000022E22EB981BB85E08A95F1F700009FBFA4
:105B10000895CF93DF930E943718C82FD0E00E94DA
:105B20003718382F20E0C22BD32B81E054DF81E0DF
:105B300052DF86EC81BB469A15B882E488B91BB85F
:105B400080E48EB987E881BB85E08A95F1F7000093
:105B500082E041DFC095D095CE01DF91CF910895CD
:105B6000CF93882339F180912F0A8F5F80932F0A7A
:105B7000853148F081E09091300A9111CDC0809339
:105B8000300A10922F0AC091330AC11179C0509186
:105B90002D0A90912E0AE091340AE13009F4DEC01A
:105BA00008F4AFC0E23009F4C4C020E0F0E0E75DE3
:105BB000F54F2487AFB7F89456EC51BB469A41E0B5
:105BC00045B980E488B91BB880E28EB937E831BBAB
:105BD00000C000C080E190E00090340A02C0880F4D
:105BE000991F0A94E2F7282F51BB469A782F770F16
:105BF000682F6695221F2227221F972F9670292B28
:105C000020648071972F990F9072982B707C972B3E
:105C1000627045B928B99BB96EB931BB00C000C0EC
:105C2000E091340AF0E0E75DF54F848551BB469A78
:105C3000582F550F982F9695252F26702064682F82
:105C4000661F6627661F262B682F6071852F880FB9
:105C50008072862B507C852B9270906245B928B952
:105C60008BB99EB931BBAFBF8091340A90E00196E9
:105C700063E070E00E94E2708093340ACF9108954F
:105C80004091310A4F5F4093310AE8E3FAE0019016
:105C90000020E9F7E953FA402091320A332727FD23
:105CA0003095C90101966E2F772767FD70950E9488
:105CB000E270F901E75DF54F278530E020383105C6
:105CC00088F15FEFE82FFF27E7FDF095E75DF54FDF
:105CD000278530E02038310550F5F901E45EFE4FAC
:105CE0009081403108F457CF8093320A1092310AE4
:105CF000811151CF1C160CF04ECFC150C093330A06
:105D00004ACF2091290A8091300A882309F44ECF86
:105D100080912B0A28274ACF80E08093300A109286
:105D20002F0A31CFF901E45EFE4F5081CBCF9FEFB8
:105D3000D8CF292F2F778091290A90912A0A90FD98
:105D4000206880912B0A90912C0A90FF2FCF809190
:105D5000300A882309F42ACF205828CF252F2F77FF
:105D60008091290A90912A0A91FD206880912B0A3E
:105D700090912C0A91FF1ACFEACFCF9380912F0AEE
:105D80008F5F80932F0A853148F081E09091300A2F
:105D90009111D3C08093300A10922F0AC091330A18
:105DA000CC2309F441C04091310A4F5F4093310A3E
:105DB000E8E3FAE001900020E9F7E953FA40209186
:105DC000320A332727FD3095C90101966E2F7727B8
:105DD00067FD70950E94E270F901E75DF54F278538
:105DE00030E02038310508F4A3C05FEFE82FFF272B
:105DF000E7FDF095E75DF54F278530E02038310568
:105E000008F09DC0F901E45EFE4F9081403180F0C2
:105E10008093320A1092310A81110AC01C1644F490
:105E2000C150C093330A04C050912D0A90912E0A9C
:105E3000E091340AE13009F499C008F46EC0E23010
:105E400009F47FC020E0F0E0E75DF54F2487AFB7AD
:105E5000F89456EC51BB469A41E045B980E488B9C4
:105E60001BB880E28EB937E831BB00C000C080E1CA
:105E700090E00090340A02C0880F991F0A94E2F75C
:105E8000282F51BB469A782F770F682F6695221FCF
:105E90002227221F972F9670292B20648071972F1D
:105EA000990F9072982B707C972B627045B928B926
:105EB0009BB96EB931BB00C000C0E091340AF0E07C
:105EC000E75DF54F848551BB469A582F550F982FA3
:105ED0009695252F26702064682F661F6627661FFB
:105EE000262B682F6071852F880F8072862B507C3F
:105EF000852B9270906245B928B98BB99EB931BB98
:105F0000AFBF8091340A90E0019663E070E00E9498
:105F1000E2708093340ACF9108952091290A8091EC
:105F2000300A882309F48FCF80912B0A28278BCF42
:105F3000F901E45EFE4F508159CF80E02BCF9FEFF7
:105F400065CF292F2F778091290A90912A0A90FDF9
:105F5000206880912B0A90912C0A90FF74CF809139
:105F6000300A882309F46FCF20586DCF252F2F7763
:105F70008091290A90912A0A91FD206880912B0A2C
:105F800090912C0A91FF5FCF8091300A882309F409
:105F90005ACFEACF86EC81BB469A15B896E898B9F5
:105FA00093E09BB91EB897E891BBEFE9FFE031970A
:105FB000F1F700C0000081BB469A15B823E828B964
:105FC00023E12BB922E02EB991BBFAE0FA95F1F763
:105FD00000C081BB469A20EE27B997E09AB92DB947
:105FE00015B820E828B99BB91EB897E491BB92E098
:105FF0009A95F1F700C096B199B19CB181BB479ACF
:1060000087EE87B987EF8AB982EE8DB9EAE0EA9523
:10601000F1F700C0089526EC90EE87E0F0E8E7E4A1
:1060200077EE67EF52EE4FB7F89421BB469A97B9D7
:106030008AB99DB915B8F8B98BB91EB8E1BB32E081
:106040003A95F1F700C036B1A9B1ACB121BB479A7E
:1060500077B96AB95DB94FBF45E04A95F1F70000DD
:1060600032FFE1CF8FB7F89496EC91BB469A15B802
:1060700091E898B993ED9BB990E29EB997E891BBEE
:1060800095E09A95F1F700008FBF08950F931F9345
:10609000CF93DF9380E492E4AFE0B0E036EC20EE03
:1060A00017E0D1E0C0E4F0E2E7E477EE67EF52EE0C
:1060B00004C00097A105B10521F131BB469A27B96B
:1060C0001AB92DB9D5B9C8B91BB8FEB9E1BB42E0C0
:1060D0004A95F1F700C046B109B10CB131BB479AFE
:1060E00077B96AB95DB90197A109B10942FDE1CF5C
:1060F000892B8A2B8B2B29F0DF91CF911F910F9148
:106100000895DF91CF911F910F910C940B1F0F9366
:106110001F93CF93DF9380E492E4AFE0B0E036ECDE
:1061200020EE17E0D1E0C0E4F0E2E7E477EE67EFBD
:1061300052EE04C00097A105B10521F131BB469A8A
:1061400027B91AB92DB9D5B9C8B91BB8FEB9E1BB81
:1061500042E04A95F1F700C046B109B10CB131BB3C
:10616000479A77B96AB95DB90197A109B10942FFA8
:10617000E1CF892B8A2B8B2B29F0DF91CF911F91B7
:106180000F910895DF91CF911F910F910C940B1FE8
:106190001F93CF93DF9380E492E4AFE0B0E036EC5E
:1061A00020EE17E0D1E0C0E4F0E2E7E477EE67EF3D
:1061B00052EE04C00097A105B10519F131BB469A12
:1061C00027B91AB92DB9D5B9C8B91BB8FEB9E1BB01
:1061D00042E04A95F1F700C046B149B14CB131BB3C
:1061E000479A77B96AB95DB90197A109B10941FD2B
:1061F000E1CF892B8A2B8B2B21F0DF91CF911F913F
:106200000895DF91CF911F910C940B1F1F93CF9393
:10621000DF9380E492E4AFE0B0E036EC20EE17E0EC
:10622000D1E0C0E4F0E2E7E477EE67EF52EE04C0BD
:106230000097A105B10519F131BB469A27B91AB9E2
:106240002DB9D5B9C8B91BB8FEB9E1BB42E04A9532
:10625000F1F700C046B149B14CB131BB479A77B9AB
:106260006AB95DB90197A109B10941FFE1CF892B55
:106270008A2B8B2B21F0DF91CF911F910895DF9115
:10628000CF911F910C940B1F2F923F924F925F92D0
:106290006F927F928F929F92AF92BF92CF92DF9236
:1062A000EF92FF920F931F93CF93DF93CDB7DEB79B
:1062B00028970FB6F894DEBF0FBECDBF8D832FB7E2
:1062C0002E83F894282F259525952595259580E2F0
:1062D00090E002C0959587952A95E2F79D819F7081
:1062E000982B86EC81BB469A492F440F292F26957F
:1062F000392F331F3327331F842F8670382B306498
:106300009071842F880F8072892B407C842B22709F
:10631000206491E095B938B98BB92EB987E881BB73
:1063200035E03A95F1F700002D81332727FD3095B0
:106330003A832983F901E852F94FC080D12C80E1DA
:1063400090E08C199D092FEF3FEF082E02C0369583
:1063500027950A94E2F702C0220F331F8A95E2F7CD
:106360003C832B83E12CF12C00E010E82FEF3FEF72
:1063700056ECA52E60EEB62E77E0272E332433940C
:10638000E0E44E2EF0E25F2EA7E46A2EB7EE7B2EFD
:1063900087EF882E92EE992E0AC0200F311F169596
:1063A0000795AFEFEA1AFA0ACE14DF042CF1C901FF
:1063B0002F83388758D982E08A95F1F700C0A1BAB7
:1063C000469AB7B82AB8BDB835B848B81BB85EB851
:1063D00061BA92E09A95F1F700C086B189B19CB19B
:1063E000A1BA479A77B88AB89DB82F81388585FDBC
:1063F000D4CF201B310BD3CF86EC81BB469A81E0F2
:1064000085B987E488B980EF8BB982E48EB987E8D3
:1064100081BBB5E0BA95F1F70000EB81FC812E233A
:106420003F23E981FA81EE0FFF1FEF50F44F3183D4
:106430002083232F3327E981FA81E353F44F8481AA
:1064400090E0821B930B97FD1DC0059704F53E81DC
:106450003FBF28960FB6F894DEBF0FBECDBFDF91C9
:10646000CF911F910F91FF90EF90DF90CF90BF9051
:10647000AF909F908F907F906F905F904F903F90E4
:106480002F900895919581959109059704F32483A0
:1064900081E090E0A0E0B0E00D8004C0880F991F7B
:1064A000AA1FBB1F0A94D2F74091CD0B5091CE0B7F
:1064B0006091CF0B7091D00B842B952BA62BB72B13
:1064C0008093CD0B9093CE0BA093CF0BB093D00BBA
:1064D0002D812093320CBBCFCF93DF9320915A12A2
:1064E00027FD0BC06F7070E0332727FD30956217D2
:1064F000730719F0DF91CF91089580915912882385
:10650000C9F34436B8F7C42FD0E080915712909168
:106510005812C817D90771F3CE010E94B61A882302
:1065200049F3D0935812C0935712109227110E942A
:106530008F54DF91CF910C94D8460F931F93CF9334
:10654000DF93CDB7DEB7C455D1090FB6F894DEBFDF
:106550000FBECDBF92E2E8EFF6E0DE01D3960190E8
:106560000D929A95E1F7813031F580915A12992771
:1065700087FD9095029661E170E00E94E270815083
:1065800080935A120E948F54E0915A12FF27E7FD20
:10659000F0953196EE0FFF1F81E090E08C0F9D1F6C
:1065A000E80FF91F62A973A9CE0101960E94F27447
:1065B0006AED78E026C0823069F580915B129927F8
:1065C00087FD9095019660E170E00E94E2708093F3
:1065D0005B120E948F54E0915B12FF27E7FDF0955C
:1065E0003196EE0FFF1F81E090E08C0F9D1FE80FAA
:1065F000F91F62A973A9CE0101960E94F27460EEA0
:1066000078E0CE0101960E94E774CE0101960E94C7
:106610001A1703C1833089F48091110C9091120CE8
:1066200090935612809355120E948F540E94192302
:1066300086EE98E00E941A17F0C08430D1F4809161
:106640008714992787FD9095019666E070E00E9477
:10665000E270182F8093871468EF78E0CE010196DE
:106660000E94F2741F5C1B83CE0101960E941A17D0
:10667000D4C08530E9F510915C1200918714212F68
:1066800030E0002E02C0359527950A94E2F720FFEE
:1066900012C06CEF78E0CE0101960E94F27421E006
:1066A00030E0002E01C0220F0A94EAF72095212342
:1066B00020935C1210C064E079E0CE0101960E9444
:1066C000F27481E090E0002E01C0880F0A94EAF78E
:1066D000812B80935C120E948F54809187148F5C71
:1066E0008B83CE0101960E941A170E94D84695C04E
:1066F000863059F40E9467628BE099E00E941A1775
:106700000E943B480E94D84688C0883029F5809175
:106710005D12992787FD9095019663E070E00E94D5
:10672000E27080935D120E948F5480915D128130DF
:1067300049F0823061F081116EC08AE199E00E94D7
:106740001A1769C083E299E00E941A1764C08DE2AB
:1067500099E00E941A175FC0893009F051C081E0AA
:1067600090915E12911101C080E090915F12992387
:1067700011F092E001C090E0890F90E001969C0139
:106780002170332720935E1283709927869580931A
:106790005F120E948F5467E379E0CE0101960E9458
:1067A000F27480915E12882339F068E079E0CE01BE
:1067B00001960E94E77406C060E079E0CE01019680
:1067C0000E94E7746FE379E0CE0101960E94E774BE
:1067D00080915F12882339F068E079E0CE0101965C
:1067E0000E94E77406C060E079E0CE0101960E9445
:1067F000E774CE0101960E941A170E94D8460DC078
:1068000081110BC00E94FE1981E0809327118BE457
:1068100099E00E941A170E94D846CC5ADF4F0FB653
:10682000F894DEBF0FBECDBFDF91CF911F910F91C6
:10683000089520919C1730919D172C593541213096
:10684000324038F4BC0180E090E04CE955E10C9412
:1068500066540895FF920F931F93CF93DF938C019B
:10686000FFB60E94FB19882309F43FC00E94D71984
:10687000C0E0EC2FF0E0EE0FFF1FED51FF4E8081E6
:1068800091810E94F119CF5FC93199F78091E2108F
:106890008093D910D0E0ED2FF0E0E753FF4E8081D8
:1068A0000E94CC19DF5FD731B1F7EC2FF0E0EE0F8B
:1068B000FF1FED51FF4E808191810E94F119CF5F42
:1068C000CE3199F78091E0100E94CC198091E110AF
:1068D0000E94CC19CFE1D1E189910E94CC1981E1CC
:1068E000C532D807C9F7C801A4DF8F2DDF91CF913A
:1068F0001F910F91FF900C94BF19609133118A3052
:1069000030F5681305C0862F865F8093331114C05D
:10691000462F552747FD5095282F332727FD3095C3
:10692000265F3F4F4217530729F4862F8A508093E2
:10693000331102C0809333118FEF9FEFDC018093FE
:106940002F1190933011A0933111B0933211809197
:106950003311861749F00E944D24809159128111FC
:1069600003C08BED90E076CF0895FF920F931F93B5
:10697000CF93DF93F82EEB010FB70E94FB1988230A
:1069800081F00E94D71911E803C089910E94CC19A7
:106990001150D9F78F2D992787FD909588539F4FD8
:1069A00048DF802FDF91CF911F910F91FF900C94C2
:1069B000BF19BF92CF92DF92EF92FF920F931F9376
:1069C000CF93DF93B62E082F112707FD1095E8010E
:1069D000CD5FD24F9881691761F0992329F19330E7
:1069E00009F44FC0923009F45EC082E0B81659F045
:1069F000B882DF91CF911F910F91FF90EF90DF90C0
:106A0000CF90BF900895F801EE0FFF1FE95FF14F9F
:106A10008FEF9FEF918380838FEF9FE790930F0E0F
:106A200080930E0EB882E5CF7801F694FE2CEE240A
:106A3000F794E79475E0C72E7DE0D72ECE0CDF1CCF
:106A4000B6010E948D1A882331F1FE01EE5FFE4FE0
:106A500080E88083F701EC57F24F80818F3F29F661
:106A6000DE01AE5FBE4F8FE78C93F701EC57F24F1C
:106A70008EE792919F3F09F0B8CF8C938150C8F771
:106A8000B4CFB8017695762F6627779567956B5FBB
:106A9000724F6BDFAACF40E850E06FEF70E0C601A5
:106AA0000E94E074D2CF60E00E945B579ECFCF93EC
:106AB000DF93DFB70E94111F882309F474C00E947E
:106AC000931E0E94392C60E080E090E00E942F2C01
:106AD000C2E18C2F0E94DB2B8C2F86500E94102C41
:106AE000CF5FC831B1F781E00E94032B60E08FEFE8
:106AF0009FEF0E94252C60E080E090E00E941B2C1C
:106B0000C0E06C2F6E5E8C2F0E944550CF5FC63068
:106B1000C1F780E00E94032B81E00E94FB2A60E025
:106B200080E090E00E94252C60E08FEF9FEF0E94B4
:106B30001B2C6C2F645F8C2F0E944550CF5FCC3094
:106B4000C1F780E00E94FB2A60E080E090E00E94B4
:106B5000252C60E080E090E00E941B2C60E08FEF2D
:106B60009FEF0E942F2C8C2F0E94DB2BCF5FC23116
:106B7000D1F7CCE06C2F6A5F8C2F0E944550CF5F1D
:106B8000C231C1F760E080E090E00E942F2C8C2F92
:106B90000E94DB2BCF5FC831D1F70E94A64B0E9429
:106BA00001200E948F548D2FDF91CF910C94091FEB
:106BB0000F931F93CF93DF93182FEB010E94BC47D5
:106BC000209709F04CC1123191F571DF30C081E09E
:106BD000113109F080E0E82FF0E0ED5FF24F908195
:106BE000913001F128F0923001F1933001F512C09B
:106BF00090912511923031F463E0DBDE85E08093E3
:106C0000251115C090913411992311F061E00EC047
:106C100062E00CC091E020915912211101C090E076
:106C20009093251162E0C5DE02C060E0C2DE809173
:106C3000030D811104C08091040D8823E1F0209799
:106C400009F443C01D3009F010C181E09091040D9A
:106C5000911101C080E0E82FF0E0ED5FF24F9081EC
:106C6000933011F462E001C063E0A3DE85E080931D
:106C7000251101E02BC000E0209741F19091020D19
:106C80001A3049F481E0913009F480E06091010DFF
:106C90000E946B561BC01B30C9F4923081F018F073
:106CA0009330A1F406C06091010D83E00E946B5601
:106CB0000DC06091010D82E00E946B5607C060918B
:106CC000010D80E00E946B5601C000E08091020D32
:106CD000882379F0209709F4CEC01D3009F0C7C091
:106CE00061E09091010D911160E00E946B5601E00E
:106CF0002DC0173289F4209719F00E94EB1702C0BB
:106D00000E94CE170E942D188091591281111BC02C
:106D10008BED90E09FDD17C0209789F01E3079F44D
:106D200080915912882391F080912511882319F0C0
:106D3000109225110BC081E08093251107C01F30F0
:106D400011F4C0933411CD2B09F483C08091B8099C
:106D500080FF03C0812FF1DB7CC01C30A9F480913F
:106D60005912811103C08BED90E074DD81E09091A8
:106D70005912911180E0809359120E948F540E9401
:106D80003B480E94D84665C0909125111D30B1F452
:106D9000011114C0923011F0943061F481E09091AF
:106DA0005912911101C080E0809325118FEF8093DB
:106DB00026114FC082E0809325114BC0953021F4FD
:106DC000812F0E94E32845C0911103C0812F95DDDA
:106DD00040C01A3008F03DC0923069F018F491308C
:106DE000C1F503C09530A8F50CC01093261183E0BF
:106DF000809325112EC01093261184E080932511D5
:106E000028C0809126112AE0829F100D1124812F25
:106E100010932611943021F4992787FD90951ADD5F
:106E200080912611992787FD90950E94B61A882394
:106E300059F080912611992787FD909590935812CB
:106E4000809357120E948F548FEF809326110E94D7
:106E50003B48DF91CF911F910F910C94D846812F21
:106E60008051823008F0E3CEB2CE00E007CF173277
:106E700009F054CF42CF173209F061CF41CF98CEFD
:106E80002F923F924F925F926F927F928F929F923A
:106E9000AF92BF92CF92DF92EF92FF920F931F9328
:106EA000CF93DF93CDB7DEB763970FB6F894DEBF0D
:106EB0000FBECDBF882309F472C1198A1989110F39
:106EC000110F110F96EC792E2FE7A22EB12C6E0127
:106ED0008BE0C80ED11C6FB7F89471BA469A9989A5
:106EE000990F292F26702064892F880F8072907C3B
:106EF000892B99899695927031E035B928B98BB96B
:106F00009EB987E881BBEDE0EA95F1F7000071BA20
:106F1000469A80EE87B997E09AB98DB935B980E481
:106F200088B91BB88EB987E481BBF2E0FA95F1F716
:106F300000C046B199B18CB171BA479A242F2695F9
:106F4000237030E8439FA0011124242B392F307186
:106F5000232B392F369536953870232B96959076BE
:106F6000292B90E0880F991F84709927282B87EE92
:106F700087B987EF8AB982EE8DB96FBF912E00E095
:106F8000F8ED6F2E610EA0EC4A2E410E22242A94B9
:106F9000BFE73B2EEE24EA94FE2C88EA582E510ED1
:106FA00007C08250808326950F5F9394083001F1CB
:106FB000E92DF0E0E755F64F8081982F9E7F89F705
:106FC000922F91708170981771F3892F8A60808356
:106FD0008FE3891568F1692F772767FD7095892DF3
:106FE0002B8B4DDF2B8926950F5F9394083001F78B
:106FF00039893F5F398B185F303108F46CCF639665
:107000000FB6F894DEBF0FBECDBFDF91CF911F91B9
:107010000F91FF90EF90DF90CF90BF90AF909F9037
:107020008F907F906F905F904F903F902F9008953A
:10703000492F552747FD509580913411882351F1F0
:10704000452B09F4B0CF8AE0EAE1F7E0DE011196C2
:1070500001900D928A95E1F786E0F60111928A95EA
:10706000E9F7852D800F8093C81080930B0E8093D5
:10707000FB0C4AE050E0BE01665F7F4F992787FD19
:1070800090952B8B0E945075CE0101960E941A1785
:107090002B8989CF862C800E452BE9F45091020D67
:1070A000511139C08091C81040E050E8692F880D17
:1070B0002B8B9A8BCCD28091C810880D9A892B8902
:1070C000911148C040E4682F80915B122B8B0E9485
:1070D000D82C2B8968CF8091030D813009F498C09A
:1070E0008091040D813009F481C05091020D51113D
:1070F00012C08091030D833021F08091040D833004
:1071000089F6882D2B8B9A8B0E94141F0E94F124E4
:107110009A892B89C7CF442D400F911121C08091AE
:10712000010D882309F43FC0513009F4A8C0E8E7F5
:10713000FCE080E090E005C001968038910509F4FC
:1071400032CF51915413F8CFFC01E858F34F406807
:10715000408329CF60E070E80E94BF2C2B8923CFA9
:10716000A8E7BCE0FD0105C08CE0E83FF80709F4A2
:1071700061C081918F3FC1F3513009F466C080E056
:1071800090E005C001968038910509F40CCF5D911F
:107190005F3FC1F7FC01E858F34F408304CF38E06C
:1071A000398B132F8CCE513009F45CC0E8E7FCE03A
:1071B00080E090E004C001968038910541F0519143
:1071C0005413F9CFFC01E858F34F3FEF3083E8E761
:1071D000FCE081918F3F09F0E6CE3CE0E83FF30709
:1071E000C1F72B8B0E94C6552B89DDCEF0920A0E7B
:1071F000E092090E30920F0E20920E0E32E0309384
:10720000040D2B8B9A8B0E94F1249A892B896DCFC8
:10721000F092080EE092070E30920F0E20920E0EA2
:10722000F2E0F093030D2B8B9A8B0E94F1249A8944
:107230002B8956CF80915D1281119ECF3092FE0C2A
:107240002092FD0C513009F09ACF842F90E0FC0180
:10725000E858F34F4083F501E81BF90BE858F34F6A
:107260004083A1CE50E0FA01E858F34F8FEF8083BE
:10727000F501E41BF50BE858F34F8083A8CF50E0ED
:10728000FA01E858F34F808180688083F501E41BA0
:10729000F50BE858F34F80818068808384CEFC0131
:1072A000623009F43BC018F1633069F1643011F5C4
:1072B00011A210A2268D378D46895789AA27249FAF
:1072C000B12D359FC001529FB00D811D9A1F349F73
:1072D000B00D811D9A1F112482A393A34089518967
:1072E0006289738940835183628373830895613017
:1072F00009F443C011A210A213A212A2108211829B
:1073000012821382089511A210A28689978993A3ED
:1073100082A31082118212821382089526893789EE
:1073200044895589AA27429FB12D539FC001349F9C
:10733000B00D811D9A1F529FB00D811D9A1F1124FF
:1073400080A391A340955095AA27429FB12D539FAA
:10735000C001349FB00D811D9A1F529FB00D811D39
:107360009A1F112482A393A344855585668577854A
:107370004083518362837383089526893789468DBC
:10738000578DAA27429FB12D539FC001349FB00D46
:10739000811D9A1F529FB00D811D9A1F112480A339
:1073A00091A340955095AA27429FB12D539FC001AC
:1073B000349FB00D811D9A1F529FB00D811D9A1FE1
:1073C000112482A393A340855185628573854083F0
:1073D00051836283738308951F93CF93DF93EC01EE
:1073E000898D0E94E41F18A5012E04C096958795EB
:1073F000779567950A94D2F724E0660F771F881F68
:10740000991F2A95D1F7688779878A879B878B8D03
:107410000E94E41F012E04C0969587957795679585
:107420000A94D2F734E0660F771F881F991F3A95A8
:10743000D1F76C877D878E879F878D8D0E94E41F93
:1074400004C096958795779567951A95D2F744E08D
:10745000660F771F881F991F4A95D1F7688B798B24
:107460008A8B9B8B69A5CE01DF91CF911F9117CF9E
:10747000FC01268937892617370719F0778B668B29
:10748000ABCF08950F931F93FC01808D918D8617CC
:10749000970721F0718F608F61E001C060E0828DFD
:1074A000938D8417950719F0538F428F61E084897B
:1074B00095898217930719F0358B248B61E0848DB1
:1074C000958D8017910719F0158F048F02C06623E0
:1074D00021F0CF011F910F917FCF1F910F91089540
:1074E000FC0160A779CF0F931F93CF93DF938B019C
:1074F0004091131150911411AA27049FB12D159F8B
:10750000B001509FB00D611D7A1F149FB00D611D19
:107510007A1F112440955095640F751F9AE28902D5
:10752000E0011124CE018E5E914FA2DF4091111136
:1075300050911211AA27049FB12D159FB001509FA1
:10754000B00D611D7A1F149FB00D611D7A1F1124AB
:1075500040955095640F751FCE01825F904FDF916B
:10756000CF911F910F9184CFAF92BF92CF92DF92B4
:10757000EF92FF920F931F93CF93DF931F92CDB79C
:10758000DEB7F82E8B0149830E94D1186F2D81E060
:107590000E9436594981442329F08091020D8823A5
:1075A00009F447C08F2D9AE289026001112452E14B
:1075B000A52E5EE0B52EAC0CBD1CF5011482158223
:1075C0001682178264A175A1CB01A0E0B0E07727F5
:1075D00066272689378940E050E00E94CA75F50188
:1075E000378F268FEE24E394E1A6C5010E94294B34
:1075F000F501E7A28EE09FE0C80ED91EF6011482C5
:1076000015821682178264A175A1CB01A0E0B0E0BB
:10761000772766272689378940E050E00E94CA759F
:10762000F601378F268FE1A6C6010E94294BF6018D
:10763000E7A2B8018F2D0F90DF91CF911F910F918D
:10764000FF90EF90DF90CF90BF90AF904CCF2F92F4
:107650003F924F925F926F927F928F929F92AF92E2
:10766000BF92CF92DF92EF92FF920F931F93CF932F
:10767000DF93882E742E652E86958695869590E0EC
:10768000E82DE770F0E0E75CF84F2081FC01E65957
:10769000F54F662309F4B5C08081822B8083E82DE5
:1076A000F0E0EE0FFF1FE658F54F40835183312C79
:1076B000C090A409D090A509E090A609F090A70970
:1076C0008091C40B882309F404C18091C20B8823E4
:1076D00029F1282D30E0823009F4D9C5813009F430
:1076E000B2C580E090E082179307A1F0E82FE695FD
:1076F000E695E695F0E0E659F54F4081442351F0D8
:10770000FC01E770FF27E75CF84F5081542311F02C
:107710003324339401968038910529F790E0DCEB0F
:10772000AD2EDBE0BD2E1BE0212E99249394482C36
:10773000512C06E010E0E50189915E018F3F09F4CC
:107740004DC0C92FDD27C7FDD0952C9E90012D9EE1
:10775000300D11242659354FF901E85EFE4F908215
:10776000F901E75EFE4F9082F901E65EFE4F9082DE
:10777000F901EC5EFE4F70826182F901EA5EFE4F14
:107780008082F901E95EFE4FA201480F511D40833E
:10779000F901E05FFE4FC082D182E282F382432D85
:1077A000672D762D892FE0DE4091C30B04C0C92FD1
:1077B000DD27C7FDD095CE010196B8010E94E27089
:1077C0009C01982FF901E75CF84F8081842379F3BD
:1077D000D2ECAD16DBE0BD0609F0ADCFDF91CF9165
:1077E0001F910F91FF90EF90DF90CF90BF90AF90DF
:1077F0009F908F907F906F905F904F903F902F90D1
:10780000089520958081282320839090820B70908A
:10781000800B072D10E0A0908D0BA0918B0BB0E09A
:10782000E090980B2091960B30E0F090A30B6091C4
:10783000A10B70E0C090AE0B4091AC0B50E0B0904B
:10784000B90BC091B70B2C2E312C8091C20B82301A
:1078500009F4BBC180E090E0992009F40FC1A110A8
:1078600077C2B110E1C0D82EE82FE695E695E695EF
:10787000F0E0E659F54FA081AA2309F463C2FC01A8
:10788000E770FF27E75CF84FE081EA2309F45AC26A
:107890000817190709F456C2EE2021F028173907F6
:1078A00009F450C2FF2021F06817790709F44AC291
:1078B000CC2021F04817590709F444C2FC01EE0F0F
:1078C000FF1FE658F54F708061808D2C3324339470
:1078D000EFCE8091C30B80FF17C09091820B409137
:1078E0007A0B50917B0B60917C0B70917D0B9923EF
:1078F00009F4C7C14C155D056E057F0528F490910C
:10790000810B891609F40ACF4FEF5FEFBA019FEFA1
:1079100081FF17C020918D0B222309F4BBC1009178
:10792000850B1091860B2091870B3091880B0C15DD
:107930001D052E053F0528F420918C0B821609F4B5
:10794000D0C482FF17C02091980B222309F4C6C12E
:107950000091900B1091910B2091920B3091930B11
:107960000C151D052E053F0528F42091970B821656
:1079700009F4B5C483FF17C02091A30B222309F497
:107980009BC100919B0B10919C0B20919D0B309102
:107990009E0B0C151D052E053F0528F42091A20B0A
:1079A000821609F49AC484FF17C02091AE0B2223DB
:1079B00009F4B6C10091A60B1091A70B2091A80B5A
:1079C0003091A90B0C151D052E053F0528F42091BB
:1079D000AD0B821609F47FC485FF17C08091B90BE7
:1079E000882309F48DC14091B10B5091B20B609185
:1079F000B30B7091B40B4C155D056E057F0528F433
:107A00008091B80B881609F489C19F3F09F087CE91
:107A1000882D0E94011C982F87FDE0CE80CE019614
:107A20008038910509F40AC1D82EE82FE695E6952D
:107A3000E695F0E0E659F54FA081AA2381F3FC0119
:107A4000E770FF27E75CF84FE081EA2341F308176E
:107A5000190729F3EE2019F02817390701F3FF2041
:107A600019F068177907D9F2CC2019F0481759078F
:107A7000B1F22816390609F021CFD1CFB110CCC10F
:107A8000A1107BC0D82EE82FE695E695E695F0E0AC
:107A9000E659F54FA081AA23C9F0FC01E770FF2742
:107AA000E75CF84FE081EA2389F0EE2019F028170F
:107AB000390761F0FF2019F06817790739F0CC20F9
:107AC00009F4FCCE4817590709F0F8CE0196803822
:107AD0009105C1F68091980B882329F08091960B2F
:107AE000881509F497C38091A30B882329F080910E
:107AF000A10B881509F475C38091AE0B882329F07A
:107B00008091AC0B881509F453C38091B90B88237D
:107B100009F464CE8091B70B881160CE1092BB0B34
:107B20008091C50B81115ACE1092BA0B0E94D118C8
:107B300065E081E00E94365960E084EE9EE00E949C
:107B4000612060E080EE9FE0DF91CF911F910F9167
:107B5000FF90EF90DF90CF90BF90AF909F908F906D
:107B60007F906F905F904F903F902F900C9461208A
:107B700001968038910509F464C0D82EE82FE69567
:107B8000E695E695F0E0E659F54FC081CC2381F308
:107B9000FC01E770FF27E75CF84FE081EC2341F33D
:107BA000A817B90729F3EE2019F02817390701F3B0
:107BB000FF2019F068177907D9F2CC2009F47ECE9E
:107BC0004817590709F07ACED3CFFF2009F481C1B5
:107BD000EE2009F473C2EFE7F0E0A11032C2CF014A
:107BE000DE2EAE2FA695A695A695B0E0A659B54F68
:107BF000FC90FF20F9F0DF01A770BB27A75CB84F0E
:107C0000AC91AF21B9F0992019F00E171F0791F030
:107C10002E173F0779F06E177F0761F0CC2019F01F
:107C20004E175F0739F0BB2009F448CE2E163F06E9
:107C300009F044CE319798F6992019F0781409F498
:107C40009CC2AA2009F446CF80918B0B881142CFA9
:107C500010928F0B8091C50B81113CCF10928E0B2F
:107C60000E94D11861E081E00E94365960E08CE307
:107C70009EE00E94612060E088E39FE00E94612016
:107C800029CF4F3F9FEF59076907790709F43FCE86
:107C900090E03ECE0091850B1091860B2091870BD2
:107CA0003091880B041715072607370708F049CECF
:107CB000B901A80191E045CE00919B0B10919C0B5E
:107CC00020919D0B30919E0B04171507260737074F
:107CD00008F069CEB901A80193E065CE0091900B40
:107CE0001091910B2091920B3091930B0417150773
:107CF0002607370708F03ECEB901A80192E03ACE38
:107D00000091B10B1091B20B2091B30B3091B40BD9
:107D1000041715072607370708F077CE95E0FFCC44
:107D20000091A60B1091A70B2091A80B3091A90BE5
:107D3000041715072607370708F04ECEB901A8012A
:107D400094E04ACE01968038910509F08CCD76CF2B
:107D5000E11034C0D82EE82FE695E695E695F0E0E0
:107D6000E659F54F20812223F9F0FC01E770FF2747
:107D7000E75CF84F30813223B9F008171907A1F0FA
:107D8000A817B90789F0FF2019F06817790761F083
:107D9000CC2019F04817590739F0BB2009F48ECDD3
:107DA0002816390609F08ACD01968038910591F69A
:107DB00045CF01968038910509F440CFD82EE82FA1
:107DC000E695E695E695F0E0E659F54FE080EE2081
:107DD00081F3FC01E770FF27E75CF84FE081EE21BB
:107DE00041F38017910729F38A179B0711F3821734
:107DF0009307F9F2FF2019F086179707D1F2CC20EC
:107E000019F084179507A9F2BB2009F457CD821504
:107E1000930509F053CDCDCFC1102DC0D82EE82F3A
:107E2000E695E695E695F0E0E659F54F4081442366
:107E3000C1F0FC01E770FF27E75CF84F5081542345
:107E400081F0AA2019F0A817B90759F0EE2019F00F
:107E50002817390731F0F11038C02816390609F013
:107E60002DCD019680389105C9F6EBCE019680386C
:107E7000910509F4E6CED82EE82FE695E695E6952D
:107E8000F0E0E659F54F1081112381F3FC01E77012
:107E9000FF27E75CF84FE081E12341F3AA2019F0C6
:107EA000A817B90719F3EE2019F028173907F1F2CE
:107EB000FF2019F068177907C9F248175907B1F27E
:107EC0002816390609F0FACCD1CF6817790729F6B8
:107ED000C8CF6FE770E0992009F45DC0A1102CC0F5
:107EE000CB01D62EE62FE695E695E695F0E0E6592D
:107EF000F54FA081AA23E1F0FB01E770FF27E75CC3
:107F0000F84FE081EA23A1F00617170789F0EE2069
:107F100019F02617370761F0CC2019F046175707DC
:107F200039F0BB2009F4CACC2616370609F0C6CCB6
:107F300061507109A8F682CECB01D62EE62FE695C8
:107F4000E695E695F0E0E659F54FF080FF20F9F070
:107F5000FB01E770FF27E75CF84FE081EF21B9F004
:107F600006171707A1F0A617B70789F0EE2019F03A
:107F70002617370761F0CC2019F04617570739F05C
:107F8000BB2009F49BCC2616370609F097CC61502C
:107F9000710990F653CEB11029C0CB01D62EE62F31
:107FA000E695E695E695F0E0E659F54FC081CC23DD
:107FB000C9F0FB01E770FF27E75CF84FE081EC2395
:107FC00089F0AA2019F0A617B70761F0EE2019F082
:107FD0002617370739F0CC2009F470CC461757071D
:107FE00009F06CCC61507109C0F62BCECB01D62EB6
:107FF000E62FE695E695E695F0E0E659F54F108117
:108000001123D9F0FB01E770FF27E75CF84FE0810F
:10801000E12399F0AA2019F0A617B70771F0EE2016
:1080200019F02617370749F0CC2019F046175707E3
:1080300021F02616370609F041CC61507109B0F6DF
:1080400000CECF01DE2EEE2EE694E694E694F12CDF
:10805000CAE64C2ECAE05C2EE40CF51CE7016880F1
:10806000662049F1C7E0EC2EF12CEE22FF22D9E385
:108070004D2ED7E05D2EE40CF51CE701F880F620CC
:10808000D1F0992019F0E017F107A9F0EA17FB07E2
:1080900091F0E217F30779F0E617F70761F0CC20CB
:1080A00019F0E417F50739F0BB2009F407CCE21505
:1080B000F30509F003CC319720F6BECD2FE730E071
:1080C00091102CC0C901D22EE22FE695E695E695D7
:1080D000F0E0E659F54F10811123E1F0F901E77066
:1080E000FF27E75CF84FE081E123A1F0AA2019F017
:1080F000A217B30779F06217730761F0CC2019F06B
:108100004217530739F0BB2009F4D8CB22163306A7
:1081100009F0D4CB21503109A8F693CDC901D22E54
:10812000E22FE695E695E695F0E0E659F54FF0800A
:10813000FF20F9F0F901E770FF27E75CF84FE081D5
:10814000EF21B9F002171307A1F0AA2019F0A21726
:10815000B30779F06217730761F0CC2019F042176A
:10816000530739F0BB2009F4A9CB2216330609F0D6
:10817000A5CB2150310990F661CD1092840B8091EE
:10818000C50B81115ECD1092830B0E94D11860E067
:1081900081E00E94365960E082E19EE00E94612009
:1081A00060E08EE09FE00E946120A0908D0B49CDA1
:1081B0001092B00B8091C50B8111A7CC1092AF0B20
:1081C0000E94D11864E081E00E94365960E08AEB99
:1081D0009EE00E94612060E086EB9FE00E946120AB
:1081E00094CC1092A50B8091C50B811185CC109277
:1081F000A40B0E94D11863E081E00E94365960E030
:1082000080E99EE00E94612060E08CE89FE00E948F
:10821000612072CC10929A0B8091C50B811163CCB6
:108220001092990B0E94D11862E081E00E943659A9
:1082300060E086E69EE00E94612060E082E69FE0CA
:108240000E94612050CC80E090E007C0332433943A
:1082500001968038910509F461CA82179307C1F32A
:10826000E82FE695E695E695F0E0E659F54F408172
:10827000442371F3FC01E770FF27E75CF84F50815E
:10828000542331F3821793070CF4A8CADFCF80E0A0
:1082900090E007C03324339401968038910509F4A7
:1082A0003DCA82179307C1F3E82FE695E695E69558
:1082B000F0E0E659F54F4081442371F3FC01E7708B
:1082C000FF27E75CF84F5081542331F32817390713
:1082D0000CF484CADFCF94E022CA93E020CA92E073
:1082E0001ECA91E01CCA2F923F924F925F926F92EA
:1082F0007F928F929F92AF92BF92CF92DF92EF9236
:10830000FF920F931F93CF93DF93CDB7DEB72C97D8
:108310000FB6F894DEBF0FBECDBFE0900111F09014
:1083200002112090F9103090FA108091D8108093AB
:10833000340F8091D6108093380E8091E2108823FC
:1083400009F4E6C463E08EE09FE0CAD88091D710BC
:10835000882309F4DBC463E082E19EE0C1D8809108
:108360005E12882309F4CEC480E091E0A0E0B0E082
:1083700020910511309106112C013D01420E531E32
:10838000611C711C2091031130910411AC01BD01DD
:10839000420F531F611D711D2091FF10309100117C
:1083A0005C016D01A20EB31EC11CD11CA982BA8250
:1083B000CB82DC822091FD103091FE105C016D01BA
:1083C000A20EB31EC11CD11CAD82BE82CF82D88644
:1083D0002091FB103091FC105C016D01A20EB31EC8
:1083E000C11CD11CA986BA86CB86DC862091F710E9
:1083F0003091F8104C015D01820E931EA11CB11C3E
:1084000009811A812B813C810115110581E0280722
:10841000310524F00FEF1FEF20E030E0411551054A
:10842000E1E06E07710524F04FEF5FEF60E070E070
:1084300041145104F1E06F0671042CF044244A9475
:10844000542C612C712C9701B2018EE09FE01AD858
:10845000950184018114910441E0A406B10424F043
:108460000FEF1FEF20E030E049845A846B847C8456
:108470004114510481E0680671042CF044244A94AC
:10848000542C612C712C6D817E818F8198856115B2
:108490007105E1E08E07910524F06FEF7FEF80E03A
:1084A00090E09101A20182E19EE00E94423A809117
:1084B000D81080935E0F8091D6108093620E8091C9
:1084C000E210882309F41CC463E088E39FE008D825
:1084D0008091D710882309F411C463E08CE39EE0F7
:1084E0000E94703A80915E12882309F403C480E0F0
:1084F0009FEFAFEFBFEF20910511309106112C01D6
:108500003D01420E531E611C711C77FC03C4209177
:10851000031130910411AC01BD01420F531F611DC5
:10852000711D77FD41C42091FF10309100115C0155
:108530006D01A20EB31EC11CD11C96018501D7FC92
:108540002FC48090FD109090FE105C016D01A80C6E
:10855000B91CC11CD11CA982BA82CB82DC82D7FC97
:108560001AC48090FB109090FC105C016D01A80C67
:10857000B91CC11CD11CAD82BE82CF82D886D7FC6B
:1085800005C4E091F710F091F8104C015D018E0EDA
:108590009F1EA11CB11CB7FCF5C30115110581E09C
:1085A0002807310524F00FEF1FEF20E030E04115E0
:1085B0005105E1E06E07710524F04FEF5FEF60E0D9
:1085C00070E041145104F1E06F0671042CF0442472
:1085D0004A94542C612C712C9701B20188E39FE0DE
:1085E0000E94423A950184018114910441E0A4065D
:1085F000B10424F00FEF1FEF20E030E04D805E80EB
:108600006F8078844114510481E0680671042CF075
:1086100044244A94542C612C712C69817A818B8179
:108620009C8161157105E1E08E07910524F06FEFE3
:108630007FEF80E090E09101A2018CE39EE00E9438
:10864000423A8091D8108093880F8091D610809301
:108650008C0E8091E210882309F44AC363E082E61D
:108660009FE00E94703A8091D710882309F43EC39E
:1086700063E086E69EE00E94703A80915E12882355
:1086800009F430C380E092E0A0E0B0E02091051151
:10869000309106112C013D01420E531E611C711CCC
:1086A0002091031130910411AC01BD01420F531F01
:1086B000611D711D2091FF10309100115C016D0151
:1086C000A20EB31EC11CD11CA982BA82CB82DC824D
:1086D0002091FD103091FE105C016D01A20EB31EC1
:1086E000C11CD11CAD82BE82CF82D8862091FB10E6
:1086F0003091FC105C016D01A20EB31EC11CD11C97
:10870000A986BA86CB86DC862091F7103091F810C6
:108710004C015D01820E931EA11CB11C09811A81BE
:108720002B813C810115110581E02807310524F0DA
:108730000FEF1FEF20E030E041155105E1E06E073B
:10874000710524F04FEF5FEF60E070E041145104D9
:10875000F1E06F0671042CF044244A94542C612CEF
:10876000712C9701B20182E69FE00E94423A950186
:1087700084018114910441E0A406B10424F00FEFB8
:108780001FEF20E030E049845A846B847C844114DC
:10879000510481E0680671042CF044244A94542C5E
:1087A000612C712C6D817E818F8198856115710599
:1087B000E1E08E07910524F06FEF7FEF80E090E01D
:1087C0009101A20186E69EE00E94423A8091D81073
:1087D0008093B20F8091D6108093B60E8091E210F4
:1087E000882309F47DC263E08CE89FE00E94703A20
:1087F0008091D710882309F471C263E080E99EE07C
:108800000E94703A80915E12882309F463C280E06E
:108810009EEFAFEFBFEF20910511309106112C01B3
:108820003D01420E531E611C711C77FCA7C22091B2
:10883000031130910411AC01BD01420F531F611DA2
:10884000711D77FD97C22091FF10309100115C01DE
:108850006D01A20EB31EC11CD11C96018501D7FC6F
:1088600085C28090FD109090FE105C016D01A80CF7
:10887000B91CC11CD11CA982BA82CB82DC82D7FC74
:1088800070C28090FB109090FC105C016D01A80CF0
:10889000B91CC11CD11CAD82BE82CF82D886D7FC48
:1088A0005BC2E091F710F091F8104C015D018E0E63
:1088B0009F1EA11CB11CB7FC4BC20115110581E024
:1088C0002807310524F00FEF1FEF20E030E04115BD
:1088D0005105E1E06E07710524F04FEF5FEF60E0B6
:1088E00070E041145104F1E06F0671042CF044244F
:1088F0004A94542C612C712C9701B2018CE89FE0B2
:108900000E94423A950184018114910441E0A40639
:10891000B10424F00FEF1FEF20E030E04D805E80C7
:108920006F8078844114510481E0680671042CF052
:1089300044244A94542C612C712C69817A818B8156
:108940009C8161157105E1E08E07910524F06FEFC0
:108950007FEF80E090E09101A20180E99EE00E941B
:10896000423A8091D8108093DC0F8091D61080938A
:10897000E00E8091E210882309F4AAC163E086EB3F
:108980009FE00E94703A8091D710882309F49EC11D
:1089900063E08AEB9EE00E94703A80915E12882329
:1089A00009F490C180E093E0A0E0B0E020910511CF
:1089B000309106112C013D01420E531E611C711CA9
:1089C0002091031130910411AC01BD01420F531FDE
:1089D000611D711D2091FF10309100115C016D012E
:1089E000A20EB31EC11CD11CA982BA82CB82DC822A
:1089F0002091FD103091FE105C016D01A20EB31E9E
:108A0000C11CD11CAD82BE82CF82D8862091FB10C2
:108A10003091FC105C016D01A20EB31EC11CD11C73
:108A2000A986BA86CB86DC862091F7103091F810A3
:108A30004C015D01820E931EA11CB11C09811A819B
:108A40002B813C810115110581E02807310524F0B7
:108A50000FEF1FEF20E030E041155105E1E06E0718
:108A6000710524F04FEF5FEF60E070E041145104B6
:108A7000F1E06F0671042CF044244A94542C612CCC
:108A8000712C9701B20186EB9FE00E94423A95015A
:108A900084018114910441E0A406B10424F00FEF95
:108AA0001FEF20E030E049845A846B847C844114B9
:108AB000510481E0680671042CF044244A94542C3B
:108AC000612C712C6D817E818F8198856115710576
:108AD000E1E08E07910524F06FEF7FEF80E090E0FA
:108AE0009101A2018AEB9EE00E94423A8091D81047
:108AF000809306108091D61080930A0F8091E21027
:108B0000882309F4DDC063E080EE9FE00E94703AA4
:108B10008091D710882309F4D1C063E084EE9EE0F1
:108B20000E94703A80915E12882309F4C3C080E0ED
:108B30009DEFAFEFBFEF20910511309106112C0191
:108B40003D01420E531E611C711C77FCFDC020913B
:108B5000031130910411AC01BD01420F531F611D7F
:108B6000711D77FDEDC02091FF10309100115C0167
:108B70006D01A20EB31EC11CD11C96018501D7FC4C
:108B8000DBC08090FD109090FE105C016D01A80C80
:108B9000B91CC11CD11CA982BA82CB82DC82D7FC51
:108BA000C6C08090FB109090FC105C016D01A80C79
:108BB000B91CC11CD11CAD82BE82CF82D886D7FC25
:108BC000B1C0E091F710F091F8104C015D018E0EEC
:108BD0009F1EA11CB11CB7FCA1C00115110581E0AD
:108BE0002807310524F00FEF1FEF20E030E041159A
:108BF0005105E1E06E07710524F04FEF5FEF60E093
:108C000070E041145104F1E06F0671042CF044242B
:108C10004A94542C612C712C9701B20180EE9FE094
:108C20000E94423A950184018114910441E0A40616
:108C3000B10424F00FEF1FEF20E030E04D805E80A4
:108C40006F8078844114510481E0680671042CF02F
:108C500044244A94542C612C712C69817A818B8133
:108C60009C8161157105E1E08E07910524F06FEF9D
:108C70007FEF80E090E09101A20184EE9EE00E94EF
:108C8000423A2C960FB6F894DEBF0FBECDBFDF91EF
:108C9000CF911F910F91FF90EF90DF90CF90BF90F9
:108CA000AF909F908F907F906F905F904F903F908C
:108CB0002F90089580E090E0DC013DCF61E02ECF61
:108CC00061E022CF80E090E0DC0170CE61E061CE17
:108CD00061E055CE80E090E0DC019DCD61E08ECD7D
:108CE00061E082CD80E090E0DC01D0CC61E0C1CCDD
:108CF00061E0B5CC80E090E0DC01FDCB61E0EECB43
:108D000061E0E3CB80E090E0DC0132CB61E024CB9A
:108D100061E019CB412C512C3201F9CB812C912CE3
:108D200054015BCF1D821E821F8218864ACF198292
:108D30001A821B821C8235CF00E010E0980121CFFF
:108D400040E050E0BA010FCF412C512C3201FFCE50
:108D5000812C912C5401B1CD1D821E821F82188658
:108D6000A0CD19821A821B821C828BCD00E010E0FC
:108D7000980177CD40E050E0BA0165CD412C512CEF
:108D8000320155CD812C912C540107CC1D821E82BD
:108D90001F821886F6CB19821A821B821C82E1CBB5
:108DA00000E010E09801CDCB40E050E0BA01BBCB31
:108DB000CF9380916A0A90916B0A892B90916C0AEB
:108DC000892B90916D0A892B90916E0A892B909135
:108DD0006F0A892B9091700A892B9091710A892BC7
:108DE0009091720A892B9091730A892B9091740A41
:108DF000892B9091750A892B9091760A892B9091F5
:108E0000770A892B9091780A892B9091790A982B6F
:108E100021E009F420E08091980B90918D0B892B33
:108E20009091A30B892B9091AE0B892B9091820B83
:108E3000892B9091B90B892B59F48FEF9FEFDC01AF
:108E40008093C1109093C210A093C310B093C4102C
:108E5000222329F080918814882309F449C02093A3
:108E600088140E94B91825D48091DA10811151C05C
:108E70000E94CE17C0915C128091C30BC81721F0DD
:108E80000E943017C093C30BC091DB108091C20BBE
:108E9000C81731F00E943017C33040F5C093C20BA1
:108EA0000E94FC2120DA0E940F1580915F1281112F
:108EB00036C08FEF9FEF9093891080938810909326
:108EC0008B1080938A1090938D1080938C109093C8
:108ED0008F1080938E1090939110809390109093A8
:108EE000931080939210CF910C94F124C0E0D6CFD0
:108EF0008091A4099091A509A091A609B091A70914
:108F00008093C1109093C210A093C310B093C4106B
:108F1000A6CF61E08FE191E10E949217ABCF8CE088
:108F20000E944C1690938910809388108DE00E94C7
:108F30004C1690938B1080938A108EE00E944C16F2
:108F400090938D1080938C108FE00E944C1690931C
:108F50008F1080938E1080E10E944C169093911098
:108F60008093901081E10E944C169093931080930F
:108F70009210CF910C94F124E82FF0E0E755F64FD2
:108F800090819170803209F456C078F0843209F4EF
:108F90004CC0A0F1863209F445C008F058C0909347
:108FA000D01081E08093271103CF8C31C8F08C3131
:108FB00009F444C08091C60981709091D4109073D7
:108FC000892B9091C70990FD47C090E0892B909123
:108FD000C80990FF45C092E0892B8093D410E1CF5F
:108FE0008A31A8F08091C40981709091C30990FDE5
:108FF00035C090E0892B8093D510D3CF8232C1F059
:1090000018F09093CC10CDCF9093CA10CACF88316E
:1090100031F0893109F008959093CE10C2CF90932A
:10902000CB10BFCF9093D110BCCF9093CD10B9CFC0
:109030009093CF10B6CF9093C910B3CF9091C5093C
:109040008091D21090FB80F98093D210AACF873202
:1090500011F79093DA10A5CF98E0B8CF92E0CACF7D
:1090600090E0BACFCF93C8E18C2F86DFCF5FC832B4
:10907000D9F7CF9108952F923F924F925F926F92BE
:109080007F928F929F92AF92BF92CF92DF92EF9298
:10909000FF921F93CF93DF93CDB7DEB762970FB6E2
:1090A000F894DEBF0FBECDBF80915912882381F1A5
:1090B00080915712909158120E94B61A882371F12C
:1090C00080915912882381F10E94741810922711FF
:1090D00081E090915912911101C080E08093251197
:1090E00062960FB6F894DEBF0FBECDBFDF91CF9171
:1090F0001F91FF90EF90DF90CF90BF90AF909F9027
:109100008F907F906F905F904F903F902F90089539
:109110008BED90E00E94B61A8111D2CF0E94FE1909
:10912000809159128111D0CF9DDF80910E019091D5
:109130000F012091120130911301A0901001B09005
:1091400011014501809490946C01C21AD30ADA820D
:10915000C9822501612C712CC0901401D090150199
:10916000E0901601F0901701A901480F591F5C8388
:109170004B83CA01A0E0B0E08D839E83AF83B887A4
:10918000209118013091190140911A0150911B0151
:1091900029873A874B875C879091271110E0CF860B
:1091A000D88AE98AFA8A0FC022242A94322CED85C3
:1091B000FE85EE0FFF1FED51FF4E3182208291E0C0
:1091C0001F5F1E31E9F1C12ED12CDE86CD86F6015E
:1091D000E057F94F80818F3F99F3E82FEE0FFF0B97
:1091E000EF50F44F208031800E94821E8823F9F2D4
:1091F00082149304C8F22A143B04B0F0C101A0E029
:10920000B0E0E980FA802E143F0488F49C01AD019F
:1092100024193509460957096F85788989899A89FA
:109220000E94C7701C01C3CF212C312CC0CFCB8032
:10923000DC80C214D30438F0212C20E8322EB7CFC2
:109240009093271141CF9C01AD01CD80DE80EF804E
:10925000F8842C193D094E095F0969857A858B854B
:109260009C850E94C77090581C01A1CFCF92DF92BD
:10927000EF92FF92CF93DF93EC01CC80DD80EE8004
:10928000FF808F2D9927AA27BB27892B8A2B8B2B11
:1092900009F042C089A5823009F433C070F58130ED
:1092A00009F445C040E050E02AA13BA1AA27429F13
:1092B000B12D539FC001349FB00D811D9A1F529F45
:1092C000B00D811D9A1F112428A139A1820F931F6F
:1092D0009DA38CA3488159816A817B814C0D5D1DC2
:1092E0006E1D7F1D4C835D836E837F83DF91CF91E5
:1092F000FF90EF90DF90CF9008958330A9F08430F5
:1093000089F68EA1811123C0BB27AF2D9E2D8D2DF7
:10931000AC0140955095C8CFCE010E941020CC8062
:10932000DD80EE80FF80B6CF4C895D89BDCF8EA1F8
:10933000811105C077276F2D5E2D4D2DB5CF40EAE9
:1093400053E0C701B6010E949519AC01ADCF40EAC8
:1093500051E0C701B6010E949519DACFFC013FB771
:10936000F89421819081291728F48281820F891B2A
:109370003FBF0895822F891B3FBF08956F928F9240
:109380009F92AF92BF92CF92DF92EF92FF920F9394
:109390001F93CF93DF93E091BF19F091C0193097DD
:1093A00019F08FE999E1099587E89AE1D7DF082F4D
:1093B00010E00115110509F478C0C0E0D0E09091EB
:1093C000871A2091891AEE24E394F12CE3E09E2E73
:1093D000F4E08F2EA2E0AA2EBB24B394892F622F33
:1093E00090E070E00E94E270E0918A1AF0918B1A8E
:1093F000E80FF91FF081F83F08F065C0F7FF71C072
:109400008091C419843031F0F093C119F092C619DB
:10941000E092C5198F2F807F803B79F198F48039D5
:1094200061F1803A51F1803841F1F03F09F4B1C067
:10943000F73F09F4C3C01092C4191092C6191092D4
:10944000C5191DC0803D09F4A1C008F49CC0803E30
:10945000A1F0803F51F7EF2FE15FEF3030F7AE2FF3
:10946000B0E0A65DB84F8C91813009F49BC0E8F262
:10947000823009F48BC08330F1F69092C4193FB763
:10948000F8949091871A892F90E001962091891A7B
:10949000622F70E00E94E270982F8093871A3FBF7E
:1094A0002196C017D10708F499CFDF91CF911F9172
:1094B0000F91FF90EF90DF90CF90BF90AF909F9073
:1094C0008F906F900895D090C419B092C41920E085
:1094D00040E06F2F81E090E00E947B12D092C4198F
:1094E000CECF6090C419662051F24091C5195091B9
:1094F000C6199A01ABEABAEA0E94BE756C01D6940D
:10950000C794C601880F991F8C0D9D1D6A01C81A4A
:10951000D90AD601A156B64E9296FC93CA0101967D
:109520009093C6198093C51921E0C216D104B9F0F1
:1095300022E0C216D10409F0A2CF2091C3194091B4
:10954000C2196091C1190E947B128091C4198430A4
:1095500009F495CFF092C619E092C51990CF22E098
:1095600062128DCF20E04091C2196091C1190E9412
:109570007B128091C419843009F481CFD092C6192E
:10958000C092C5197CCF803C09F04FCFA092C4197E
:1095900076CF8092C419F093C119F092C619E09267
:1095A000C5196DCF8093C41920E040E06F2F81E092
:1095B00090E00E947B121092C41961CF4091C519AE
:1095C0005091C6199A01ABEABAEA0E94BE75969507
:1095D00087959C01220F331F280F391FDA01A21B28
:1095E000B30BA156B64E9296FC93CA010196909386
:1095F000C6198093C5192091C3194091C219609171
:10960000C1190E947B121092C41939CFCF93DF93F6
:10961000E6ECFBE08081C8ECDBE0688190E070E084
:109620000E94E270A091C90BB091CA0BA80FB91F9C
:109630002C913FB7F894808190E00196688170E0AA
:109640000E94E27080833FBF822FDF91CF910C9404
:10965000012DFC0126893789468D578DAA27429F07
:10966000B12D539FC001349FB00D811D9A1F529F91
:10967000B00D811D9A1F112480A391A34095509590
:10968000AA27429FB12D539FC001349FB00D811D69
:109690009A1F529FB00D811D9A1F112482A393A37C
:1096A00040855185628573854083518362837383CE
:1096B00008958091770C8E7F9091C91091118160EF
:1096C0008093770C0E94D52A8091770C877F9091A8
:1096D000CC10911188608093770C0E94D52A8091DC
:1096E000770C8D7F9091CA10911182608093770CD6
:1096F0000E94D52A8091770C8F7E9091CD10911188
:1097000080618093770C0E94D52A8091770C8B7FA3
:109710009091CF10911184608093770C0E94D52A8C
:109720008091770C8F7D9091D01091118062809301
:10973000770C0E94D52A8091770C8F7B9091D11065
:10974000911180648093770C0C94D52A6F927F924C
:109750009F92AF92BF92CF92DF92EF92FF920F93C0
:109760001F93CF93DF931F92CDB7DEB717E3612E20
:109770001CE0712E60E008E010E086ECC82EDD24CD
:10978000D39490EFB92E27E8E22EF30181919191C5
:109790003F01B8EFFB2EF62A262F26952695269513
:1097A000A80102C0440F551F2A95E2F7942E909409
:1097B0009F20AFB6F89469830E94332BC1BA469AB2
:1097C0003F2D330F367031649F2D96959270906ABD
:1097D000D5B838B9BBB89EB9E1BA55E05A95F1F79A
:1097E0000000C1BA469A792D770F492D4695592D1B
:1097F000551F5527551F872F8670582B5064292DCC
:109800002071872F880F8072822B707C872B42708B
:10981000406AD5B858B98BB94EB9E1BA8AE08A9591
:10982000F1F700C0C1BA469AD5B838B9BBB89EB9ED
:10983000E1BAEAE0EA95F1F700C0AFBE69816F5F77
:10984000603209F0A2CF0F90DF91CF911F910F915D
:10985000FF90EF90DF90CF90BF90AF909F907F9060
:109860006F900C94D52A60918C14663028F46F5C4C
:1098700081E60E94F6160BC06C3028F4655D82E626
:109880000E94F61604C06B5D86E60E94F6160E94E2
:10989000BD2E5CCFCF92DF92EF92FF92CF93C9E1C2
:1098A000E2DFC150E9F710928B1410928A146AE03B
:1098B00081E10E94C3290E94892DC0E8C12CD12CCE
:1098C00076010E94A72A0E947B2A0E9446300E94AD
:1098D0004F2A0E9487300E94222A0E94C83080E1CD
:1098E0000E94F3290E94222A0E9406318AE00E94E7
:1098F000F3290E94892DC80ED91EE11CF11CB3DF8B
:1099000080918914853050F4C150D9F6B601C70151
:10991000CF91FF90EF90DF90CF900895CC24CA9420
:10992000DC2C7601B601C701CF91FF90EF90DF905C
:10993000CF900895CF92DF92EF92FF92CF93C9E13B
:1099400092DFC150E9F710928B1410928A146AE0EA
:1099500081E10E94C3290E94892D0E94A72A0E94AA
:109960007B2A0E9446300E944F2A0E9487300E9424
:10997000222A0E94C83080E10E94F3290E94222AF4
:109980000E9406318AE00E94F3290E94892D6C0111
:10999000E12CF12C68DF80918914853008F002C138
:1099A0000E94A72A0E947B2A0E9446300E944F2ACA
:1099B0000E9487300E94222A0E94C83080E10E94C3
:1099C000F3290E94222A0E9406318AE00E94F3298C
:1099D0000E94892DC80ED91EE11CF11C44DF809124
:1099E0008914853008F0DEC00E94A72A0E947B2AD5
:1099F0000E9446300E944F2A0E9487300E94222AED
:109A00000E94C83080E10E94F3290E94222A0E940D
:109A100006318AE00E94F3290E94892DC80ED91EC2
:109A2000E11CF11C20DF80918914853008F0BAC058
:109A30000E94A72A0E947B2A0E9446300E944F2A39
:109A40000E9487300E94222A0E94C83080E10E9432
:109A5000F3290E94222A0E9406318AE00E94F329FB
:109A60000E94892DC80ED91EE11CF11CFCDE8091DC
:109A70008914853008F096C00E94A72A0E947B2A8C
:109A80000E9446300E944F2A0E9487300E94222A5C
:109A90000E94C83080E10E94F3290E94222A0E947D
:109AA00006318AE00E94F3290E94892DC80ED91E32
:109AB000E11CF11CD8DE80918914853008F072C059
:109AC0000E94A72A0E947B2A0E9446300E944F2AA9
:109AD0000E9487300E94222A0E94C83080E10E94A2
:109AE000F3290E94222A0E9406318AE00E94F3296B
:109AF0000E94892DC80ED91EE11CF11CB4DE809194
:109B00008914853008F04EC00E94A72A0E947B2A43
:109B10000E9446300E944F2A0E9487300E94222ACB
:109B20000E94C83080E10E94F3290E94222A0E94EC
:109B300006318AE00E94F3290E94892DC80ED91EA1
:109B4000E11CF11C90DE80918914853058F50E944B
:109B5000A72A0E947B2A0E9446300E944F2A0E9418
:109B600087300E94222A0E94C83080E10E94F32997
:109B70000E94222A0E9406318AE00E94F3290E9454
:109B8000892DC80ED91EE11CF11C6DDE809189144F
:109B9000853040F4B601C701CF91FF90EF90DF9080
:109BA000CF900895CC24CA94DC2C7601B601C7016D
:109BB000CF91FF90EF90DF90CF900895CF93DF93F8
:109BC00000D000D01F92CDB7DEB70E94392CC12C37
:109BD000D12CA6ECAA2E88248394B0E4BB2E10EEE0
:109BE000912E07EF302E82EE282E02E110E0FFB614
:109BF0000E94111F882309F43FC0A1BA469A85B874
:109C0000B8B81BB81EB887E881BB9DE09A95F1F7FC
:109C10000000A1BA469A97B8E7E0EAB99DB885B8BE
:109C2000B8B81BB8BEB8F7E4F1BB82E08A95F1F78B
:109C300000C046B199B12CB1A1BA479AC42EC694BE
:109C4000E3E0CE22F0E84F9FA0011124C42A892F1F
:109C50008071C82A392F369536953870C32A969563
:109C60009076C92A30E0220F331F24703327C22A8E
:109C700087EE87B93AB82DB88F2D0E94091FC1FE13
:109C800008C08D2D90E00196B8010E94E270D82E98
:109C900009C0C2FE07C08D2D90E04196B8010E9418
:109CA000E270D82ED0928C149BE09D1518F48FEFA3
:109CB0009FEF02C080E090E060E00E942F2C8D2D8D
:109CC00066E00E94D670E92EF12C412C512CE41450
:109CD000F50419F46FEF7FEF02C060E070E0842DAF
:109CE0008E5E0E94D22B842D845F0E94102C842DC6
:109CF0000E94102C842D8A5F0E94102CEFEF4E1AC8
:109D00005E0AF6E04F16510411F785E08D1518F044
:109D10008FEF9FEF02C080E090E060E00E94252C72
:109D200095E09D1510F08FEF01C080E00E94032B9D
:109D30002D2D2650263018F48FEF9FEF02C080E0C3
:109D400090E060E029830E941B2C2981263010F4CA
:109D50008FEF01C080E00E94FB2AEBE08D2DED1516
:109D600048F00E94052CE6DD2B013C018D2D0E9460
:109D7000FA2B08C00E94EF2BDDDD2B013C018D2D5D
:109D80000E94E42B87DDAB01BC0192E1892F49835E
:109D90005A836B837C839D830E94DB2B9D819F5F15
:109DA00049815A816B817C81983181F74419550929
:109DB00066097709BB2777FDBA95A72F962F852FC0
:109DC00084369105A105B10524F083E690E0A0E07A
:109DD000B0E02C013D018D39FFEF9F07AF07BF07B2
:109DE00034F45DE9452E55245A94652C752CC20136
:109DF00057FE03C0919581959109BC01882777FD95
:109E00008095982F0E940A17C301B201662797FD1B
:109E1000639577278827992789E00E94CF1642E328
:109E2000F42E8FE39CE90197F1F700C000000E9437
:109E3000BD2E8CDCFA94A9F7DACECF92DF92EF92A6
:109E4000FF92CF93DF93D82FC9E10DDDC150E9F721
:109E500010928B1410928A146AE081E10E94C32947
:109E60000E94892DC12CD12C760124C00E94A72AE2
:109E70000E947B2A0E9446300E944F2A0E9487300F
:109E80000E94222A0E94C83080E10E94F3290E9489
:109E9000222A0E9406318AE00E94F329D1500E94B2
:109EA000892DC80ED91EE11CF11CDDDC80918914BE
:109EB000853058F4D111DACFB601C701DF91CF91C7
:109EC000FF90EF90DF90CF900895CC24CA94DC2CC3
:109ED0007601F2CF2F923F924F925F926F927F92D4
:109EE0008F929F92AF92BF92CF92DF92EF92FF92AA
:109EF0000F931F93CF93DF93CDB7DEB729970FB69C
:109F0000F894DEBF0FBECDBF782E662E4A83109226
:109F1000891470E080E090E00E9422729B01AC0105
:109F200060E070E080E090E40E94E57324EA30EDA8
:109F300042E851E40E9482739B01AC0160E074E24C
:109F400084EF99E40E945D716B837C838D839E8393
:109F5000262D235081E090E0022E01C0880F0A9444
:109F6000EAF789833EE0532E00E010E88FEF9FEF81
:109F700099878887E22FFF27E1950CF4F0954F0130
:109F8000AA2497FCA094BA2C672D8A810E945314AE
:109F9000288539858217930760F5B901872D0E94BE
:109FA000D22B89814ADF6B017C016F3F3FEF730742
:109FB0008307930709F44FC0C501B4010E942472BE
:109FC0009B01AC0160E070E080E090E40E94E573EA
:109FD0001B01482E9F83C701B6010E9422729B017C
:109FE000AC01FF80622D732D842D9F2D0E94827302
:109FF00004C06FEF7FEF8FE79FE7BB81AC81ED81FE
:10A00000FE802B2F3A2F4E2F5F2D0E940E731816B5
:10A010003CF488859985800F911F9987888706C0B1
:10A02000E885F985E01BF10BF987E8871695079518
:10A030005A9409F0A9CF22E1629EF0011124E70DA4
:10A04000F11DEE0FFF1FEB5CFE4E88859985918315
:10A05000808380E001C08FEF29960FB6F894DEBFB1
:10A060000FBECDBFDF91CF911F910F91FF90EF9069
:10A07000DF90CF90BF90AF909F908F907F906F9028
:10A080005F904F903F902F9008950F931F93CF9321
:10A09000DF93D82F062F80938C14862F0E94102CCC
:10A0A000DC3008F057C013E04CE0612F8D2F12DF39
:10A0B000811103C01F5F1730B9F7ED2FF0E0DF010A
:10A0C000AA0FBB1FAF55BE4E8D919C919C01220FD4
:10A0D000331FDF01AA0FBB1FAB53BE4E4D915C91E6
:10A0E000241B350BDF01AA0FBB1FA358BE4E2D93B7
:10A0F0003C93A901440F551F481B590BDF01AA0FC0
:10A10000BB1FA75ABE4E4D935C93440F551FDF01F2
:10A11000AA0FBB1FAB5CBE4E421B530B4D935C930F
:10A12000DF01AA0FBB1FAF5CBD4ECF01880F991F87
:10A13000835F9D4EEC0128813981220F331FEE0F82
:10A14000FF1FE751FE4E80819181281B390B2D9313
:10A150003C9323C014E044E2612F8D2FBBDE8823A3
:10A1600041F0ED2FF0E0EE0FFF1FEB53FE4E44E009
:10A1700004C01F5F183079F7F4CFDF019497208176
:10A180003181220F331F84A195A1281B390B119611
:10A190003C932E934150FD0181F7802F0E94DB2BD1
:10A1A000DF91CF911F910F91D1CA882339F086ECAE
:10A1B0009BE0D4D8811101C0089528CADFD8F7CF19
:10A1C000CF93DF93FC01D62FCFB7F894218130E0F5
:10A1D000C90101964281642F70E00E94E2704081C3
:10A1E00050E08417950791F0A381B481A20FB31FAB
:10A1F000DC93818190E00196628170E00E94E270C0
:10A200008183CFBF81E0DF91CF910895CFBF80E000
:10A21000DF91CF910895CF93C82F6C2F86EC9BE0F0
:10A22000CFDF81110CC086EC9BE098D88823A9F37E
:10A23000EDD96C2F86EC9BE0C3DF8823A1F3CF918F
:10A240000895EF92FF920F93CF93DF931F92CDB7B4
:10A25000DEB77B016115710539F40F90DF91CF9165
:10A260000F91FF90EF900895842F2983D4DF2981E7
:10A2700082E0E816F10488F3822FCDDFE2E0EE16EB
:10A28000F10459F3802F0F90DF91CF910F91FF9040
:10A29000EF90C1CF842F20915A1227FD09C06F7013
:10A2A00070E0332727FD30956217730709F0089592
:10A2B00040E050E060E00C94273B842FE0915A127C
:10A2C000E7FD09C06F7070E0FF27E7FDF0956E179E
:10A2D0007F0709F00895422F50E0542F4427550F6F
:10A2E00041505E4F61E0211101C060E00C94273BBA
:10A2F0002F923F924F925F926F927F928F929F9296
:10A30000AF92BF92CF92DF92EF92FF920F931F9383
:10A31000CF93DF93682EE82FE695E695E695F0E07B
:10A32000E659F54FA82FA770B0E0A75CB84F808121
:10A330009C91892B8083A62CB12CF501EE0FFF1F79
:10A34000E658F54F80E090E891838083C090A4099F
:10A35000D090A509E090A609F090A7098091C40BC0
:10A36000882309F49DC08091C20B312C882319F1F8
:10A37000823009F4ABC1813009F4CCC180E090E0B7
:10A38000A816B906A1F0E82FE695E695E695F0E067
:10A39000E659F54F2081222351F0FC01E770FF2799
:10A3A000E75CF84F3081322311F033243394019667
:10A3B0008038910529F790E02CEB822E2BE0922E2D
:10A3C0003BE0232E77247394412C40E8542E06E082
:10A3D00010E0F40181914F018F3F09F44EC0C92F65
:10A3E000DD27C7FDD0952C9E90012D9E300D1124A8
:10A3F0002659354FF901E85EFE4F7082F901E75E9C
:10A40000FE4F7082F901E65EFE4F7082F901EC5E4C
:10A41000FE4F51824082F901EA5EFE4F6082F901EF
:10A42000E95EFE4FA501480F511D4083F901E05F31
:10A43000FE4FC082D182E282F382432D60E070E859
:10A44000892F0E94B43A4091C30B04C0C92FDD2765
:10A45000C7FDD095CE010196B8010E94E2709C0123
:10A46000982FF901E75CF84F8081842379F3F2ECAF
:10A470008F16FBE09F0609F0ACCFDF91CF911F91C3
:10A480000F91FF90EF90DF90CF90BF90AF909F9093
:10A490008F907F906F905F904F903F902F90089596
:10A4A0008091C30B80FD8BC04FEF5FEFBA019FEF30
:10A4B00081FF17C020918D0B222309F4A2C00091C7
:10A4C000850B1091860B2091870B3091880B0C1512
:10A4D0001D052E053F0528F420918C0B621609F40A
:10A4E000F2C082FF17C02091980B222309F49BC071
:10A4F0000091900B1091910B2091920B3091930B46
:10A500000C151D052E053F0528F42091970B6216AA
:10A5100009F4D6C083FF17C02091A30B222309F4AE
:10A5200094C000919B0B10919C0B20919D0B30913E
:10A530009E0B0C151D052E053F0528F42091A20B3E
:10A54000621609F4BAC084FF17C02091AE0B222313
:10A5500009F49EC00091A60B1091A70B2091A80BA7
:10A560003091A90B0C151D052E053F0528F42091EF
:10A57000AD0B621609F49EC085FF17C08091B90B20
:10A58000882309F474C04091B10B5091B20B6091D3
:10A59000B30B7091B40B4C155D056E057F0528F467
:10A5A0008091B80B681609F470C09F3F31F4862D76
:10A5B0000E94011C982F87FD60CF312CFDCE909119
:10A5C000820B40917A0B50917B0B60917C0B7091C8
:10A5D0007D0B992369F04C155D056E057F0508F02C
:10A5E00063CF9091810B69125FCF90E0312CE4CE64
:10A5F0004F3F9FEF59076907790709F458CF90E05B
:10A6000057CF0091850B1091860B2091870B3091CD
:10A61000880B041715072607370708F062CFB90122
:10A62000A80191E05ECF0091900B1091910B2091C9
:10A63000920B3091930B041715072607370708F084
:10A6400069CFB901A80192E065CF00919B0B1091F1
:10A650009C0B20919D0B30919E0B0417150726072C
:10A66000370708F070CFB901A80193E06CCF0091D3
:10A67000B10B1091B20B2091B30B3091B40B0417B6
:10A6800015072607370708F090CF95E0312C94CEB8
:10A690000091A60B1091A70B2091A80B3091A90B4C
:10A6A000041715072607370708F066CFB901A80178
:10A6B00094E062CF94E0312C7FCE93E0312C7CCEBD
:10A6C00092E0312C79CE91E0312C76CE80E090E092
:10A6D00007C03324339401968038910509F46BCE7A
:10A6E000A816B906C1F3E82FE695E695E695F0E0E1
:10A6F000E659F54F2081222371F3FC01E770FF2713
:10A70000E75CF84F3081322331F3A816B9060CF418
:10A71000B4CEDFCF80E090E007C0332433940196BD
:10A720008038910509F447CEA816B906C1F3E82F81
:10A73000E695E695E695F0E0E659F54F208122236F
:10A7400071F3FC01E770FF27E75CF84F308132239B
:10A7500031F38A159B050CF490CEDFCF1092C50B18
:10A760008091C30B80FF04C09091830B911184C032
:10A7700081FF04C090918E0B911166C082FF04C0CE
:10A780009091990B911148C083FF04C09091A40B44
:10A7900091112AC084FF04C09091AF0B91110CC09D
:10A7A00085FF09C08091BA0B882329F08091BB0BEB
:10A7B000882309F479C008959091B00B9111F0CFDE
:10A7C0000E94D11864E081E051D560E08AEB9EE000
:10A7D0000E94612060E086EB9FE00E946120109261
:10A7E000AF0B8091C30BDCCF9091A50B9111D2CF11
:10A7F0000E94D11863E081E039D560E080E99EE0F5
:10A800000E94612060E08CE89FE00E94612010922D
:10A81000A40B8091C30BBECF90919A0B9111B4CF32
:10A820000E94D11862E081E021D560E086E69EE0DA
:10A830000E94612060E082E69FE00E946120109209
:10A84000990B8091C30BA0CF90918F0B911196CF54
:10A850000E94D11861E081E009D560E08CE39EE0C0
:10A860000E94612060E088E39FE00E9461201092D6
:10A870008E0B8091C30B82CF9091840B911178CF76
:10A880000E94D11860E081E0F1D460E082E19EE0B6
:10A890000E94612060E08EE09FE00E9461201092A3
:10A8A000830B8091C30B64CF0E94D11865E081E0D7
:10A8B000DDD460E084EE9EE00E94612060E080EEE6
:10A8C0009FE00E9461201092BA0B0895603E7105CE
:10A8D0008105910508F00895DC01CB019F5FAF4F22
:10A8E000BF4F6627782F892F9A2F0C9400F88091FC
:10A8F0009C1790919D178C5995418130924070F42E
:10A900004CE955E16CED70E080E090E0DFDF4CE970
:10A9100056E16DED70E080E090E0D8CF0895FF92B1
:10A920000F931F93CF93DF93FFB60E94FB198823E9
:10A9300009F442C00E94D719C5E3D1E111C0FE015C
:10A94000E00FF11F808191810E94F1190E5F1F4F6E
:10A9500004321105A1F7A49682E1C535D80719F094
:10A9600000E010E0ECCF80915712909158120E94B5
:10A97000F11980915512909156120E94F11980910F
:10A9800059120E94CC1980915A120E94C1198091CB
:10A990005C120E94CC1980915B120E94C1198091B7
:10A9A0005D120E94CC1980915E120E94C1198091A3
:10A9B0005F120E94C1199BDF8F2DDF91CF911F91F4
:10A9C0000F91FF900C94BF191F93CF93DF9300D08A
:10A9D000CDB7DEB780915A1287FD0EC06F7070E060
:10A9E000992787FD90956817790731F00F900F90A0
:10A9F000DF91CF911F910895411138C030915912C4
:10AA0000223008F47DC0332389F3842F80518E31A6
:10AA1000B0F1842F80558E3108F04CC0E42FF0E067
:10AA2000EE0FFF1FED5BFF4E4081518130E0CA0108
:10AA300096958795969587958F779927821793078F
:10AA4000A9F2CA0188279E7F220F331F220F331FCE
:10AA5000822B932B9183808381E0809327110F9029
:10AA60000F90DF91CF911F910C94D846413009F49B
:10AA70005FC0403409F46BC030915912C4CFE42F49
:10AA8000F0E0EE0FFF1FED53FF4E8081918130E02B
:10AA9000AC01452F552746954217530709F4A6CF19
:10AAA0008C7F9170322F2227330F822B932B91832F
:10AAB0008083D2CF842F80538A3108F097CFE42F40
:10AAC000F0E0F09730E0DF01AF5BB84F4C9187E0EA
:10AAD00090E0841B910902C0359527958A95E2F78D
:10AAE000822FDF01A753BF4E9C91291709F449C05B
:10AAF0002C9311E07197B9F1112309F477CFACCF02
:10AB0000632F772767FD7095822F90E0681779078C
:10AB100009F479CF209359122A83498300DF0E94D8
:10AB20003B480E94D846309159122A8149816BCF07
:10AB3000822F880F10929410809395102A83498356
:10AB40000E94FC21309159122A8149815CCF211148
:10AB500006C00F900F90DF91CF911F91FFCD81E044
:10AB60008093C50B43CF882371F00E94EB1786E0DA
:10AB7000ECEBFBE0AFE1B1E101900D928A95E1F7DA
:10AB8000BBCF10E0B7CF0E94CE17F1CFCF9380910B
:10AB9000FA0C8F3FA9F0C82FCF778091FC0C8C0F57
:10ABA00040E050E060E0885E0E94273B6091FC0C32
:10ABB0006C0F685E40E080915B12CF910C94D82CB2
:10ABC000CF910895CF938091020D882359F1209160
:10ABD000FF0C3091000D2F3F8FEF380719F1809156
:10ABE000FD0C9091FE0C01969093FE0C8093FD0C51
:10ABF00082179307B8F01092FE0C1092FD0CE8E754
:10AC0000FCE004C08CE0E83FF80761F081918F3FE1
:10AC1000C9F3BCDF8091020D8230E1F0833019F17D
:10AC2000813009F1CF91089561507109810991092D
:10AC300060687F6F8F6F9F6F6F5F7F4F8F4F9F4FEA
:10AC4000FB017093F90C6093F80CE858F34F808186
:10AC50008F3F21F50E9444756F777727882790787A
:10AC600097FFEECFE1CF2091F80C3091F90C07C09F
:10AC70009C01FC01E858F34F40814F3F59F4C90152
:10AC800001968F77907897FFF3CF019780689F6F39
:10AC90000196EECF8093F80C9093F90CC081CF779A
:10ACA0008091FB0C885E8C0F23DB8091FB0C885E0F
:10ACB00060E070E88C0F0E94BF2CE091F80CF091DE
:10ACC000F90CE858F34F80818093FA0C8091FB0CCB
:10ACD0008093FC0CA7CF0F931F93CF93DF93182F74
:10ACE000062F8091020D8117C1F050DFCFEFDFEF0B
:10ACF000D093F90CC093F80C8FEF8093FA0C40E8D6
:10AD000050E06FEF70E088E79CE00E94E0740E94E2
:10AD1000301780915D1281110FC0011104C0809124
:10AD2000010D811114C01093020D0093010DDF91EC
:10AD3000CF911F910F910895D093F90CC093F80C07
:10AD40002FEF3FE73093FE0C2093FD0CE6CFA8E7F2
:10AD5000BCE0FD012FEF05C031968CE0E83FF8071D
:10AD600049F0908197FFF8CF2083F6CF8CE0A83F81
:10AD7000B80721F09D919F3FC9F3D5CF07DFD3CF0F
:10AD80000F93CF934FB7F89436EC31BB469A80EED1
:10AD900087B997E09AB98DB981E085B980E488B91F
:10ADA0001BB880E28EB987E481BB52E05A95F1F777
:10ADB00000C026B199B18CB131BB479AC22FC6955C
:10ADC000C37050E8259F90011124C22B292F2071B8
:10ADD000C22B292F269526952870C22B9695907602
:10ADE000C92B90E0880F991F84709927C82B87EE94
:10ADF00087B987EF8AB982EE8DB94FBF8091DA109B
:10AE0000882381F080918D14C5FF2FC08C2785FD8C
:10AE10000EC080915D128230C1F0C0938D14CF912D
:10AE20000F91089580918D148C2785FFF2CF80912A
:10AE3000020D882341F161E0C5FD60E04CDF0E9416
:10AE4000F12480915D12823041F7C0FFE6CF8091FE
:10AE50008D1480FDE2CF8091C7108F5F8093C71063
:10AE6000C0938D14CF910F91089585FFCFCF0E948D
:10AE7000EB1786E0ECEBFBE0AFE1B1E101900D9266
:10AE80008A95E1F7C6CFC5FF11C068DC00E04091AC
:10AE90005B124F70406BE0919F19F091A01920E474
:10AEA00063E070E08FE999E10995B3CF81E0809389
:10AEB000C50B0FE7ECCFCF92DF92EF92FF920F938B
:10AEC0001F93CF93DF931F92CDB7DEB7082F1127C3
:10AED00007FD109583E0E82E8DE0F82EE00EF11EC0
:10AEE000F701EE5FFE4F2081222309F44AC0F801EA
:10AEF000EE0FFF1FE95FF14FC080D1808FEFC81ABE
:10AF0000D80AC601860F911D67FD9A9530E0169507
:10AF1000102F0027179507950D5F124F02C07D3F38
:10AF200069F4820F931F0197B9010E94E270F80142
:10AF3000E80FF91F7281C816D90689F7872F8D5F30
:10AF40008230F8F0E7EFEE1AEEEFFE0AF7018081AB
:10AF500040E050E060E0870F79830E94273BF701D3
:10AF600060817981670F40E080915B120F90DF91E3
:10AF7000CF911F910F91FF90EF90DF90CF900C94A5
:10AF8000D82C0F90DF91CF911F910F91FF90EF90F0
:10AF9000DF90CF900895CF932091100E3091110E35
:10AFA0002F3F8FEF3807C1F080910E0E90910F0E5A
:10AFB000019690930F0E80930E0E8217930760F008
:10AFC00010920F0E10920E0E8091030D823099F1A7
:10AFD0008091040D823011F0CF9108956091060E9A
:10AFE0006623D1F38091090E90910A0E019670E0CC
:10AFF0000E94E27090930A0E8093090EFC01EB57B9
:10B00000F24FC081CD3F41F36FEF81E054DF8C2FD1
:10B010008D5F823008F380910B0E8C0F69D980917F
:10B020000B0E60E070E88C0F0E94BF2C80910B0E1D
:10B0300080930D0ED1CF6091050E662349F2809169
:10B04000070E9091080E019670E00E94E2709093B6
:10B05000080E8093070EFC01ED5FF24FC281CD3FD9
:10B0600009F4B6CF6FEF80E026DF8C2F8D5F823042
:10B0700008F4AECF80910B0E8C0F3AD980910B0E55
:10B0800060E070E88C0F0E94BF2C80910B0E8093C3
:10B090000C0E9ECF26EC90EE87E0F0E8E7E477EE2A
:10B0A00067EF52EE4FB7F89421BB469A97B98AB929
:10B0B0009DB915B8F8B98BB91EB8E1BB32E03A9525
:10B0C000F1F700C036B1A9B1ACB121BB479A77B94D
:10B0D0006AB95DB94FBF45E04A95F1F7000032FF0C
:10B0E000E1CF8FB7F89496EC91BB469A15B890E8EB
:10B0F00098B993E09BB990E29EB997E891BB95E02F
:10B100009A95F1F700008FBF089526EC90EE87E046
:10B11000F0E8E7E477EE67EF52EE4FB7F89421BB23
:10B12000469A97B98AB99DB915B8F8B98BB91EB8BE
:10B13000E1BB32E03A95F1F700C036B1A9B1ACB14C
:10B1400021BB479A77B96AB95DB94FBF45E04A95C7
:10B15000F1F7000032FFE1CF8FB7F89496EC91BB86
:10B16000469A15B892E898B993EC9BB990E29EB9CB
:10B1700097E891BB95E09A95F1F700008FBF08958D
:10B1800026EC90EE87E0F0E8E7E477EE67EF52EE2A
:10B190004FB7F89421BB469A97B98AB99DB915B8AB
:10B1A000F8B98BB91EB8E1BB32E03A95F1F700C0AF
:10B1B00036B1A9B1ACB121BB479A77B96AB95DB9CB
:10B1C0004FBF45E04A95F1F7000032FFE1CF8FB75E
:10B1D000F89496EC91BB469A15B894E898B993E127
:10B1E0009BB992E29EB997E891BB95E09A95F1F7E9
:10B1F00000008FBF089526EC90EE87E0F0E8E7E4CA
:10B2000077EE67EF52EE4FB7F89421BB469A97B9A5
:10B210008AB99DB915B8F8B98BB91EB8E1BB32E04F
:10B220003A95F1F700C036B1A9B1ACB121BB479A4C
:10B2300077B96AB95DB94FBF45E04A95F1F70000AB
:10B2400032FFE1CF8FB7F89496EC91BB469A15B8D0
:10B2500092E898B993E09BB990E29EB997E891BBC8
:10B2600095E09A95F1F700008FBF08952F923F92D5
:10B270004F925F926F927F928F929F92AF92BF9206
:10B28000CF92DF92EF92FF920F931F93CF93DF93B2
:10B29000CDB7DEB76B970FB6F894DEBF0FBECDBF4C
:10B2A000762E882309F494C0E091EF10F091F0100D
:10B2B0008090F1109090F2104091E3105091E410C2
:10B2C0008091E9109091EA1020911B1130911C118E
:10B2D00040900F0C5090100C6090D5106091DF10D2
:10B2E00050928F1540928E15F0939115E093901522
:10B2F00090929315809292155093951540939415C2
:10B3000090939715809396153093991520939815DF
:10B3100060929A1560939B15440C452C441C55086B
:10B32000519482011A9518870F83EE0FEF2FEE1FAD
:10B33000FF0BF1958F011A951A8B098BA12CB12C5B
:10B3400075016401CC0CDD1CEE1CFF1CCC0CDD1C5B
:10B35000EE1CFF1CC80CD91CEA1CFB1C13E0F69465
:10B36000E794D794C7941A95D1F756954795569573
:10B37000479596958795969587950D2D11271C874E
:10B380000B87052F11271A830983092F1127DD2425
:10B39000EE24FF24662309F440C0623008F436C668
:10B3A000ECE0F0E089819A81BF010E94E27049815E
:10B3B0005A81481B590B5A834983C801BF010E9417
:10B3C000E270081B190B188A1F861E861D862DC069
:10B3D00040900F0C5090100C80918E1590918F150D
:10B3E000E091EF10F091F0108415950509F4E9C58E
:10B3F0008090F1109090F2104091E3105091E41081
:10B400008091E9109091EA1020911B1130911C114C
:10B410006090D5106091DF1063CFBA0177277E87E7
:10B420006D87DC01BB27B88BAF875091DA105D8B3D
:10B4300070915E127F8B832F99279C8B8B8B209131
:10B44000C0102E8B77FC29C1772009F426C177FC28
:10B45000CEC431E0731609F4CAC477FCDFC332E00E
:10B46000731609F4DBC377FCEDC233E0731609F4FD
:10B47000E9C277FCFAC134E0731609F4F6C177FC2F
:10B480001CC045E07416C9F06B960FB6F894DEBF89
:10B490000FBECDBFDF91CF911F910F91FF90EF9025
:10B4A000DF90CF90BF90AF909F908F907F906F90E4
:10B4B0005F904F903F902F9008958091B90B882313
:10B4C00019F38091B80B282F30E0285131093C83C3
:10B4D0002B83020F131F2F813885442737FD40959A
:10B4E000542F2F83388749875A878090A2109090D5
:10B4F000A310AA2497FCA094BA2C820E931EA41E1B
:10B50000B51E89819A812B813C81820F931F97FD03
:10B51000F6C645E06D850E948F1314012501280EA3
:10B52000391E411C511C57FCA3C62114310431E0C3
:10B53000430651040CF09AC58090AE109090AF1065
:10B54000AA2497FCA094BA2C2F81388549855A8566
:10B55000820E931EA41EB51E29893A89C901AA2705
:10B5600097FDA095BA2F880E991EAA1EBB1EC80172
:10B5700017FD86C64BE06F850E948F13880E991EBB
:10B58000A11CB11CB7FC7FC68114910431E0A30655
:10B59000B1040CF060C58B859C856110BBC5009122
:10B5A000BA101091BB1041E16C2D0E948F13A801BD
:10B5B000662757FD6095762F480F591F611D711D35
:10B5C00077FDAAC64115510531E06307710524F0E6
:10B5D0004FEF5FEF60E070E00D89011104C01F893B
:10B5E000112309F48FC68B899C89880F991F2B8999
:10B5F0003C89820F931F919581959109AA2797FD08
:10B60000A095BA2F92018101080F191F2A1F3B1F15
:10B6100037FD96C601151105E1E02E07310524F02E
:10B620000FEF1FEF20E030E09801880E991EAA1E50
:10B63000BB1EB7FCA5C681149104F1E0AF06B104AE
:10B640002CF088248A94982CA12CB12C480F591FD7
:10B650006A1F7B1F77FD90C64115510501E0600709
:10B66000710524F04FEF5FEF60E070E01E89112359
:10B6700009F4D8C530936F1020936E1090927B1010
:10B6800080927A1050938710409386106110FCCE00
:10B690005093631040936210F7CE8091820B882301
:10B6A00009F4D5CE8091810B282F30E02851310943
:10B6B0003B8F2A8F200F311F4F815885662757FDFA
:10B6C0006095762F4B835C836D837E8320909810EA
:10B6D000309099104101AA2497FCA094BA2C840EB2
:10B6E000951EA61EB71E89819A816A8D7B8D860F55
:10B6F000971F97FDB3C540E06D85288F398F0E9455
:10B700008F1314012501280E391E411C511C288D50
:10B71000398D57FCEAC52114310471E04706510404
:10B720000CF0B4C48090A4109090A510AA2497FCAB
:10B73000A094BA2C8B819C81AD81BE81880E991E0C
:10B74000AA1EBB1EE989FA89CF01AA2797FDA095F9
:10B75000BA2F880E991EAA1EBB1EC90137FD81C5CE
:10B7600046E06F850E948F13880E991EA11CB11CA4
:10B77000B7FC7AC581149104F1E0AF06B1040CF076
:10B780007BC48B859C856110A7C42091B01030913B
:10B79000B1104CE06C2D288F398F0E948F13288DAB
:10B7A000398DA901662757FD6095762F480F591FDF
:10B7B000611D711D77FDA8C54115510521E0620786
:10B7C000710524F04FEF5FEF60E070E03D893111CB
:10B7D00003C03F893323C9F12B893C89C901AA27BA
:10B7E00097FDA095BA2F280E391E4A1E5B1E57FCE6
:10B7F000BFC52114310431E0430651042CF022244A
:10B800002A94322C412C512C880E991EAA1EBB1E44
:10B81000B7FCAAC581149104E1E0AE06B1042CF096
:10B8200088248A94982CA12CB12C480F591F6A1F88
:10B830007B1F77FD95C541155105F1E06F07710537
:10B8400024F04FEF5FEF60E070E02E892111C4C457
:10B85000309241102092401090924D1080924C10E6
:10B860005093591040935810F2CD8091AE0B88231D
:10B8700009F405CE8091AD0B282F30E02851310915
:10B880003B8F2A8F200F311F4F815885662757FD28
:10B890006095762F4B835C836D837E832090A01010
:10B8A0003090A1104101AA2497FCA094BA2C840ED8
:10B8B000951EA61EB71E89819A816A8D7B8D860F83
:10B8C000971F97FD16C544E06D85288F398F0E941C
:10B8D0008F1314012501280E391E411C511C288D7F
:10B8E000398D57FCC9C42114310471E04706510455
:10B8F0000CF0ECC38090AC109090AD10AA2497FC93
:10B90000A094BA2C8B819C81AD81BE81880E991E3A
:10B91000AA1EBB1EE989FA89CF01AA2797FDA09527
:10B92000BA2F880E991EAA1EBB1EC90137FDBEC4C0
:10B930004AE06F850E948F13880E991EA11CB11CCE
:10B94000B7FCB7C481149104F1E0AF06B1040CF068
:10B95000B3C38B859C856110CEC32091B810309104
:10B96000B91040E16C2D288F398F0E948F13288DDC
:10B97000398DA901662757FD6095762F480F591F0D
:10B98000611D711D77FDCCC44115510521E0620791
:10B99000710524F04FEF5FEF60E070E03D893111F9
:10B9A00003C03F893323F1F18B899C89880F991F4C
:10B9B0002B893C89820F931FAA2797FDA095BA2F48
:10B9C000280E391E4A1E5B1E57FCE2C421143104A6
:10B9D00031E0430651042CF022242A94322C412CCD
:10B9E000512C880E991EAA1EBB1EB7FCCDC4811413
:10B9F0009104E1E0AE06B1042CF088248A94982CDE
:10BA0000A12CB12C480F591F6A1F7B1F77FD94C4CE
:10BA100041155105F1E06F07710524F04FEF5FEF1D
:10BA200060E070E02E89211106C430924910209206
:10BA3000481090925510809254105093611040938A
:10BA400060101DCD8091A30B882309F412CD809145
:10BA5000A20B282F30E0285131093B8F2A8F200F6D
:10BA6000311F4F815885662757FD6095762F4B8390
:10BA70005C836D837E8320909E1030909F104101E7
:10BA8000AA2497FCA094BA2C840E951EA61EB71E5D
:10BA900089819A816A8D7B8D860F971F97FD2CC4B3
:10BAA00043E06D85288F398F0E948F131401250183
:10BAB000280E391E411C511C288D398D57FCEBC3B3
:10BAC0002114310471E0470651040CF0EFC280905C
:10BAD000AA109090AB10AA2497FCA094BA2C8B814A
:10BAE0009C81AD81BE81880E991EAA1EBB1EE9896C
:10BAF000FA89CF01AA2797FDA095BA2F880E991E23
:10BB0000AA1EBB1EC90137FDCAC349E06F850E944A
:10BB10008F13880E991EA11CB11CB7FCC3C38114DE
:10BB20009104F1E0AF06B1040CF0B6C28B859C85A0
:10BB30006110FFC22091B6103091B7104FE06C2D0C
:10BB4000288F398F0E948F13288D398DA901662780
:10BB500057FD6095762F480F591F611D711D77FDA8
:10BB6000E7C34115510521E06207710524F04FEF4D
:10BB70005FEF60E070E03D89311103C02F8922231F
:10BB8000E9F18B899C89919581959109880F991F7D
:10BB9000AA2797FDA095BA2F280E391E4A1E5B1EB4
:10BBA00057FC02C421143104E1E04E0651042CF08C
:10BBB00022242A94322C412C512C880E991EAA1E24
:10BBC000BB1EB7FCEDC381149104F1E0AF06B104D4
:10BBD0002CF088248A94982CA12CB12C480F591F42
:10BBE0006A1F7B1F77FDD8C34115510521E062070D
:10BBF000710524F04FEF5FEF60E070E03E89311196
:10BC0000FEC23092471020924610909253108092BC
:10BC1000521050935F1040935E102BCC8091980B84
:10BC2000882309F420CC8091970B282F30E02851ED
:10BC300031093B8F2A8F200F311F4F81588566278E
:10BC400057FD6095762F4B835C836D837E832090B8
:10BC50009C1030909D104101AA2497FCA094BA2C0E
:10BC6000840E951EA61EB71E89819A816A8D7B8DD2
:10BC7000860F971F97FD28C342E06D85288F398F67
:10BC80000E948F1314012501280E391E411C511CDE
:10BC9000288D398D57FC25C32114310471E04706E6
:10BCA00051040CF0CCC18090A8109090A910AA2447
:10BCB00097FCA094BA2C8B819C81AD81BE81880EAB
:10BCC000991EAA1EBB1EE989FA89CF01AA2797FDF2
:10BCD000A095BA2F880E991EAA1EBB1EC90137FD5A
:10BCE000F9C248E06F850E948F13880E991EA11C2F
:10BCF000B11CB7FCF2C281149104F1E0AF06B104AB
:10BD00000CF093C18B859C85611022C22091B410E8
:10BD10003091B5104EE06C2D288F398F0E948F1313
:10BD2000288D398DA901662757FD6095762F480F1C
:10BD3000591F611D711D77FDEBC24115510521E0B1
:10BD40006207710524F04FEF5FEF60E070E03D891E
:10BD5000311103C02F892223D1F18B899C89880F4F
:10BD6000991FAA2797FDA095BA2F280E391E4A1EA3
:10BD70005B1E57FC25C321143104E1E04E0651043B
:10BD80002CF022242A94322C412C512C880E991EFE
:10BD9000AA1EBB1EB7FC10C381149104F1E0AF06CC
:10BDA000B1042CF088248A94982CA12CB12C480F33
:10BDB000591F6A1F7B1F77FDFBC24115510521E00A
:10BDC0006207710524F04FEF5FEF60E070E03E899D
:10BDD0003111EFC1309245102092441090925110D1
:10BDE0008092501050935D1040935C103CCB80913A
:10BDF0008D0B882309F431CB80918C0B282F30E0F8
:10BE0000285131093B8F2A8F200F311F4F815885D0
:10BE1000662757FD6095762F4B835C836D837E8309
:10BE200020909A1030909B104101AA2497FCA09476
:10BE3000BA2C840E951EA61EB71E89819A816A8D22
:10BE40007B8D860F971F97FD42C241E06D85288F3D
:10BE5000398F0E948F1314012501280E391E411CB1
:10BE6000511C288D398D57FC12C22114310471E008
:10BE7000470651040CF0E9C08090A6109090A710DE
:10BE8000AA2497FCA094BA2C8B819C81AD81BE81A1
:10BE9000880E991EAA1EBB1EE989FA89CF01AA271E
:10BEA00097FDA095BA2F880E991EAA1EBB1EC90128
:10BEB00037FD03C247E06F850E948F13880E991EDD
:10BEC000A11CB11CB7FCFCC181149104F1E0AF06C8
:10BED000B1040CF0A0C08B859C85611048C12091F5
:10BEE000B2103091B3104DE06C2D288F398F0E9425
:10BEF0008F13288D398DA901662757FD6095762F00
:10BF0000480F591F611D711D77FD0EC24115510566
:10BF100021E06207710524F04FEF5FEF60E070E011
:10BF20003D89311103C02F892223D9F18B899C8946
:10BF3000919581959109AA2797FDA095BA2F280E72
:10BF4000391E4A1E5B1E57FC07C221143104E1E072
:10BF50004E0651042CF022242A94322C412C512CD0
:10BF6000880E991EAA1EBB1EB7FCF2C18114910453
:10BF7000F1E0AF06B1042CF088248A94982CA12C0F
:10BF8000B12C480F591F6A1F7B1F77FDDDC141157A
:10BF9000510521E06207710524F04FEF5FEF60E08B
:10BFA00070E03E893111F2C030924310209242106D
:10BFB00090924F1080924E1050935B1040935A1005
:10BFC0004CCA80919015909191158090F1109090AD
:10BFD000F210E817F90709F00FCA809192159091B5
:10BFE00093154091E3105091E4108816990609F4D6
:10BFF00027C28091E9109091EA1020911B11309195
:10C000001C116090D5106091DF106AC9188A1F86D4
:10C010001E861D860ACA88248A94982CA12CB12CCD
:10C020008B859C856110A3C05ACF88248A94982C54
:10C03000A12CB12C8B859C8561108AC067CE2224EF
:10C040002A94322C412C512C2ECE22242A94322C8C
:10C05000412C512C11CF88248A94982CA12CB12CDE
:10C060008B859C85662009F49ACA54C022242A94A0
:10C07000322C412C512C60CA88248A94982CA12CF3
:10C08000B12C8B859C85611027C07FCB22242A94FC
:10C09000322C412C512C46CB88248A94982CA12CEC
:10C0A000B12C8B859C85611044C044CD22242A94F8
:10C0B000322C412C512C0BCD88248A94982CA12C05
:10C0C000B12C8B859C85611016C047CC22242A9404
:10C0D000322C412C512C0ECC41E0641609F47EC167
:10C0E0008B859C852A8D3B8D820F931F97FF4DCBAF
:10C0F00080E090E04ACB41E0641609F465C18B858D
:10C100009C852A8D3B8D820F931F97FF26CC80E064
:10C1100090E023CC41E0641609F488C18B859C85AE
:10C120002B813C81820F931F97FF39CA80E090E0FA
:10C1300036CA31E0631609F465C18B859C852A8D6A
:10C140003B8D820F931F97FFF5CC80E090E0F2CCFF
:10C1500031E0631609F44CC18B859C852A8D3B8D9B
:10C16000820F931F97FFD2CD80E090E0CFCD31E0DA
:10C17000631609F451C18B859C852A8D3B8D820FF6
:10C18000931F97FFACCE80E090E0A9CE309267106D
:10C1900020926610909273108092721050937F10CC
:10C1A00040937E10611059C950935B1040935A1010
:10C1B00054C9309269102092681090927510809244
:10C1C0007410509381104093801061104CC95093AB
:10C1D0005D1040935C1047C9309265102092641046
:10C1E000909271108092701050937D1040937C104B
:10C1F00061102DC9509359104093581028C930929E
:10C200006B1020926A109092771080927610509363
:10C2100083104093821061102CC950935F1040939B
:10C220005E1027C930934B1020934A1090925710FC
:10C23000809256102DCA30926D1020926C10909200
:10C24000791080927810509385104093841061107B
:10C2500016C9509361104093601011C980E090E0BE
:10C260004ACA80E090E07CCA812C912C540182CA99
:10C27000212C312C210159C9212C312C210133CB06
:10C2800080E090E077C9812C912C54017DC9212C4C
:10C29000312C2101EACD212C312C210111CC80E05F
:10C2A00090E033CC812C912C540139CC80E090E08B
:10C2B0003FCB812C912C540145CB80E090E0FACD0E
:10C2C000812C912C540100CE80E090E0D5CC80E010
:10C2D00090E0BBCD80E090E004CD812C912C540106
:10C2E0000ACD212C312C2101D7CC212C312C21013C
:10C2F00012CA80E090E0E7CA80E090E0D1CB80E015
:10C3000090E007C99101B2C940E050E0BA0154CAB7
:10C3100040E050E0BA0111CD40E050E0BA0152C90E
:10C3200040E050E0BA0130CB40E050E0BA01EECD41
:10C3300040E050E0BA0115CC40E050E0BA0168CBD3
:10C3400000E010E0980166C940E050E0BA011FCE5D
:10C35000812C912C54010ACE212C312C2101F5CDB8
:10C3600040E050E0BA0167CA812C912C540152CAB6
:10C37000212C312C21013DCA40E050E0BA016CC9AA
:10C38000812C912C540157C9812C912C54012FCB15
:10C39000212C312C21011ACB40E050E0BA0124CCF1
:10C3A000812C912C54010FCC212C312C2101FACB62
:10C3B00040E050E0BA0101CD812C912C5401ECCC2D
:10C3C000212C312C2101D7CC8A8D9B8D97FD55C016
:10C3D0009C01359527953B8F2A8F91CE8A8D9B8D19
:10C3E00097FD4DC09C01359527953B8F2A8F78CEC0
:10C3F0008A8D9B8D97FD45C09C01359527953B8F78
:10C400002A8FAACE8A8D9B8D97FD3FC09C013595C2
:10C4100027953B8F2A8F91CE8A8D9B8D97FD33C0B8
:10C420009C01359527953B8F2A8FA5CE8B819C81CA
:10C4300097FD2DC08C01159507951C830B836ECE3F
:10C4400080919415909195154817590709F0D1CD11
:10C450008091E9109091EA102091961530919715EE
:10C4600082179307B1F020911B1130911C1160903D
:10C47000D5106091DF100C9470590196A9CF0196E8
:10C48000B1CF0196B9CF0196CBCF0196BFCF019620
:10C49000D1CF20911B1130911C1160919815709192
:10C4A00099156090D5102617370721F06091DF109D
:10C4B0000C94705960919A156612F8CF6091DF1054
:10C4C00070919B1567130C9470590C94445A7F9289
:10C4D0008F929F92AF92BF92CF92DF92EF92FF9294
:10C4E0000F931F93CF93DF9300D0CDB7DEB71A829F
:10C4F0001982C12CD12C08C08FEFC81AD80A84E643
:10C50000C816D10409F468C0C6010E94B61A88236F
:10C5100099F3BE016F5F7F4FC6010E94511AE980F7
:10C52000FA807FB6F89481E0E81AF108F594E79470
:10C53000F594E7948FEFE81AF80A0E940B300E94F6
:10C540004A580E9485580E94C0580E94FB581E14E9
:10C550001F04BCF500E010E0F801EE0FFF1FEE0F26
:10C56000FF1FE156F84E8080A1809280B380882D15
:10C570008F770E94012D8A2D8F770E94012D892DA2
:10C580008F770E94012D8B2D8F770E94012D992D81
:10C590009295969594703A2D3295369536953270DF
:10C5A000932B2B2D22952870922B882D881F88275E
:10C5B000881F892B0E94012D0F5F1F4F0E151F052D
:10C5C0005CF20E944F2D7FBE8FEFC81AD80A84E616
:10C5D000C816D10409F098CF0F900F90DF91CF913A
:10C5E0001F910F91FF90EF90DF90CF90BF90AF9091
:10C5F0009F908F907F900895CF92DF92FF920F933C
:10C600001F93CF93DF9300D0CDB7DEB78C01FFB679
:10C610007A8369830E94FB195A8169818823E1F03A
:10C62000ECE9F5E120E032E0DF01C9011D9201975C
:10C63000E9F7C62ED52E24EA37E1462FB901CF01FE
:10C640000E94C674C60184569A4E90939D1780939B
:10C650009C17C8010E9419348F2D0F900F90DF9105
:10C66000CF911F910F91FF90DF90CF900C94BF1945
:10C670002F923F924F925F926F927F928F929F92F2
:10C68000AF92BF92CF92DF92EF92FF920F931F93E0
:10C69000CF93DF93CDB7DEB7C958D1090FB6F89461
:10C6A000DEBF0FBECDBF839709F0F6C280919F1702
:10C6B000813009F0F1C28091A017823009F0ECC2FC
:10C6C0002091A117AE962FAFAE97243608F0E4C2A2
:10C6D000DE01A35ABF4F80E090E09C012156384E06
:10C6E000F9014481F0E14F9FA0011124F901238158
:10C6F0002F70242B2D9302968032910571F7A3960B
:10C700002FADA397922F9295969596959370A49698
:10C710004FADA497842F8F70880F880F892B982E88
:10C72000990C990C812CB40160957095E0967FAFBF
:10C730006EAFE097A2968FADA297A82EA694AA0CF2
:10C74000AA0CA1963FADA197932F96959695969595
:10C75000FF24F394F822F294FF0CB0EEFB22F92AA6
:10C76000FF0CFF0C582F551F5527551F2F73220FF5
:10C77000922F952B80E0BC017058E2967FAF6EAF90
:10C78000E2976E968FAD6E97782F770FCF57DF4F6A
:10C790007883C158D040AB962FADAB97922F9E7F38
:10C7A000CE57DF4F9883C258D04042954F70A59620
:10C7B0009FADA59717E0D12ED922D29400EFD022B9
:10C7C000D42A492F469546954695A6969FADA6979D
:10C7D000092F01700295000F007E042B000F000F3F
:10C7E000692F660F660F562F587740E0BA017058D0
:10C7F000E4967FAF6EAFE497492F42954695477018
:10C80000A7969FADA797A92FA170AA0FAA0FAA0F4D
:10C81000A42BB0E0A55AB84F7C91EC967FAFEC9773
:10C82000B92EB694B29440EFB422492F4295469562
:10C830004770A8969FADA897A92FA170AA0FAA0F1D
:10C84000AA0FA42BB0E0A55AB84F4C91ED964FAF6C
:10C85000ED97A92FA695AF70B0E0A55AB84F6C918F
:10C86000EE966FAFEE97492F429546954770A99681
:10C870009FADA997A92FA170AA0FAA0FAA0FA42B49
:10C88000B0E0A55AB84F7C91EF967FAFEF97C92ED5
:10C89000C694C29450EFC522929596959770AA9629
:10C8A0004FADAA97A42FA170AA0FAA0FAA0FA92B68
:10C8B000B0E0A55AB84F9C91C158DF4F9883CF572D
:10C8C000D040A42FA695AF70B0E0A55AB84F6C9198
:10C8D000C058DF4F6883C058D040881F8827881F02
:10C8E0006F965FAD6F97652F6770660F682B962FF9
:10C8F000990F990F990F80E0BC017058E6967FAFB1
:10C900006EAFE697952F991F9927991FA0968FAD27
:10C91000A097182F1F73110F192B110F952F969594
:10C920009C7382958695869583703770330F330F8D
:10C93000382B80E1389FB0011124E8967FAF6EAFAD
:10C94000E8974295469547702170220F220F220FDB
:10C95000242B40E050E029F0522F550F550F40E0B6
:10C960005054AD964FACAD97742D717041FA662757
:10C9700060F9AC968FADAC97282F2170E9962FAF58
:10C98000E99743FA332730F9EA963FAFEA9744FA3A
:10C99000332730F981FB222720F942FA222420F89C
:10C9A00045FA332430F846FA442440F884FB5524F1
:10C9B00050F886FBEE27E0F9F0E0EE0FFF1F87FB53
:10C9C000EE24E0F8EE0CEE0CEE2A85FBEE27E0F903
:10C9D000EE2A83FB662460F882FF02C082E001C079
:10C9E00080E0680EAD967FACAD9777FA772470F84B
:10C9F0008FB7EB968FAFEB97CA57DF4F2883C65898
:10CA0000D040CB57DF4F3883C558D040C957DF4F90
:10CA10004883C758D040C857DF4F5883C858D040C4
:10CA2000CC57DF4F6883C458D040CD57DF4F788351
:10CA3000C358D040C757DF4F9883C958D0400E9491
:10CA4000BC19CA57DF4F2881C658D040CB57DF4F9B
:10CA50003881C558D040C957DF4F4881C758D040AA
:10CA6000C857DF4F5881C858D040CC57DF4F688136
:10CA7000C458D040CD57DF4F7881C358D040C757F6
:10CA8000DF4F9881C958D040882309F4E7C08CE56E
:10CA9000E9ECF0E1DE01119601900D928A95E1F743
:10CAA0007093C9106093CA10E9966FADE9976093CF
:10CAB000CB10EA967FADEA977093CC103093CD10EF
:10CAC0002093CE102092CF103092D0104092D110EF
:10CAD0005092D2101092D310E092D4106092D510E0
:10CAE0001092D61081E08093D7101092D8107092D7
:10CAF000DA101092DB1023E02093DC108093DD101D
:10CB000022E02093DE108093DF108093E2101092D9
:10CB1000E310A092E410E0962EAD3FADE097309385
:10CB2000E6102093E5101092E710CF57DF4F3881C1
:10CB3000C158D0403093E8101092E910F092EA10FA
:10CB40009092EC108092EB101092ED10CE57DF4FC8
:10CB50006881C258D0406093EE10E2962EAD3FAD92
:10CB6000E2973093F0102093EF101092F110D092D2
:10CB7000F2101092F3100093F410E4966EAD7FADB6
:10CB8000E4977093F6106093F5101092F710EC96FE
:10CB90007FADEC977093F8101092F910B092FA10E4
:10CBA0001092FB10ED962FADED972093FC10109294
:10CBB000FD10EE963FADEE973093FE101092FF10F1
:10CBC000EF966FADEF976093001110920111C09234
:10CBD000021110920311C158DF4F7881CF57D04016
:10CBE0007093041110920511C058DF4F2881C0586E
:10CBF000D04020930611E6966EAD7FADE697709318
:10CC00000811609307111092091110930A111092E4
:10CC10000B1190930C11E8962EAD3FADE897309331
:10CC20000E1120930D115093101140930F1110927B
:10CC30001211109211111092141110921311AE963C
:10CC40008FADAE9790E00E942A348CE5FE013196BC
:10CC5000A9ECB0E101900D928A95E1F7EB968FADCA
:10CC6000EB97C757DF4F0FB6F894DEBF0FBECDBFAF
:10CC7000DF91CF911F910F91FF90EF90DF90CF90B8
:10CC8000BF90AF909F908F907F906F905F904F90EC
:10CC90003F902F900C94BA19C757DF4F0FB6F894F6
:10CCA000DEBF0FBECDBFDF91CF911F910F91FF90DF
:10CCB000EF90DF90CF90BF90AF909F908F907F903C
:10CCC0006F905F904F903F902F9008952F923F92DA
:10CCD0004F925F926F927F928F929F92AF92BF928C
:10CCE000CF92DF92EF92FF920F931F93CF93DF9338
:10CCF000803F09F440C0873FB1F02091CB0B3091C9
:10CD0000CC0B211592E039070CF456C041E050E0FD
:10CD100020E030E0F901E156F84E80835093CC0BCF
:10CD20004093CB0B36C080919F17813009F448C0E7
:10CD3000811109C08091A017813629F48091A11733
:10CD4000863109F448C01092CC0B1092CB0BDF91C6
:10CD5000CF911F910F91FF90EF90DF90CF90BF90F8
:10CD6000AF909F908F907F906F905F904F903F908B
:10CD70002F900C94D8461092CC0B1092CB0B80E0E5
:10CD800092E0EFE9F7E1DF019C011D922150304074
:10CD9000E1F7DF91CF911F910F91FF90EF90DF901E
:10CDA000CF90BF90AF909F908F907F906F905F904B
:10CDB0004F903F902F900895A9014F5F5F4FAACFEA
:10CDC0008091A017823009F0BECF8091CB0B90915B
:10CDD000CC0B4EDCB8CF8091A217813009F0B3CFD5
:10CDE0008091CB0B9091CC0B049765E070E00E9492
:10CDF000E2701B0177FD72C0E3EAAE2EE7E1BE2EC2
:10CE0000F4EACF2EF7E1DF2EA5EAEA2EA7E1FA2E0B
:10CE100006EA17E12B01440C551C440C551C460E28
:10CE2000571E39E0430E511CC4E0D0E084E0682E68
:10CE3000712C7FE9872E77E1972E8C0E9D1E44E0A2
:10CE400050E0B401C3018156984E0E94CF74D401C2
:10CE500014962C91B0E82B9FC0011124F50190810C
:10CE6000982B9083922F92709295990F990F907CA6
:10CE7000D6018C91982B9C93922F94709295990F38
:10CE8000907EF7018081982B9083822F8870829505
:10CE9000807FD8019C91892B8C93B4E06B0E711C20
:10CEA0002596E4E0AE0EB11CF4E0CF0ED11C24E0D8
:10CEB000E20EF11C0C5F1F4FC415D50509F0B9CF68
:10CEC000C1010296880F991F880F991FBC016550F8
:10CED00071098091A31790E08FDB35CF84E090E05B
:10CEE000F5CFEF92FF920F93CF93DF931F92CDB7C1
:10CEF000DEB77B016091CB0B7091CC0B6115710596
:10CF000029F0E61AF70A81E0E81AF108E114F104C1
:10CF100039F40F90DF91CF910F91FF90EF9008952A
:10CF2000842F2983D3DE2981E2E0EE16F10488F311
:10CF3000822FCCDEF2E0EF16F10459F3802F0F9030
:10CF4000DF91CF910F91FF90EF90C0CE1F920F9283
:10CF50000FB60F9211240F900FBE0F901F901895CF
:10CF60001F920F920FB60F9211240F900FBE0F90C9
:10CF70001F9018951F920F920FB60F9211240BB6A7
:10CF80000F922F933F934F935F936F937F938F9362
:10CF90009F93AF93BF93CF93DF93EF93FF93349916
:10CFA0007CC0CFB7F89456EC51BB469A70EE77B977
:10CFB00067E06AB97DB915B8D0E8D8B96BB91EB8C1
:10CFC000B7E4B1BB82E08A95F1F700C026B199B110
:10CFD0008CB151BB479A422F46954370E0E82E9F93
:10CFE00090011124422B292F2071422B292F2695A5
:10CFF00026952870422B96959076492B90E0880FC5
:10D00000991F84709927482BA7EEA7B9F7EFFAB9B3
:10D01000E2EEEDB985E08A95F1F7000047FF54C0D4
:10D0200040FF52C051BB469A77B96AB97DB915B86D
:10D03000D8B96BB980E28EB9B1BB82E08A95F1F7BD
:10D0400000C026B199B18CB151BB479A622F669549
:10D05000637050E8259F90011124622B292F2071C5
:10D06000622B292F269526952870622B969590760F
:10D07000692B90E0880F991F84709927682BA7B9B6
:10D08000FAB9EDB985E08A95F1F7000044FD1AC0C0
:10D0900087E89AE10E94E050CFBFFF91EF91DF91C6
:10D0A000CF91BF91AF919F918F917F916F915F9140
:10D0B0004F913F912F910F900BBE0F900FBE0F908D
:10D0C0001F9018950E94CA2FCFBFE7CF1F920F92D3
:10D0D0000FB60F9211240BB60F922F933F934F93DD
:10D0E0005F936F937F938F939F93AF93BF93CF93F0
:10D0F000DF93EF93FF93CEE6D0E088818D7F888326
:10D1000085B3876085BB78940E944602F894888135
:10D1100082608883FF91EF91DF91CF91BF91AF91B2
:10D120009F918F917F916F915F914F913F912F913F
:10D130000F900BBE0F900FBE0F901F901895CF93BE
:10D14000DF93CDB7DEB7AC970FB6F894DEBF0FBE56
:10D15000CDBF20E82093610010926100F89414B8CC
:10D1600017B81AB81DB810BA15B8B0EEDB2ED8B87B
:10D170001BB81EB883EE81BBCC24CA94C4B8D7B800
:10D1800017E0912E9AB8DDB880BB8CE787BD84B5D7
:10D19000826084BD85B5836085BD80916E008260AC
:10D1A00080936E00EC9A06ECB02EB1BA469AD7B8CE
:10D1B0009AB8DDB815B828B91BB81EB887E4582E40
:10D1C00051BA32E03A95F1F700C086B189B18CB11D
:10D1D000B1BA479A97EE692E67B837EF732E7AB8CF
:10D1E00042EE842E8DB852E1E52E5EE0F52E87EBFF
:10D1F00092E0D701FC011D923197E9F7E9EAF9E0E5
:10D20000DF011D922A95E9F781E4E9E2FAE0DF0106
:10D210001D928A95E9F760E2A62EA092380A85E46D
:10D22000E3E3FCE0DF011D928A95E9F786E6EDEC89
:10D23000FBE0DF011D928A95E9F7C092320C0E9453
:10D24000931E8CE591E0EAE6FAE0DF019C011D9275
:10D2500021503040E1F78FE38093C30B46E050E06C
:10D260006FEF70E08CEB9BE00E94E0741092BC0BBF
:10D270000E94CA2F8FE091E0E3E0FDE0DF019C0116
:10D280001D9221503040E1F70FEF1FEF1093080E71
:10D290000093070E40E850E06FEF70E085E09DE0FE
:10D2A0000E94E07410930A0E0093090E40E850E0CB
:10D2B0006FEF70E085E89DE00E94E0748BE8E8E79E
:10D2C000FCE0DF011D928A95E9F740E850E06FEF3E
:10D2D00070E0CF010E94E0741093F90C0093F80CF9
:10D2E000C092FA0C80E1E5E2F1E1DF011D928A953E
:10D2F000E9F7C0922611C09228118FEF9FEFDC0151
:10D300008093291190932A11A0932B11B0932C1183
:10D3100011E010932711C09233111092C41910928A
:10D32000C6191092C51980EC8093891A87EC99E18F
:10D3300090938B1A80938A1A1092881A1092871AE7
:10D340001092A8191092A7191092AC191092AB194B
:10D350001092B0191092AF191092B2191092B1191F
:10D360001092B4191092B3191092B8191092B719FB
:10D370001092BC191092BB191092BE191092BD19CF
:10D380001092C0191092BF1981E291E59093A019F3
:10D3900080939F198DE591E59093A4198093A3192B
:10D3A0008AE491E59093A6198093A51984EE94E5FB
:10D3B0009093A2198093A1198CE692E39093AE19F1
:10D3C0008093AD1988EF92E29093AA198093A919DE
:10D3D00081E797E69093BA198093B91989EB98E29F
:10D3E0009093B6198093B5191092CC0B1092CB0B79
:10D3F000A092C80B80E692E19093CA0B8093C90B70
:10D400001092C70B1092C60B8AE2EEE0FFE0DF013C
:10D41000482E1D924A94E9F7D701E82F1D92EA950C
:10D42000E9F7E8E3FFE0DF01482E1D924A94E9F7AF
:10D43000ECE3FEE0DF01482E1D924A94E9F7E2E6B4
:10D44000FFE0DF01482E1D924A94E9F7E6E6FEE090
:10D45000DF01482E1D924A94E9F7ECE8FFE0DF0176
:10D46000482E1D924A94E9F7E0E9FEE0DF01482EDC
:10D470001D924A94E9F7E6EBFFE0DF01482E1D928A
:10D480004A94E9F7EAEBFEE0DF01482E1D924A9448
:10D49000E9F7E0EEFFE0DF01482E1D924A94E9F73C
:10D4A000E4EEFEE0DF011D928A95E9F78AE090E163
:10D4B0000E949A1F85E290E10E949A1F61E085E236
:10D4C00090E10E947B1F64E085E290E10E945F1979
:10D4D000B1BA469AD7B89AB8DDB815B980E488B918
:10D4E0001BB8AEB851BAB2E0BA95F1F700C086B138
:10D4F00089B19CB1B1BA479A67B87AB88DB884FD42
:10D50000F1C18BED90E00E94B61A811106C00E9415
:10D51000251B8BED90E00E942A340E947E1B811116
:10D5200004C00E94EB1E0E94573581E00E944037E4
:10D530008091310C00E210E0A6E1FA2E0E94443105
:10D540002091310C203109F4C9C1332727FD3095D2
:10D550002F5F3F4F2F71307837FF06C021503109C0
:10D56000206E3F6F2F5F3F4F822F2093310C015071
:10D57000110921F781E00E94443180E10E94443189
:10D580008EE10E9444318DE10E944431A0900E0151
:10D59000B0900F01009112011091130180901001C1
:10D5A000909011019501201B310B2819390940E099
:10D5B00050E0C12CD12CE12CE0E8FE2EC701B601D1
:10D5C0000E94CA75209314013093150140931601EF
:10D5D000509317019401209530952A193B09201B7F
:10D5E000310B40E050E0C701B6010E94CA7520939C
:10D5F00018013093190140931A0150931B010091B7
:10D600005512109156121093010100930001A09041
:10D610000401B090050180900201909003019801EF
:10D620002A193B092819390940E050E0C701B60121
:10D630000E94CA75209306013093070140930801A8
:10D6400050930901940120953095201B310B2A1924
:10D650003B0940E050E0C701B6010E94CA75209323
:10D660000A0130930B0140930C0150930D010E946D
:10D670003B480E94D8468BE697E00E941A177894A0
:10D68000F6EC2F2E9FB7F894809180128F5F8093D5
:10D69000801221BA469A81708D871E864D845E84E1
:10D6A000440C551C440C551C920121633E872D8768
:10D6B0008D8586958270806C31E035B942E448B939
:10D6C00050E55BB98EB987E881BB9FBF1092CD0B47
:10D6D0001092CE0B1092CF0B1092D00B9FEF909325
:10D6E000320C8091310C0E9444312091310C203158
:10D6F00009F424C2332727FD30952F5F3F4F2F7148
:10D70000307837FDC5C3822F2093310C0E944431FD
:10D710002091310C203109F40CC2332727FD3095BC
:10D720002F5F3F4F2F71307837FDABC3822F20938F
:10D73000310C0E9444312091310C203109F4F4C1A4
:10D74000332727FD30952F5F3F4F2F71307837FDFE
:10D75000ABC3822F2093310C0E9444318091310C55
:10D76000803109F4DDC1992787FD909501968F716D
:10D77000907897FD94C38093310C81E00E944431EE
:10D7800080E10E9444318EE10E9444318DE10E948B
:10D7900044319090320C44244A94941002C09090EA
:10D7A00028119092281167E1562E951409F42EC184
:10D7B0004090CD0B5090CE0B6090CF0B7090D00B63
:10D7C00020910E0130910F013A8B298B409112016B
:10D7D000509113015C8B4B8B809110019091110142
:10D7E000988B8F877C01E094F094241B350B388F45
:10D7F0002F8B9C0140E050E02D8F3E8F4F8F58A320
:10D800008091140190911501A0911601B09117011A
:10D81000898F9A8FAB8FBC8FAB89BC89E989FA89D4
:10D82000AE0FBF1FBE8BAD8B9D0140E050E02DA31E
:10D830003EA34FA358A78091180190911901A09180
:10D840001A01B0911B0189A39AA3ABA3BCA3909129
:10D8500027118091591200E916E033EEA32E30E132
:10D86000B32E882309F417C1C92CDD24C7FCD0943A
:10D87000392C2BC0E82FFF27E7FDF095B301A2015B
:10D88000082E04C076956795579547950A94D2F768
:10D8900040FF14C0EE0FFF1FEF50F44F80809180C7
:10D8A0000E94821E882331F0E814F904E8F48824E9
:10D8B0008A94982CF5019182808291E0A2E0AA0ED0
:10D8C000B11CB6E00E3A1B0779F1D8018D918D019C
:10D8D0008F3FA1F38311CECFF601DCCFF092310C54
:10D8E00086E145CE0E94DE4D2F853889821693064B
:10D8F00008F47FC0A40160E070E08F89988D8816DD
:10D90000990608F079C09A01AB018D8D9E8DAF8D7F
:10D91000B8A1281B390B4A0B5B0B698D7A8D8B8D57
:10D920009C8D35D44C01C6CF90932711FFEF3F1645
:10D9300009F44CC0E32DEE0FFF0BEF50F44F0081C4
:10D940001181A80160E070E08091291190912A1165
:10D95000A0912B11B0912C11481759076A077B072A
:10D96000A9F14093291150932A1160932B117093C0
:10D970002C1110932E1100932D11832D09A75AA756
:10D980006BA77CA70E94821E49A55AA56BA57CA502
:10D99000882371F08F8598898095909580179107DD
:10D9A00008F000C38FEF9FEF90932E1180932D11FD
:10D9B0000E94F12480912811863109F413C380312B
:10D9C00009F421C38450883008F4E9C21091801210
:10D9D0001370123009F426C1133009F4D0C011308D
:10D9E00009F4C7C10E94FC216FEF80E00E94365904
:10D9F00049CE812C912C5ECFAD89BE89A815B90581
:10DA000008F4ABC0812C90E8992E54CFE0913311EB
:10DA1000E7FDCECE20911F0C3091200C2901612C06
:10DA2000712C8091291190912A11A0912B11B09104
:10DA30002C11481659066A067B0609F4B9CEFF2751
:10DA4000E7FDF095CF01880F991F8E0F9F1F880F5C
:10DA5000991F880F991F80569A4F1CE0FC01DE0128
:10DA6000119601900D921A95E1F7DC010C91119637
:10DA70001C91011132C2E12FEE0FFF0BED51FF4E51
:10DA80003183208355245394509227110E94D84605
:10DA9000909028118DCE392C8F88988CCF84D8887F
:10DAA0000FC066246A94762CD5016D927C9291E029
:10DAB000B2E0AB0EB11CE6E00E3A1E0709F434CF1B
:10DAC000F80181918F018F3F99F3E82FEE0FFF0B43
:10DAD000EF50F44F608071800E94821E882321F3F2
:10DAE000E614F704F0F26C147D04B8F0C301A0E072
:10DAF000B0E06814790438F59C01AD014D8C5E8C62
:10DB00006F8C78A02419350946095709698D7A8DDB
:10DB10008B8D9C8D3CD33C01C7CF612C712CC4CF25
:10DB2000F6E1F093310C29CEE6E1E093310C86E189
:10DB300013CEB6E1B093310C86E1FBCDA6E1A09304
:10DB4000310C86E1E3CD4D885E884614570408F415
:10DB5000B2C1612C80E8782EA7CF9A01AB018DA1CC
:10DB60009EA1AFA1B8A5281B390B4A0B5B0B69A17D
:10DB70007AA18BA19CA10BD390584C019BCE0E9403
:10DB8000594B00E010E423E035E440E050EE6BE256
:10DB900076E480910F11909110110E948D189C01D4
:10DBA0009093BF108093BE1081E0203D37400CF071
:10DBB00080E08093C01080911D1190911E118115FD
:10DBC000A4E09A0708F4E0C120915D12222309F431
:10DBD00049C2AC0160E070E0DB01CA01880F991F07
:10DBE000AA1FBB1F880F991FAA1FBB1F880F991F51
:10DBF000AA1FBB1F840F951FA61FB71F880F991F51
:10DC0000AA1FBB1FFD01EE0FFF1FE255F94F8081D8
:10DC100091819093000D8093FF0C9093110E80934F
:10DC2000100EE2CE8091E5109091E610EFB6F894D8
:10DC30000E94332B21BA469A4424439445B883E486
:10DC400088B900EF0BB910EA1EB977E8572E51BA20
:10DC500025E02A95F1F7000021BA469A45B888B91F
:10DC6000E0E7FE2EFBB81EB951BA3AE03A95F1F75B
:10DC700000C021BA469A45B888B90BB91EB951BA45
:10DC80004AE04A95F1F700C0EFBE8091EB10909109
:10DC9000EC10EFB6F8940E94332B21BA469A45B89F
:10DCA00085E488B90BB91EB951BA55E05A95F1F718
:10DCB000000021BA469A45B888B9FBB81EB951BAD6
:10DCC0009AE09A95F1F700C021BA469A45B888B90A
:10DCD0000BB91EB951BAAAE0AA95F1F700C0EFBE80
:10DCE00020910D0C30910E0C8091BC109091BD10C4
:10DCF000AA2797FDA095BA2F820F931FA11DB11DD2
:10DD0000B7FD6CC11FB7F8940097E1E0AE07B1050D
:10DD100024F08FEF9FEFA0E0B0E00E94332B21BAF8
:10DD2000469AF1E0F5B997E498B920EF2BB980EA6B
:10DD30008EB967E8462E41BA35E03A95F1F7000012
:10DD400021BA469AF5B998B930E73BB98EB941BACC
:10DD50004AE04A95F1F700C021BA469AF5B998B958
:10DD60002BB98EB941BA5AE05A95F1F700C01FBFDE
:10DD70003BCE8091091190910A110FB7F8940E943F
:10DD8000332B21BA469A15B991E498B9F0EFFF2EDA
:10DD9000FBB880EA8EB9A7E87A2E71BA25E02A95F9
:10DDA000F1F7000021BA469A15B998B9B0E7EB2E01
:10DDB000EBB88EB971BA3AE03A95F1F700C021BAE2
:10DDC000469A15B998B9FBB88EB971BA4AE04A9526
:10DDD000F1F700C00FBF8091F3109091F410DFB6FF
:10DDE000F8940E94332B21BA469A15B985E488B974
:10DDF000FBB802EA0EB971BA55E05A95F1F7000086
:10DE000021BA469A15B988B9EBB80EB971BA9AE039
:10DE10009A95F1F700C021BA469A15B988B9FBB8AE
:10DE20000EB971BAAAE0AA95F1F700C0DFBEDFB65D
:10DE3000F89480E090E60E94332B21BA469A15B9F7
:10DE400083E488B9FBB80EB971BAB5E0BA95F1F7B9
:10DE5000000021BA469A15B988B9EBB80EB971BA63
:10DE6000EAE0EA95F1F700C021BA469A15B988B9F7
:10DE7000FBB80EB971BAFAE0FA95F1F700C0DFBE4F
:10DE8000B3CD21503109206E3F6F2F5F3F4F4ECCF5
:10DE900021503109206E3F6F2F5F3F4F34CC0197E7
:10DEA000806E9F6F019667CC21503109206E3F6FC5
:10DEB0002F5F3F4F4ECC9C01AD014DA05EA06FA0E7
:10DEC00078A4241935094609570969A17AA18BA1BB
:10DED0009CA15DD190583C01E7CD033008F0D2CD34
:10DEE0000E9474188D819E81892B09F423C18F8132
:10DEF0009885892B09F42EC189859A85892B09F487
:10DF00001DC18B859C85892B09F404C1B301A20135
:10DF1000440F551F661F771F440F551F661F771F3D
:10DF20006B01FF24D7FCF094EF2C80912F1190917E
:10DF30003011A0913111B0913211C816D906EA06FC
:10DF4000FB0679F0F6013296EE0FFF1F442443944E
:10DF5000512C4C0E5D1EE40DF51D808191810E94B7
:10DF60001A17013009F078C0E12FFF27E7FDF0957F
:10DF7000E753FF4EC082C0922F11D0923011E09231
:10DF80003111F09232117ECDEFEFFFEFF093000DE3
:10DF9000E093FF0CF093110EE093100E25CD0E943C
:10DFA000734114CD4F8458880415150508F46DC0CD
:10DFB00089899A896B887C888619970908171907B7
:10DFC00008F066C09A01AB012419350941095109CD
:10DFD000698D7A8D8B8D9C8DDAD0E6CC80E090E0D7
:10DFE000DC0190CE00911D0C10911E0C1093951029
:10DFF000009394100E94FC2142E0B80180E090E080
:10E000000E94612CE3CC8091110C9091120CE09154
:10E010000001F0910101A0910401B091050160910E
:10E020000201709103019B01209530952817390753
:10E03000D0F50FEF1FE710939710009396100E94F2
:10E040000F156FEF81E00E94365941E060E070E00B
:10E05000C8010E94612CBACCB701A601812F0E9491
:10E06000BA2389CF00E010E02AEF33E440E050EE1D
:10E070006BEA76E40E948D189093000D8093FF0C5C
:10E080009093110E8093100EAFCC80E090E08CCC7A
:10E09000C30169887A88860D971D8017910708F15A
:10E0A00080E090E881CC8617970788F16C01E12C1D
:10E0B000F12C8F010A1B1B0B80179107F8F4A701A5
:10E0C0009601261B370B4109510960910601709199
:10E0D0000701809108019091090159D08C011058D5
:10E0E000AACF9A01AB01281B390B4109510969A13B
:10E0F0007AA18BA19CA14BD0905856CCBD016E0F3C
:10E100007F1F6817790760F100E010E094CF00E00E
:10E1100010E891CF73016201CC0CDD1CEE1CFF1CDA
:10E12000C40CD51CE61CF71C6701FF24D7FCF09437
:10E13000EF2CFBCEC12CD12C7601F7CEB301A2017E
:10E14000440F551F661F771F6B01FF24D7FCF09407
:10E15000EF2CEBCE6301FF24D7FCF094EF2CE5CE3F
:10E16000A7019601261B370B4109510960910A014D
:10E1700070910B0180910C0190910D0108D0905885
:10E18000ADCFFCD4B7FF0895821B930B0895DB013C
:10E190008F939F93B4D4BF91AF91A29F800D911D97
:10E1A000A39F900DB29F900D11240895991B79E0C3
:10E1B00004C0991F961708F0961B881F7A95C9F717
:10E1C0008095089597FB072E16F4009406D077FDEE
:10E1D00008D0A5D407FC05D03EF4909581959F4FBB
:10E1E0000895709561957F4F08955058BB27AA27D1
:10E1F0000ED0C9C192D130F097D120F031F49F3FB9
:10E2000011F41EF462C10EF4E095E7FB58C1E92F4A
:10E21000DCD180F3BA17620773078407950718F0FB
:10E2200071F49EF5F4C10EF4E0950B2EBA2FA02DDB
:10E230000B01B90190010C01CA01A0011124FF27B3
:10E24000591B99F0593F50F4503E68F11A16F040AE
:10E25000A22F232F342F4427585FF3CF46953795AD
:10E260002795A795F0405395C9F77EF41F16BA0B72
:10E27000620B730B840BBAF09150A1F0FF0FBB1F20
:10E28000661F771F881FC2F70EC0BA0F621F731F69
:10E29000841F48F4879577956795B795F7959E3FC6
:10E2A00008F0B3CF9395880F08F09927EE0F979554
:10E2B0008795089541D1E39577C10CD064C134D1DD
:10E2C00040F02BD130F021F45F3F19F0F8C051112C
:10E2D0009FC1FBC07AD198F39923C9F35523B1F3B9
:10E2E000951B550BBB27AA2762177307840738F0C5
:10E2F0009F5F5F4F220F331F441FAA1FA9F333D024
:10E300000E2E3AF0E0E830D091505040E695001CD7
:10E31000CAF729D0FE2F27D0660F771F881FBB1F93
:10E32000261737074807AB07B0E809F0BB0B802D6D
:10E33000BF01FF2793585F4F2AF09E3F510568F0B9
:10E34000BEC066C15F3FECF3983EDCF386957795DF
:10E350006795B795F7959F5FC9F7880F911D9695BB
:10E36000879597F90895E1E0660F771F881FBB1F17
:10E37000621773078407BA0720F0621B730B840BC4
:10E38000BA0BEE1F88F7E095089519F40EF097C0C8
:10E390003EC19BC022D1C8F39638C0F707F80F9250
:10E3A000E8942BE33AEA48EB5FE7BAD10F920F9279
:10E3B0000F924DB75EB70F9272D1ECEAF0E088D0C1
:10E3C0004F915F91EF91FF91E595EE1FFF1F49F08F
:10E3D000FE57E0684427EE0F441FFA95E1F7419598
:10E3E000550B29D10F9007FE1DC10895F6D088F076
:10E3F0009F5790F0B92F9927B751A0F0D1F0660F31
:10E40000771F881F991F1AF0BA95C9F712C0B1304B
:10E4100081F0FDD0B1E00895FAC0672F782F8827EA
:10E42000B85F39F0B93FCCF3869577956795B3958A
:10E43000D9F73EF490958095709561957F4F8F4FF9
:10E440009F4F0895E89409C097FB3EF490958095FE
:10E45000709561957F4F8F4F9F4F9923A9F0F92FAA
:10E4600096E9BB279395F695879577956795B79528
:10E47000F111F8CFFAF4BB0F11F460FF1BC06F5F0E
:10E480007F4F8F4F9F4F16C0882311F096E911C020
:10E49000772321F09EE8872F762F05C0662371F041
:10E4A00096E8862F70E060E02AF09A95660F771F55
:10E4B000881FDAF7880F9695879597F9089597F949
:10E4C0009F6780E870E060E008959FEF80EC08951A
:10E4D000DF93CF931F930F93FF92EF92DF927B0115
:10E4E0008C01689405C0DA2EEF0118D1FE01E89482
:10E4F000A5912591359145915591AEF3EF0187DEB8
:10E50000FE019701A801DA9479F7DF90EF90FF9070
:10E510000F911F91CF91DF91089500240A94161650
:10E52000170618060906089500240A941216130601
:10E53000140605060895C9CF50D0E8F3E894E0E04A
:10E54000BB279F57F0F02AED3FE049EC06C0EE0FE5
:10E55000BB0F661F771F881F28F0B23A6207730748
:10E56000840728F0B25A620B730B840BE3959A95DB
:10E5700072F7803830F49A95BB0F661F771F881F9B
:10E58000D2F7904894C1092E0394000C11F488230B
:10E5900052F0BB0F40F4BF2B11F460FF04C06F5F5B
:10E5A0007F4F8F4F9F4F0895EF93E0FF06C0A2EA81
:10E5B0002AED3FE049EC5FEB2ADEE5DF0F900394A4
:10E5C00001FC9058E4EDF0E07EC157FD9058440FF7
:10E5D000551F59F05F3F71F04795880F97FB991FC2
:10E5E00061F09F3F79F0879508951216130614067F
:10E5F000551FF2CF4695F1DF08C01616170618060C
:10E60000991FF1CF86957105610508940895E894E6
:10E61000BB2766277727CB0197F9089522D108F405
:10E620008FEF08959B01AC0160E070E080E89FE30C
:10E6300044CE45CF3AC1D1DFE8F39923D9F3940F03
:10E64000511DBBF39150504094F059F0882332F0A3
:10E65000660F771F881F91505040C1F79E3F5105AC
:10E6600044F7880F911D9695879597F908955F3F18
:10E67000ACF0983E9CF0BB27869577956795B7954B
:10E6800008F4B1609395C1F7BB0F58F711F460FF20
:10E69000E8CF6F5F7F4F8F4F9F4FE3CFB9CFFA0126
:10E6A000DC01AA0FBB1F9B01AC01BF5728F4222736
:10E6B0003327442750781FC0B75188F4AB2F00246C
:10E6C000469537952795011CA395D2F3002069F054
:10E6D000220F331F441FB395DAF30DD086CD61307E
:10E6E0007105A0E88A07B94630F49B01AC016627A2
:10E6F000772788279078309621F0208331834283D2
:10E70000538308950BD03FCF08DF28F00DDF18F0BA
:10E71000952309F0D4CED9CE11247ACF56DFA0F3B9
:10E72000959FD1F3950F50E0551F629FF001729FA6
:10E73000BB27F00DB11D639FAA27F00DB11DAA1FC5
:10E74000649F6627B00DA11D661F829F2227B00D12
:10E75000A11D621F739FB00DA11D621F839FA00D9D
:10E76000611D221F749F3327A00D611D231F849FED
:10E77000600D211D822F762F6A2F11249F57504044
:10E780008AF0E1F088234AF0EE0FFF1FBB1F661FDF
:10E79000771F881F91505040A9F79E3F510570F098
:10E7A0008ECE36CF5F3FECF3983EDCF386957795BF
:10E7B0006795B795F795E7959F5FC1F7FE2B880F93
:10E7C000911D9695879597F90895FA01EE0FFF1F11
:10E7D00030962105310599F16115710561F4803894
:10E7E000BFE39B0749F168949038810561F0803858
:10E7F000BFEF9B0741F0992342F5FF3FE10531054B
:10E80000210511F1E8940894E795D901AA2329F488
:10E81000AB2FBE2FF85FD0F310C0FF5F70F4A6954A
:10E82000E0F7F73950F019F0FF3A38F49F779F93EB
:10E830000CD00F9007FC905808953EF046CE60E053
:10E8400070E080E89FE308954FE79F775F934F93D1
:10E850003F932F934ED02F913F914F915F9152DF75
:10E8600099CD990F0008550FAA0BE0E8FEEF161698
:10E870001706E807F907C0F012161306E407F507B4
:10E8800098F0621B730B840B950B39F40A2661F028
:10E89000232B242B252B21F408950A2609F4A140CB
:10E8A000A6958FEF811D811D08959F3F31F09150F6
:10E8B00020F4879577956795B795880F911D969564
:10E8C000879597F908959F938F937F936F93FF9305
:10E8D000EF939B01AC0116DFEF91FF91F9DD2F91D2
:10E8E0003F914F915F910ECF0EF0DFCFEECD689448
:10E8F000E6CD73DEC8F39923D1F3C6F3DF93CF934C
:10E900001F930F93FF92C92FDD2788232AF02197A9
:10E91000660F771F881FDAF720E030E040E85FEBF2
:10E920009FE3883920F0803E30F021968F775EDCBF
:10E93000E2EFF0E003C05ADCEFE1F1E0C9DD8B016A
:10E94000BE01EC01FB2E6F5771097595771F880B7F
:10E95000990B7ADD28E132E741E35FE3DFDEAF2D9B
:10E960009801AE01FF900F911F91CF91DF914FDC85
:10E970000ACEFB01DC0104C08D910190801921F4C5
:10E9800041505040C8F7881B990B0895FB01DC01EA
:10E9900002C001900D9241505040D8F70895681779
:10E9A000790768F4FB01DC01E40FF51FA40FB51F24
:10E9B00002C002900E9241505040D8F70895E6CF21
:10E9C000DC0101C06D9341505040E0F70895FB0118
:10E9D000DC010D900020E9F7119701900D920020C5
:10E9E000E1F70895FB01DC0101900D920020E1F7B1
:10E9F00008958F929F92AF92BF92CF92DF92EF9243
:10EA0000FF92CF93DF93EC01688179818A819B81AA
:10EA1000611571058105910521F464E279ED8BE5BD
:10EA200097E02DE133EF41E050E08DD049015A01EC
:10EA30009B01AC01A7EAB1E462D06B017C01ACEEB2
:10EA4000B4EFA501940167D0C60ED71EE81EF91ECB
:10EA5000F7FE06C081E0C81AD108E10880E8F80A8C
:10EA6000C882D982EA82FB82E894F7F8B601C7012E
:10EA7000DF91CF91FF90EF90DF90CF90BF90AF905C
:10EA80009F908F900895B5CF8CE991E0B2CF6093BD
:10EA90009C0170939D0180939E0190939F01089526
:10EAA000FB019F01E8944230BCF04532ACF44A309F
:10EAB00029F497FB1EF4909581959F4F642F77273B
:10EAC0002ED0805D8A330CF0895D8193CB01009755
:10EAD000A9F716F45DE251931082C90100C0DC0170
:10EAE000FC01672F71917723E1F7329704C07C9185
:10EAF0006D9370836291AE17BF07C8F308953ED03F
:10EB0000A59F900DB49F900DA49F800D911D112481
:10EB10000895B7FFF4CFF3DF821B930B0895AA1B70
:10EB2000BB1B51E107C0AA1FBB1FA617B70710F0F8
:10EB3000A61BB70B881F991F5A95A9F7809590952A
:10EB4000BC01CD010895052E97FB16F4009406D064
:10EB500057FD0CD01FD007FC09D07EF4909580950E
:10EB6000709561957F4F8F4F9F4F089550954095B9
:10EB7000309521953F4F4F4F5F4F0895A29FB001B1
:10EB8000B39FC001A39F01D0B29F700D811D1124BE
:10EB9000911D0895A1E21A2EAA1BBB1BFD010DC0F9
:10EBA000AA1FBB1FEE1FFF1FA217B307E407F5073D
:10EBB00020F0A21BB30BE40BF50B661F771F881F19
:10EBC000991F1A9469F760957095809590959B01AF
:0CEBD000AC01BD01CF010895F894FFCF07
:10EBDC0000809001000C000000000000000000808C
:10EBEC000000000800000000000000000000000011
:10EBFC000000000000000000000000000000000009
:10EC0C000000000000000000000000000030223670
:10EC1C006D247D20390F7646104010523F065B4F15
:10EC2C00666D7D077F6F4848614843277B777F3946
:10EC3C003F79713D76060E763837373F733F776DE7
:10EC4C00783E3E7E76665B39640F230802777C58EB
:10EC5C005E79716F74040C743837545C7367506D43
:10EC6C00781C1C7E766E5B39300F010001000000B1
:10EC7C0000006207640E3415D21B41228128942EA9
:10EC8C007B34383ACB3F37457B4A994F925467597E
:10EC9C001A5EAB621A676A6B9B6FAD73A2777B7B54
:10ECAC00387FD9826186CF89258D6290889398961A
:10ECBC009199759C449FFFA1A6A43AA7BBA92AAC25
:10ECCC0088AED5B011B33DB559B766B964BB54BD68
:10ECDC0036BF0BC1D2C28CC43AC6DCC772C9FDCADE
:10ECEC007CCCF1CD5BCFBBD011D25ED3A1D4DBD524
:10ECFC000CD734D854D96DDA7DDB85DC86DD80DE2B
:10ED0C0073DF5FE044E123E2FCE2CEE39BE461E5E8
:10ED1C0022E6DEE695E746E8F2E89AE93DEADBEA28
:10ED2C0074EB0AEC9BEC28EDB1ED36EEB8EE36EF59
:10ED3C00B0EF27F09AF00BF178F1E2F149F2ADF275
:10ED4C000EF36DF3C9F322F479F4CDF41FF56FF5DE
:10ED5C00BCF507F651F698F6DDF620F761F7A0F74B
:10ED6C00DEF71AF854F88DF8C4F8F9F82DF95FF9B4
:10ED7C0090F9C0F9EEF91BFA47FA71FA9BFAC3FA4B
:10ED8C00EAFA10FB35FB58FB7BFB9DFBBEFBDEFB65
:10ED9C00FDFB1BFC38FC55FC70FC8BFCA5FCBFFC84
:10EDAC00D8FCF0FC07FD1EFD34FD49FD5EFD72FD37
:10EDBC0086FD99FDABFDBDFDCFFDE0FDF0FD01FE37
:10EDCC0010FE1FFE2EFE3CFE4AFE58FE65FE72FE35
:10EDDC007EFE8AFE96FEA2FEADFEB7FEC2FECCFE05
:10EDEC00D6FEE0FEE9FEF2FEFBFE04FF0CFF14FF74
:10EDFC001CFF23FF2BFF32FF39FF40FF47FF4DFF66
:10EE0C0053FF59FF5FFF65FF6BFF70FF75FF7BFFC3
:10EE1C0080FF84FF89FF8EFF92FF96FF9BFF9FFF71
:10EE2C00A3FFA7FFAAFFAEFFB1FFB5FFB8FFBBFF63
:10EE3C00BFFFC2FFC5FFC8FFCAFFCDFFD0FFD2FF87
:10EE4C00D5FFD7FFDAFFDCFFDEFFE0FFE3FFE5FFD6
:10EE5C00E7FFE9FFEAFFECFFEEFFF0FFF1FFF3FF46
:10EE6C00F5FFF6FFF8FFF9FFFBFFFCFFFDFFFFFFCF
:10EE7C000000EE01DA03C305A9078C096C0B4A0DDF
:10EE8C00250FFD10D212A414741641180B1AD31BA3
:10EE9C00981D5A1F1A21D72291244926FE27B129E1
:10EEAC00612B0E2DB92E62300832AB334D35EB365B
:10EEBC008738213AB93B4E3DE03E7140FE418A43D2
:10EECC0013459A461F48A149224B9F4C1B4E944F09
:10EEDC000C518152F4536455D3563F58A959115BC8
:10EEEC00775CDB5D3D5F9C60FA615663AF640766DF
:10EEFC005C67B068016A516B9E6CEA6D346F7B7015
:10EF0C00C171057347748775C57602783C79757A3B
:10EF1C00AC7BE17C147E457F7580A381CF82F98325
:10EF2C00218548866D879188B289D28AF18B0D8DA7
:10EF3C00288E418F59906F9183929693A794B69592
:10EF4C00C496D197DB98E599EC9AF29BF79CFA9DC5
:10EF5C00FB9EFB9FFAA0F7A1F2A2ECA3E5A4DCA513
:10EF6C00D2A6C6A7B9A8AAA99AAA88AB76AC61AD55
:10EF7C004CAE35AF1CB003B1E7B1CBB2ADB38EB470
:10EF8C006EB54CB629B705B8DFB8B8B990BA67BB3F
:10EF9C003CBC10BDE3BDB4BE85BF54C022C1EEC1A4
:10EFAC00BAC284C34DC415C5DCC5A2C666C729C880
:10EFBC00ECC8ADC96DCA2BCBE9CBA5CC61CD1BCEB2
:10EFCC00D4CE8DCF44D0FAD0AFD162D215D3C7D323
:10EFDC0078D427D5D6D584D630D7DCD786D830D9B7
:10EFEC00D9D980DA27DBCCDB71DC15DDB7DD59DE56
:10EFFC00FADE9ADF39E0D7E074E110E2ACE246E3E6
:10F00C00DFE378E410E5A6E53CE6D1E665E7F9E751
:10F01C008BE81CE9ADE93DEACCEA5AEBE7EB74EC82
:10F02C0000ED8AED14EE9EEE26EFAEEF35F0BBF060
:10F03C0040F1C4F148F2CBF24DF3CEF34FF4CFF4E0
:10F04C004EF5CCF54AF6C7F643F7BEF739F8B3F8E8
:10F05C002CF9A5F91DFA94FA0AFB80FBF5FB6AFC66
:10F06C00DDFC50FDC3FD34FEA5FE16FF85FFF4FF4D
:10F07C00001D93070000000000000000020099072B
:10F08C00A307AD07B6070000001AC0070000000078
:10F09C0000000000001BC80700000000000000007A
:10F0AC000019D00700000000000000000202DA077F
:10F0BC00E407ED07F607FE070114060800090F0820
:10F0CC001308170800161B080000000000000000C1
:10F0DC00001C210800000000000000000017280898
:10F0EC000000000000000000001D9307000000005D
:10F0FC00000000000201310839083C083A08000001
:10F10C00010A3E0848084C0800000000020551089E
:10F11C005B0848084C085F08011764086C08700805
:10F12C000000000002037408E407ED07F607FE0771
:10F13C0002047E0889088D08910895080112990827
:10F14C009E0848084C0800000116A308A908AE0840
:10F15C00B70800000018BE08000000000000000006
:10F16C001E00181D0C0D1F010203040506070809DB
:10F17C000A0B191B1A1CFFFFFFFFFFFFFFFF80018B
:10F18C00C000A800900080006000480030002400FF
:10F19C00180012000C000900060004000300020015
:10F1AC00010000FFFFFFFFFF080C080A0808080811
:10F1BC0008080808080A080C0C0000000000080CDD
:10F1CC000A0A0A0A0A0C0C0857095C096009640946
:10F1DC0068096C097009740978097C09800985092A
:10F1EC008A098F09940999099E097472616E73706A
:10F1FC00203D20000000000000000203020000017E
:10F20C00000101010101000101010204081020406C
:10F21C00800101010101010101010302060201014A
:10F22C000100010204020302010201003756656F5E
:10F23C007C878B8F949AA4B0B9BFD2476C69476C0A
:10F24C0069277320503630302075706772616465A1
:10F25C0020616C7068612046656220323220323049
:10F26C003135007370656564006C666F207368617E
:10F27C0070650070756C73652D7472690072616EC7
:10F28C00642D73696E006E6F6973652D7361770001
:10F29C00566962207370640056696220616D740057
:10F2AC006D6F642064656C617900616D70207368AA
:10F2BC0061706500666173742D65787000666173AA
:10F2CC00742D6C696E00736C6F2D65787000736CA7
:10F2DC006F2D6C696E0062656E64207467740056E5
:10F2EC00636F0056636600566F6C00676C696465EB
:10F2FC0000646574756E6500616D702056656C6F89
:10F30C00006C666F207467740061620061006C664B
:10F31C006F2072616E6765006C6F77006869676853
:10F32C00006D6F642072616E6765006D696E0066BA
:10F33C00756C6C006D6F6420746774006C666F0084
:10F34C005669620066696C2073686170650062655D
:10F35C006E642072616E676500326E640033726495
:10F36C0000357468004F6374007072696F006C61D3
:10F37C007374007069746368006672656500736508
:10F38C006D69746F6E65006F6374615665006669B4
:10F39C006C2056656C6F00203D2000636C656172BB
:10F3AC000072657374007469650020726563760081
:10F3BC002073656E640062656E6465722063616CB7
:10F3CC00696272617465640056632D0056632D206A
:10F3DC006F66660056632D206F6E007072657365E4
:10F3EC0074732064756D70656400496E7420737954
:10F3FC006E63004D6964692073796E63007461708B
:10F40C00652073796E6300737072656164200020EF
:10F41C002F20566366206C696D20006261736963EE
:10F42C00207061746368006F6D6E690063683100F1
:10F43C0063683200636833006368340063683500C6
:10F44C0063683600636837006368380063683900A6
:10F45C0063683130006368313100636831320063B6
:10F46C006831330063683134006368313500636898
:04F47C003136000025
:020000021000EC
:10E000002F923F924F925F926F927F928F929F9248
:10E01000AF92BF92CF92DF92EF92FF920F931F9336
:10E02000CF93DF93CDB7DEB72A970FB6F894DEBF54
:10E030000FBECDBF2FEF31EE44E0215030404040C5
:10E04000E1F700C00000F89414B817B81AB81DB86A
:10E0500010BA15B890EE98B91BB81EB883EE81BB04
:10E060002FEF24B997B947E04AB99DB980BB36EC88
:10E0700031BB469A97B94AB99DB915B880E888B9B5
:10E080001BB81EB8F7E4F1BB52E05A95F1F700C097
:10E0900086B189B18CB131BB479AE7EEE7B977EF2A
:10E0A0007AB962EE6DB931BB469AA1E0A5B982E4B6
:10E0B00088B91BB81EB887E881BB8DE08A95F1F757
:10E0C000000031BB469A97B94AB99DB9A5B920E479
:10E0D00028B91BB82EB9F1BBB2E0BA95F1F700C070
:10E0E00086B159B1BCB131BB479AE7B97AB96DB9BC
:10E0F000BDE0BA95F1F7000031BB469A97B94AB92D
:10E100009DB9A5B928B91BB82EB9F1BBF2E0FA95B3
:10E11000F1F700C026B199B14CB131BB479AE7B9CC
:10E120007AB96DB93DE03A95F1F70000422F469576
:10E13000437060E8269F90011124242B392F307101
:10E14000322B292F269526952870232B969590768D
:10E15000922B907C21E0903C09F020E0382F3695FE
:10E160003370A0E88A9FC0011124832B952F9071F2
:10E17000982B852F869586958870982B852F869568
:10E180008076982B907C81E0903C09F080E082239F
:10E1900009F4B4C286EC81BB469A21E025B990E42B
:10E1A00098B99BB91EB897E891BBBAE0BA95F1F758
:10E1B00000C081BB469A25B934E438B930E73BB991
:10E1C00032E23EB991BBEAE0EA95F1F700C081BBCB
:10E1D000469A25B922E428B920E52BB920EC2EB9BE
:10E1E00091BBFAE0FA95F1F700C081BB469A15B8E9
:10E1F00026E828B923E02BB91EB891BBAFE9BFE0F0
:10E200001197F1F700C0000081BB469A15B823E8CA
:10E2100028B923E12BB922E02EB991BBBAE0BA9517
:10E22000F1F700C081BB469A20EE27B997E09AB972
:10E230002DB915B870E878B99BB91EB867E461BB11
:10E24000E2E0EA95F1F700C036B139B13CB181BBEB
:10E25000479A57EE57B947EF4AB932EE3DB9F5E064
:10E26000FA95F1F7000081BB469A27B99AB92DB902
:10E2700015B878B99BB990E29EB961BB22E02A95A6
:10E28000F1F700C096B199B19CB181BB479A57B9DB
:10E290004AB93DB935E03A95F1F7000099249394D5
:10E2A000612C712C0F2EF1E94F2EF4E15F2EF02D31
:10E2B0000F2EF1E92F2EF5E13F2EF02D88248394C7
:10E2C0009FD499230CF405C2803F9105C9F798D4D7
:10E2D000892B09F0FEC194D48136910509F0F9C16A
:10E2E0008FD4469709F0F5C18BD48B36910509F090
:10E2F000F0C186D499230CF4ECC1A3015827052E54
:10E300000294202D2F702527352F3025330F307E96
:10E310002327302D3527307F3695052E000C331FEF
:10E320005695569556955F7153275427422F7A017B
:10E330008F7799278C011695102F00271795079531
:10E340005FD499230CF4C5C1D701B8270B2E0294D2
:10E35000202D2F702B273B2F3025330F307E232786
:10E36000302D3B27307F36950B2E000C331FB69592
:10E37000B695B695BF71B327BA27A22F7D018F77C7
:10E380009927082B192B0115B1E01B0721F0012B50
:10E3900009F4A1C19EC134D46C0199230CF499C134
:10E3A00087011827012E0294802D8F708127912FCD
:10E3B0009025990F907E8927902D9127907F969593
:10E3C000012E000C991F1695169516951F71192789
:10E3D0001027082F15D45C0199230CF47AC1F80199
:10E3E000F8270F2E0294802D8F708F279F2F902556
:10E3F000990F907E8927902D9F27907F96950F2EBD
:10E40000000C991FF695F695F695FF71F927FE27F2
:10E41000E82FFA87E9878201F3D399230CF4F4C03B
:10E42000E984FA84A7015827052E0294202D2F7025
:10E430002527352F3025330F307E2327302D3527E4
:10E44000307F3695052E000C331F56955695569500
:10E450005F7153275427422F7A015A874987DC017D
:10E46000AF77BB27BA83A983CBD399230CF4CCC055
:10E47000F701F8270F2E0294202D2F702F273F2F02
:10E480003025330F307E2327302D3F27307F3695C0
:10E490000F2E000C331FF695F695F695FF71F327B6
:10E4A000FE27E22F7F01FA87E9879C012F77332728
:10E4B0003C832B83A5D399230CF4A6C0A70158272E
:10E4C000052E0294202D2F702527352F3025330F50
:10E4D000307E2327302D3527307F3695052E000CD2
:10E4E000331F5695569556955F7153275427422FE3
:10E4F0007A015A874987DC01AF77BB27BE83AD839A
:10E500007FD399230CF480C0F701F8270F2E0294D3
:10E51000202D2F702F273F2F3025330F307E2327BC
:10E52000302D3F27307F36950F2E000C331FF69588
:10E53000F695F695FF71F327FE27E22F7F01FA8704
:10E54000E9879C012F77332738872F8359D3992365
:10E550000CF45AC0A7015827052E0294202D2F70C5
:10E560002527352F3025330F307E2327302D3527B3
:10E57000307F3695052E000C331F569556955695CF
:10E580005F7153275427422F5A874987F8013397E1
:10E590009C013695322F2227379527955981252BB7
:10E5A0002083F80132979C0122703327002436958E
:10E5B00027950794369527950794322F202D6B8148
:10E5C000262B2083F80131979C0124703327220FDA
:10E5D000331F22953295307F3227207F3227AD813D
:10E5E0002A2B20838870992782959295907F98276F
:10E5F000807F9827BF818B2BF80180830C5F1F4F92
:10E600000215130509F008CFFBD299230CF461C061
:10E610008C01102F0027110FF3D299230CF459C04D
:10E620008F779927880F991F880F991F082B192B0F
:10E63000E7D299230CF44DC083709927082B192B2E
:10E6400029853A850217130709F043C0D9D2873FBD
:10E65000910509F03EC0990C3FE3391508F4982C58
:10E6600046EC41BB469A892D880F392D3695282FC7
:10E6700026702064992D991F9927991F292B992D70
:10E680009071482F440F4072942B807C982B832FDD
:10E690008270806285B828B99BB98EB957E851BBA2
:10E6A0006AE06A95F1F700C0B5016F777727C60178
:10E6B0008F7799279695982F882797958795682B18
:10E6C000792B762F662780E090E04EE854E198D4CD
:10E6D000F7CD89E701C08DE696EC91BB469A982F5D
:10E6E0009071906E86958270806221E025B922E457
:10E6F00028B99BB98EB987E881BBFFCF2A960FB6A0
:10E70000F894DEBF0FBECDBFDF91CF911F910F9167
:10E71000FF90EF90DF90CF90BF90AF909F908F9041
:0EE720007F906F905F904F903F902F900895E4
:10EC000045E04A95F1F70000349B04C000C000C005
:10EC10003499FCCF86EC81BB469A20EE27B997E069
:10EC20009AB92DB915B820E828B99BB91EB897E450
:10EC300091BB52E05A95F1F700C096B129B13CB1B1
:10EC400081BB479A87EE87B987EF8AB982EE8DB983
:10EC500085E08A95F1F70000392F3695337040E84A
:10EC6000949FC0011124832B922F9071892B922F96
:10EC7000969596959870892B26952076282B217B42
:10EC8000213809F040C026EC21BB469A90EE97B996
:10EC900087E08AB99DB915B890E898B98BB980E238
:10ECA0008EB987E481BB52E05A95F1F700C036B1C6
:10ECB00099B14CB121BB479A87EE87B987EF8AB9E2
:10ECC00082EE8DB985E08A95F1F70000832F869555
:10ECD000837050E8359F90011124282B892F807173
:10ECE000282B892F869586958870282B9695907667
:10ECF000292B50E0CA01880F991F84709927822B15
:10ED0000282F30E002C02FEF3FEF822F932F08957E
:10F000008F929F92AF92BF92CF92EF92FF92CF9347
:10F01000DF93EA01CFB6F894F999FECF23E0FB0124
:10F0200080935B002093570010D707B600FCFDCFFC
:10F03000DE01B3954B015C0121E04881F980E12CB0
:10F04000F701E40FF11DAF0122960A01F401A0922D
:10F050005B0020935700F9D61124F2E08F0E911C2B
:10F06000A11CB11CAC17BD0741F725E0FB01809343
:10F070005B0020935700E9D607B600FCFDCF81E185
:10F0800080935700E2D6CFBEDF91CF91FF90EF90F3
:0CF09000CF90BF90AF909F908F9008959C
:00000001FF
